:020000040800F2
:20000000EC190020430500088D0400084D130208910400089304000895040008000000008B
:200020000000000000000000000000009704000899040008000000009B0400089D04000828
:200040009F040008A1040008A3040008A5040008A7040008A9040008AB040008AD04000810
:20006000AF040008B1040008B3040008B5040008B7040008B9040008BB040008BD04000870
:20008000BF040008C1040008C3040008C5040008C7040008C9040008CB040008CD040008D0
:2000A000CF040008D1040008D3040008D5040008D7040008D9040008DB040008DD04000830
:2000C000DF040008E1040008E3040008E5040008E7040008E9040008EB040008ED04000890
:2000E000EF040008F1040008F3040008F5040008F7040008F9040008FB040008FD040008F0
:20010000FF04000801050008030500080505000807050008090500080B0500080D05000848
:200120000F05000811050008130500081505000817050008190500081B0500081D050008A7
:200140001F05000821050008230500082505000827050008290500082B0500082D05000807
:200160002F05000831050008330500083505000837050008390500083B0500083D05000867
:080180003F05000841050008DD
:020000040800F2
:20020000DECEA5ED020030784634303700000000000000000000445453325F3230303800CF
:200220000000000000004170706C69636174696F6E0000000000000000000000000000004A
:20024000000000000000040AFE00DAF7DECEA5ED02003078463430370000000000000000F8
:20026000000053504C6174436F6E74726F6C6C6572004170706C69636174696F6E00000022
:200280000000000000000000000000000000000000000000FE00DAF701000208180000006C
:2002A000D50A020818000000ED110208030000002918020806000000511D02080900000060
:2002C000252002080200000071230208100000002D250208FF000000112C02080C00000071
:2002E000B52F020800000000F1310208050000005157020812000000795A02080A00000034
:20030000D95D02080A0000008D66020814000000196B020808000000317202080700000038
:20032000D978020810000000C17C020813000000618E020813000000C5BA0208160000004D
:2003400031110308170000000D3E030816000000413F0308170000000951030815000000B1
:200360002F49072291438D462E492F480A1A06D00722914381F30988022282F314882B48A3
:200380002B492C4A00F039F82B482C492C4A00F034F82C482C492D4A00F02FF82C482D4977
:2003A0002D4A00F02AF82D482D492E4A00F025F82D482E492E4A00F020F82E482E490022C9
:2003C00000F026F82D482E49091A082903DB00220260043001601F481F49884205D0026800
:2003E000043003B4904703BCF7E700208646EC4600200021234A9047FEE7884207D0521A09
:2004000005D0037801300B700131013AF9D17047884202D002700130FAE770471A48704702
:20042000EC190020EC210020EC190020F0B70308880100204C020020000002080000020868
:20044000F0860308F0B7030888010020880100209C0500089C0500089C0500089C05000873
:200460009C0500089C050008F0860308F0860308F0B703084C020020A0160020EC16002010
:20048000EC16002025400208FFFFFFFFFEE7FEE7FEE7FEE7FEE7FEE7FEE7FEE7FEE7FEE7DD
:2004A000FEE7FEE7FEE7FEE7FEE7FEE7FEE7FEE7FEE7FEE7FEE7FEE7FEE7FEE7FEE7FEE7EC
:2004C000FEE7FEE7FEE7FEE7FEE7FEE7FEE7FEE7FEE7FEE7FEE7FEE7FEE7FEE7FEE7FEE7CC
:2004E000FEE7FEE7FEE7FEE7FEE7FEE7FEE7FEE7FEE7FEE7FEE7FEE7FEE7FEE7FEE7FEE7AC
:20050000FEE7FEE7FEE7FEE7FEE7FEE7FEE7FEE7FEE7FEE7FEE7FEE7FEE7FEE7FEE7FEE78B
:20052000FEE7FEE7FEE7FEE7FEE7FEE7FEE7FEE7FEE7FEE7FEE7FEE7FEE7FEE7FEE7FEE76B
:20054000FEE71348854600F022F84EF68850CEF20000016851F47001016000BF00BF00BFED
:20056000F1EE100A50F04070E1EE100A4FF0000080F314884EF63C71CEF20001086850F0F9
:1C05800040700860034804490160FFF7E9BE70470000022008ED00E000000008FB
:020000040801F1
:200000000000000000000000000000000000000000000000000000000000000000000000E0
:2000200000000000000000000000000000000137830035F4301E00000A83011F014413F594
:200040003183012BF5330000F4030057000000F40300FC000000094A004AFF51008F1500C6
:200060008F1600430742068F21008F14FF680020F406F40220140085F40700006400728372
:200080000125800070420743064AFF710044244A03710844257000442270084423AE00966E
:2000A00026AE01962AAE02962EAE039632AE049636AE05963A45210C018200BD0C4421F5A5
:2000C00035F406F402451460002000D7F5358100D70C018200D70C4521128100E7F407007C
:2000E000006400C38000576900204515451655510045165F009417AF008000891E0000647F
:2001000083011F014513128100FC44131E00006483011F0145131282010AF5318000FC70CE
:200120000A4A0F52096E012080012B6001200134F5390009F5390109211D1407FFFFFFFF4C
:20014000FFFFFFFFFFFFFFFFFFFFFFFFFFFFFFFFFFFFFFFFFFFFFFFFFFFFFFFFFFFFFFFFBF
:20016000FFFFFFFFFFFFFFFFFFFFFFFFFFFFFFFFFFFFFFFFFFFFFFFFFFFFFFFFFFFFFFFF9F
:20018000FFFFFFFFFFFFFFFFFFFFFFFFFFFFFFFFFFFFFFFFFFFFFFFFFFFFFFFFFFFFFFFF7F
:2001A000FFFFFFFFFFFFFFFFFFFFFFFFFFFFFFFFFFFFFFFFFFFFFFFFFFFFFFFFFFFFFFFF5F
:020000040801F1
:020000040802F0
:2000000030B583B04FF0000400944FF0F8050195204621464FF007024FF0010303F062FB77
:200020004FF00100294614F02FF94FF00300214640F27502C0F6020204F020FB4FF001008A
:2000400040F28501C0F6020140F26502C0F6020204F014FB48F20C70C0F6030008F0BCF8BE
:2000600003B030BD08B519B94FF0030015F016F808BD00BF08B5012903D14FF0010015F078
:200080000DF808BD08B54FF00A0001F013FF08BD4FF0020303704FF004000870704700BFE0
:2000A000A0F10203DBB2032B2FD8A0F1020003281FD8DFE800F00209101740F25420C2F2F0
:2000C000000003680B601AE040F25420C2F2000043680B6013E040F27440C2F200000368E8
:2000E0000B600CE040F27440C2F2000043680B6005E04FF00F0010704FF0000070474FF011
:20010000000111704FF0010070474FF0000070474FF0060303704FF004000870704700BF84
:20012000A0F10603DBB2032B2FD8A0F1060003281FD8DFE800F00209101740F25C20C2F25F
:20014000000003780B701AE040F25C20C2F2000043780B7013E040F28040C2F20000037803
:200160000B700CE040F28040C2F2000043780B7005E04FF0050010704FF0000070474FF05E
:20018000000111704FF0010070474FF0000070474FF0050303704FF001000870704700BF08
:2001A000052809D159B140F29813C2F20003187808704FF0010070474FF0000070474FF066
:2001C00001007047002810DA6FEA90414FEA81424FEA924303F1010300EE103AF8EEC00A41
:2001E000FDEE007A20EEA70A70474FEA904000EE100ABBEECF0A704710F4004F10D080F433
:200200007F4181F0F002C2F30B1303F1010307EE903AB8EEE70ADFED060A20EE200A7047CF
:20022000C0F30B1000EE100ABBEECE0A704700BF000080BD0000000070B52DED028B06469C
:20024000B0EE408AD0ED007A9FED1D7AF4EEC77AF1EE10FA06DC9FED1B0AF4EEC07AF1EE42
:2002600010FA02D586ED008A1CE017EE900A15F077F90FA3D3E9002315F010FB04460D4652
:2002800018EE100A15F06CF90BA3D3E9002315F005FB02460B462046294615F0BBF915F016
:2002A0007BF93060BDEC028B70BD00BFAFF30080CDCCCCCCCCCCEC3F9A9999999999B93F73
:2002C00000007A4400007AC470B5064640F25023C2F200031B689A6812F0020F17D148F29B
:2002E0009F65C0F2010540F25024C2F2000402F02BF92368986810F0020F08D105F1FF352F
:2003000002F022F92368996811F0020F01D01E7370BD02F019F923689A6812F0020FF6D138
:20032000023DE4D1F3E700BF70B548F2A065C0F2010540F25026C2F2000633689C6802F021
:2003400003F924F07F00C1B251B105F1FF353268946802F0F9F824F07F03D8B2002868D175
:2003600040F6E425C2F2000555E8003F03F1010345E80032012AF7D040F26021C2F2000158
:20038000086808F029FF40F25022C2F20002136818686FF38610186055E8003FA3F10103F4
:2003A00045E80032012AF7D055E8003FB3F1004F0DD14FF0000345E80032012AF4D04EF6CB
:2003C0000450CEF20000016841F080510160BFF32F8F14F0010F17D148F29F65C0F20105DB
:2003E00040F25024C2F200042668B66802F0ACF816F0010F08D105F1FF3521688E6802F0D3
:20040000A3F816F0010F0AD040F25023C2F200031968087B0A6842F040030B6070BD2268E8
:20042000966802F091F816F0010FEDD1023DDBD1EAE7013D81D193E7F8B507EE100ABBEE44
:20044000C87ADFED737A27EE270A10EE100A15F087F804460D465AA3D3E9002315F01EFA29
:2004600059A3D3E9002315F0D5F815F095F815F077F815F09BFD15F08FF815F071F854A33B
:20048000D3E9002315F0C4F815F086F815F068F851A3D3E9002315F0B7FA15F07DF800EEE3
:2004A000100AB5EEC00AF1EE10FA40F18880204629464BA3D3E9002315F0F0F94AA3D3E95A
:2004C000002315F0A5F806460F462046294648A3D3E9002315F0E2F902460B4620462946C9
:2004E00015F0DCF902460B463046394615F092F806460F46204629463FA3D3E9002315F0C9
:20050000CDF902460B462046294615F0C7F902460B462046294615F0C1F902460B463046A6
:20052000394615F075F806460F462046294634A3D3E9002315F0B2F902460B462046294680
:2005400015F0ACF902460B462046294615F0A6F902460B462046294615F0A0F902460B463A
:200560003046394615F054F806460F462046294625A3D3E9002315F091F902460B4620468A
:20058000294615F08BF902460B462046294615F085F902460B462046294615F07FF902463F
:2005A0000B462046294615F079F902460B463046394615F02FF814F0EFFF00EE100AF8BD35
:2005C00033AC91FDADCD58BEA9628CDD6270F23E1C64ED4A2602703FFC9D375F364BB3BEF9
:2005E000F163CC5D4BC80140713D0AD7A3406E40BB82C87D062F653F93C266C7E03DD43EFE
:20060000CE563151E2425E3E3EFAE46127F3E43D0000C943AFF3008038B540F26423C2F234
:200620000003187868B14FF0050540F26424C2F2000401F089FF284606F0A0FE2178002916
:20064000F7D140F26423C2F200034FF001021A7038BD00BF40F26423C2F200034FF0000231
:200660001A70704770B50E46144692F8FB30FB2B28BFFB2382F8FB3033B3FFF7CDFF3046C3
:200680004FF001010A460AF08FFB0546F0B994F8FB0070B14FF00005605DFFF715FEFFF7A9
:2006A00043FE605505F10105EDB294F8FB10A942F2D830464FF000014FF001020AF074FBFC
:2006C0000546FFF7C7FF01E04FF01605284670BD10B582B00446FFF79FFF4FF00A004FF0E0
:2006E0000C014FF00B020DF1070301F021FD40F25022C2F20002106008B900F013FD9DF86A
:200700000700214601F0FCFD44F2043360F3C50340F28441C2F200010A7842B140F27C41E9
:20072000C2F200010A7862B943F0010309E041F21001C4F202010A6812F4805F18BF43F0E9
:20074000030340F25021C2F200010A6813604FF0020303FA00F044F24021C0F20F0101FBD0
:2007600000F39DF8070049F2EC61C0F6030151F82000B3FBF0F340F26021C2F200010B60DB
:20078000106840F040031360FFF764FF02B010BD10B5072971D8DFE801F004101C28323E65
:2007A0004A5640F27C44C2F200044FF00003237047F24074C0F21B044EE040F27C41C2F28B
:2007C00000014FF000020A704FF41C64C0F20E0442E040F27C43C2F200034FF00000187045
:2007E00048F27024C0F2030436E040F27C41C2F200014FF000040C704EF290242CE040F2C7
:200800007C40C2F200004FF00102027047F24074C0F21B0420E040F27C44C2F200044FF00D
:20082000010323704FF41C64C0F20E0414E040F27C40C2F200004FF00101017048F2702484
:20084000C0F2030408E040F27C43C2F200034FF001021A704EF2902440F28440C2F20000E5
:200860004FF001010170FFF7D7FE2046FFF730FFFFF7F0FE4FF0000010BD4FF0160010BD5E
:2008800070B506460D461446FFF7C6FE3EB140F21A40C4F202004FF48061018006E040F290
:2008A0001A43C4F202034FF480521A804FF0010008F092FC45F08000FFF706FDFFF734FDD6
:2008C0004FEA1420FFF700FDFFF72EFDE0B2FFF7FBFCFFF729FD4FF0010008F07DFC40F219
:2008E0001843C4F202034FF480521A804FF480601880FFF7AFFE4FF0320008F06DFC70BDD6
:2009000070B506460D461446FFF786FE3EB140F21A40C4F202004FF48061018006E040F24F
:200920001A43C4F202034FF480521A804FF0010008F052FC45F08000FFF7C6FC2046FFF7A1
:20094000C3FCFFF7F1FC4FF0010008F045FC40F21843C4F202034FF480521A804FF4806062
:2009600018804FF0320008F037FCFFF773FE70BD38B505460C46FFF74FFE3DB140F21A4068
:20098000C4F202004FF48061018006E040F21A43C4F202034FF480521A804FF0010008F0E3
:2009A0001BFC04F07F00FFF78FFCFFF7BDFC4FF00000FFF789FCFFF7B7FC04464FF0010090
:2009C00008F00AFC40F21843C4F202034FF480521A804FF480601880FFF73CFE4FF03200C6
:2009E00008F0FAFB204638BD10B50C4605282FD140F29813C2F20003187888422BD040F250
:200A00009811C2F200010C704FF000000146FFF7AFFF024604F0010464F300024FF00000F9
:200A20004FF08001D2B2FFF76BFF4FF001004FF00001FFF79DFF034664F300034FF001001D
:200A40004FF08001DAB2FFF75BFF4FF0010010BD4FF0000010BD4FF0010010BD10B50446C5
:200A60004FF00701FFF784FF0346C3F3C01140F28042C2F20002115503F07C03191C18BF58
:200A8000012140F25C22C2F200021155003018BF012010BD10B504464FF00001FFF768FFC7
:200AA00040F0020220464FF08001D2B2FFF728FF10BD00BF10B504464FF00001FFF758FF13
:200AC00040F0200220464FF08001D2B2FFF718FF10BD00BF2DE9F04184B04FF0000440F291
:200AE0007D43C2F200031C70FFF7B4FD40F28440C2F20000047044F24020C0F20F00FFF7E1
:200B0000E7FD41F21001C4F202010A6812F4805F0ED020464FF080014FF08402FFF7F0FEF0
:200B20004FF001004FF080014FF08402FFF7E8FEFFF772FD4FF0650048F22C71C0F603017A
:200B400040F26842C2F2000209F046FF40F28810C2F200004FF0010109F0ACFF40F2901090
:200B6000C2F200004FF0010109F04CFF40F29C10C2F200004FF0010109F070FF41F21003BB
:200B8000C4F20203186810F4805F19BF40F64972C0F6020240F60552C0F602024FF000032B
:200BA000009340F26821C2F2000101914FF08000029048F26870C0F603004FF0070106F047
:200BC0007FFAFFF747FD41F21002C4F20202136813F4805F0AD16AE040463946FFF7C8FE1C
:200BE00010F00C0F14BF0024012407E04FF0000425464FF0010827464FF41676002D5ED04A
:200C0000002C71D04FF00000FFF728FF4FF00100FFF724FF4FF000004FF085014FF0F0027D
:200C2000FFF72EFE4FF001004FF085014FF0F002FFF726FE4FF000004FF083014FF4774244
:200C4000FFF71EFE4FF001004FF083014FF47742FFF716FE4FF00004254640F29811C2F23C
:200C60000001087860F3000545F0020262F06F03DDB220464FF080012A46FFF741FE4FF005
:200C800001004FF080012A46FFF73AFE20462146FFF76EFE4FF001002146FFF769FEFFF7CC
:200CA000BBFC4FF4FA7006F069FBFFF7D3FC40F27D41C2F200014FF0010008701EE0FFF760
:200CC000ABFC304608F088FA01F03EFCFFF7C2FC38463946FFF74CFE10F00C0F14BF00254E
:200CE0000125002C8AD177E7FFF796FC304608F073FA01F029FCFFF7ADFC6DE704B0BDE824
:200D0000F08100BF2DE9F84F40F27D43C2F20003187840B940F27D45C2F2000506F0FCFA7B
:200D200029780029FAD04FF0320006F027FB40F21A49C4F2020940F21848C4F2020840F2BC
:200D4000542BC2F2000B40F2744AC2F2000A40F28047C2F2000740F25C26C2F2000606F08F
:200D6000DBFAFFF759FC4FF48055A9F800504FF0010008F031FA4FF00000FFF7A5FAFFF71D
:200D8000D3FA60F31F644FF00000FFF79DFAFFF7CBFA60F317444FF00000FFF795FAFFF7C1
:200DA000C3FA60F30F244FF00000FFF78DFAFFF7BBFA60F307044FF0010008F00DFAA8F84C
:200DC00000502046FFF7FEF95846FFF735FA2046FFF712FA5046FFF72FFA04F00112B2F1E6
:200DE000011F14BF002201223A7014F4803F05D014F0060F0CBF0023012301E04FF0000327
:200E0000337006F089FA4FF0320008F0E5F94FF48065A9F800504FF0010008F0DDF94FF009
:200E20000000FFF751FAFFF77FFA60F31F644FF00000FFF749FAFFF777FA60F317444FF060
:200E40000000FFF741FAFFF76FFA60F30F244FF00000FFF739FAFFF767FA60F307044FF020
:200E6000010008F0B9F9A8F800502046FFF7AAF91148FFF7E1F92046FFF7BEF90F48FFF74F
:200E8000DBF904F00110B0F1011F14BF00200120787014F4803F05D014F0060F0CBF00211B
:200EA000012101E04FF000017170FFF7D3FB4FF0320008F091F952E7580200207804002008
:200EC00038B505460C46FFF7A7FB3DB140F21A40C4F202004FF48061018006E040F21A43A4
:200EE000C4F202034FF480521A804FF0010008F073F904F07F00FFF7E7F9FFF715FA4FF057
:200F00000000FFF7E1F9FFF70FFA4FEA00244FF00000FFF7D9F9FFF707FA24184FF001002B
:200F200008F05AF940F21843C4F202034FF480621A804FF480501880FFF78CFB4FF03200C6
:200F400008F04AF9A0B238BD2DE9F0412DED028B40F27D43C2F20003187840B940F27D44FC
:200F6000C2F2000406F0D8F921780029FAD04FF4FA7006F003FA4FF00000FFF79BFD4FF0BA
:200F80000100FFF797FD4FF00E0540F25426C2F2000643F6F678C4F21C689FED5B8A06F1C5
:200FA000040706F0B9F9284604F0DEFC002851D04FF000004FF00101FFF782FF044640F286
:200FC0004C22C2F2000210804FF00000FFF746FD18B14FF00000FFF75DFD2046FFF72CFA0B
:200FE000B4F5774F0AD24BF23863C0F60303D3ED007AB4EE670AF1EE10FA09D140F280410F
:20100000C2F200014FF001040C7000EE108A1AE0F02C06D840F25C20C2F200004FF001013C
:20102000017040F28044C2F2000422784AB940F25C23C2F200031878002818BFB0EE480A0D
:2010400001E000EE108A3046FFF7F6F84FF00000FFF730FD06F060F94FF00F0004F084FC5A
:2010600000289ED04FF001000146FFF729FF044640F24C22C2F2000250804FF00100FFF78F
:20108000EDFC18B14FF00100FFF704FD2046FFF7D3F9B4F5774F0AD24BF23863C0F6030360
:2010A000D3ED000AB4EE600AF1EE10FA09D140F28041C2F200014FF001044C7000EE108A67
:2010C0001AE0F02C06D840F25C20C2F200004FF00101417040F28044C2F2000462784AB93D
:2010E00040F25C23C2F200035878002818BFB0EE480A01E000EE108A3846FFF79DF84FF018
:201100000100FFF7D7FC4CE7F63F1CC648F29873C0F603031A684EF60C50CEF20000026076
:20112000FEE700BF08B5FFF7F1FF00BF51E8002FBFF35F8F41E80003012B3FF4F7AF10461A
:20114000704700BF13461A462DE9F00F0B460C460D460E460F46884689468A468B46092A3B
:20116000C0F00780A0E8F80FA2F10902092ABFF4F9AF4FF0080303FB02F2144B1A449746A7
:2011800000F020B800BF00BF046000F01BB800BF80E8300000F016B880E8700000F012B83B
:2011A00080E8F00000F00EB880E8F00100F00AB880E8F00300F006B880E8F00700F002B804
:2011C00080E8F00FBDE8F00F7047134680110208EFF311804FF0800181F3118870474FF023
:2011E000000000BF80F31188704700BF30B440F20003C0F6000340F28812C0F60002D01A6E
:201200004FEAA001B1F5C47F04D81346264A9A4201D324E0FEE7254D254C601B20F0030557
:201220004FF0000340F20002C2F2000240F20001C0F6000105F10400C5F380045D589D50C0
:2012400003F10403834226D109E05C589C5003F104035C58D45003F104038342F5D14EF6B1
:201260000853CEF2000340F20002C2F200021A604FF0B501CBF26B1141F2EC60C2F200008B
:2012800001604EF61453CEF200031A6842F01001196030BC7047002CD7D05C589C5003F137
:2012A00004038342D1D1DAE700000008040000088B01000830B4034600283FD002F11004EC
:2012C00040F20000C2F2000040F82430002A0ADA12F10C0F36DB02F10C024EF61850CEF2F2
:2012E000000011542EE04EF20015CEF200054CB211EA240438BF80244EF20041CEF2000163
:2013000054541346002AB8BF02F11F034FEA631005EB80014FF01F03C8F200031340002B5D
:2013200005DA03F1FF3262F01F0303F1010358B24FF0010202FA00F30B6003E0002AC7DBE8
:20134000014DD4E730BC704780E100E01EF0040F0CBFEFF30880EFF3098020E9F00F00F0E7
:2013600001B800BF10B5026841F2A063C2F200031A604168596082689A60C168D96002694C
:201380001A614169596182699A61C169D961026A1A62416A5962826A9A62C16AD962026B1B
:2013A0001A63416B5963826B9A63C16BD96300F1400018644EF62850CEF2000002685A64A5
:2013C00017F056F9002800F0FB8148F29C70C0F6030017F053F94EF62C54CEF200042368BE
:2013E000002B05DA48F2AC70C0F6030017F046F94EF62C51CEF20001086810F0020F05D0B6
:2014000048F2BC70C0F6030017F038F94EF62852CEF200025478002C72D048F2D470C0F687
:20142000030017F02BF94EF62853CEF20003597811F0010F05D048F2E470C0F6030017F0F7
:201440001DF94EF62850CEF20000427802F00204E3B22BB148F60400C0F6030017F00EF9CE
:201460004EF62851CEF20001487800F00402D4B22CB148F62800C0F6030017F0FFF84EF674
:201480002853CEF20003597801F00800C2B22AB148F64C00C0F6030017F0F0F84EF6285403
:2014A000CEF20004637803F01001C8B228B148F66C00C0F6030017F0E1F84EF62852CEF275
:2014C0000002547804F02003D9B229B148F68C00C0F6030017F0D2F84EF62850CEF20000F2
:2014E000427802F08004E3B253B14EF63851CEF20001096848F6AC00C0F6030017F0BEF8C4
:201500004EF62850CEF20000428894B2002C5ED048F6CC00C0F6030017F0B0F84EF62853B4
:20152000CEF20003598811F0010F05D048F6DC00C0F6030017F0A2F84EF62850CEF2000031
:20154000428802F00204A3B22BB148F60810C0F6030017F093F84EF62851CEF200014888A9
:2015600000F0040294B22CB148F62C10C0F6030017F084F84EF62853CEF20003598801F048
:20158000080082B22AB148F66C10C0F6030017F075F84EF62854CEF20004638803F48071F6
:2015A00088B228B148F69C10C0F6030017F066F84EF62852CEF20002548804F4007399B2FE
:2015C00029B148F6B810C0F6030017F057F84EF62850CEF200000278002A63D048F6D010AB
:2015E000C0F6030017F04AF84EF62854CEF20004237813F0010F05D048F6E010C0F60300FB
:2016000017F03CF84EF62851CEF20001087800F00202D4B22CB148F60020C0F6030017F01C
:201620002DF84EF62853CEF20003197801F00800C2B22AB148F61820C0F6030017F01EF8DE
:201640004EF62854CEF20004237803F01001C8B228B148F63C20C0F6030017F00FF84EF66F
:201660002852CEF20002147804F02003D9B229B148F66020C0F6030017F000F84EF62850F4
:20168000CEF20000027802F08004E3B253B14EF63451CEF20001096848F68020C0F603006F
:2016A00016F0ECFF41F2A064C2F20004216A48F6AC20C0F6030016F0E1FF616A48F6C0202D
:2016C000C0F6030016F0DAFFA16A48F6D420C0F6030016F0D3FFE16A48F6E820C0F603005A
:2016E00016F0CCFF216848F6FC20C0F6030016F0C5FF616848F61030C0F6030016F0BEFFF0
:20170000A16848F62430C0F6030016F0B7FFE16848F63830C0F6030016F0B0FF216948F694
:201720004C30C0F6030016F0A9FF616948F66030C0F6030016F0A2FFA16948F67430C0F62C
:20174000030016F09BFFE16948F68830C0F6030016F094FF216B48F69C30C0F6030016F0FF
:201760008DFF216C48F6B030C0F6030016F086FF616B48F6C430C0F6030016F07FFFA16BA7
:2017800048F6E830C0F6030016F078FF41F2E860C2F20000026848F60C40C0F6030011468A
:2017A000126816F06BFF40F6D423C2F200031A6848F62440C0F603001146126816F05EFF4A
:2017C000FFF7B0FC10BD00BF00B505F04BFF002808BF5DF804FBEFF30981EFF3118221E9B9
:2017E000F40F5DF804EB1EF0100F08BF21ED108A41F804ED0B4C2268002A18BF516005F054
:20180000A3FF2268516851F804EB1EF0100F08BFB1EC108AB1E8F40F82F3118881F30988D1
:2018200070470000E816002008B541F2C970C0F602004FF0FF016FF00102FFF73BFD08BD5E
:20184000F8B507460C461E460799089D14F0030F00D0FEE722B1A4EB8500A0F1480401E023
:2018600004F14800012D01D8A16205E02A4601F0CDFCA7EB8507A7624FF0000363604FF0A7
:201880001130E0624FF0223121634FF0333262634FF04433A3604FF05530E0604FF06631B3
:2018A00021614FF0773262614FF08833A3614FF09930E0614FF0AA3121624FF0BB32626227
:2018C0004FF0CC33A363E663069820644FF0807161646FF00202226005F11200F8BD00BF03
:2018E00062B64EF60453CEF200031A6842F08050186000BF43F64003C4F202031A6861F3AA
:201900005D721A60704700BF4FEA001048F63C43C0F603031A5849F2E461C0F6030151F851
:20192000220070472DE9F04F8BB083468A46914698469DF950709DF954609DF958509DF97C
:201940005C1000919DF960200192FFF7DDFF036848F63C41C0F6030101EB0B1BDBF8042026
:20196000012A02D0022A34D119E01C46C3F340310991C3F300310891C3F303210791C3F375
:2019800081110691C3F3C2010591C3F380010491C3F34001039103F00101029119E043F301
:2019A0000F44C3F340710991C3F300710891C3F303610791C3F381510691C3F3C2410591F3
:2019C000C3F380410491C3F340410391C3F300410291BAF1000FA4BF0AF0010ACDF808A017
:2019E000B9F1000FA4BF09F00109CDF80C90B8F1000FA4BF08F00108CDF81080002FA4BF64
:201A000007F007070597002EA4BF06F003060696002DA4BF05F00F05079500990029A4BF9F
:201A200001F00101089101990029A4BF01F001010991012A02D0022A35D11AE0029A62F34D
:201A40000004039961F34104049A62F38204059961F3C504069A62F38714079961F30B2466
:201A6000089A62F30C34099961F34D3464F30F0319E0029A62F30004039961F34104049A8E
:201A800062F38204059961F3C504069A62F38714079961F30B24089A62F30C34099961F3D0
:201AA0004D3464F31F4303600BB0BDE8F08F00BF38B504460D46FFF727FF48F63C43C0F6D2
:201AC000030303EB04146168012902D0022903D101E0856038BD456138BD00BF10B540F22A
:201AE0000403C4F202031A681A6040F20441C4F202010C6848F62862C0F60302506824EA3B
:201B0000000448F6FC43C0F60303586804430C6040F60401C4F202010868086040F60441CE
:201B2000C4F202010C68D06824EA0004D86804430C6041F20401C4F202010868126920EA55
:201B400002001B6940EA03040C6041F20441C4F202010868086041F60403C4F202031A68DE
:201B60001A6041F60444C4F202042168216042F20400C4F202000368036040F20C01C4F2F3
:201B800002010C6848F6B442C0F60302106824EA000448F68C43C0F60303186804430C6059
:201BA00040F20C41C4F202010C68506824EA0004586804430C6040F60C01C4F202010C68CC
:201BC000906824EA0004986804430C6040F60C41C4F202010C68D06824EA0004D8680443C7
:201BE0000C6041F20C01C4F202010868126920EA02001B6940EA03040C6041F20C41C4F232
:201C000002010868086041F60C03C4F202031A681A6041F60C44C4F202042168216042F26B
:201C20000C00C4F20200036803604FF0000440F21402C4F20202146048F68453C0F6030388
:201C4000596840F21440C4F20200016040F61402C4F202021460D96840F61440C4F2020027
:201C600001601B6941F21402C4F20202136041F21441C4F202010C6041F61400C4F2020059
:201C8000046041F61443C4F202031C6042F21402C4F20202146040F20001C4F202010C6843
:201CA00048F6CC52C0F60302106824EA000448F6A853C0F60303186804430C6040F20041E8
:201CC000C4F202010C68506824EA0004586804430C6040F60001C4F202010C68906824EA30
:201CE0000004986804430C6040F60041C4F202010C68D06824EA0004D8682043086041F201
:201D00000001C4F202010868126920EA02001B691843086041F20041C4F202010A680A60C2
:201D200041F60003C4F202031868186041F60041C4F202010A680A6042F20003C4F20203B7
:201D4000186818604FF0010003F0CAFD10BD00BF08B543F63002C4F2020213686FEA5320DC
:201D60006FEA4021116043F62003C4F201031A6842F001001860FFF7B1FE08BD2DE9F00184
:201D80009DF814709DF81860079D48F6D844C0F6030454F820004FEA4104FF2F12D0D0F8A0
:201DA0000C8048F6B04CC0F6030C1CF8077007FA04FC4FF0030707FA04F728EA07074CEA71
:201DC0000707C760FF2B10D0D0F804C048F68057C0F60307FF5C07FA01F74FF0010303FACF
:201DE00001F32CEA03033B434360FF2E0FD0876848F62063C0F603039E5D06FA04F64FF006
:201E0000030303FA04F327EA030333438360B5F1FF3F16D04FEAD10303F1080350F82360B7
:201E200001F007014FEA810105F00F0505FA01F54FF00F0707FA01F126EA0101294340F8F2
:201E40002310FF2A10D0016848F62463C0F603039B5C03FA04F34FF0030202FA04F421EA2E
:201E6000040143EA01040460BDE8F001704700BF48F65053C0F6030353F820100A6848F6F3
:201E80002053C0F6030353F820100A4048F64C63C0F6030353F82000824214BF0020012062
:201EA000704700BF48F6D843C0F6030353F820000069704748F62053C0F6030353F8203004
:201EC0007BB139B148F6F051C0F6030151F820201360704748F65C42C0F6030252F82000FF
:201EE0000360704700EB800048F67C63C0F6030353F8202049F23871C0F6030151F82200F0
:201F0000704700BF38B504460D46FFF7EBFF04EB840148F67C63C0F6030303EB8104626857
:201F200002F1FF3103290AD8DFE801F002040608456338BD856338BDC56338BD056438BDAF
:201F400040F28843C2F200031B689BB1A8B91A686FF300021A604FF00000586240F28C4145
:201F6000C2F2000108801A6842F0010018604FF0010070474FF0000070474FF00000704714
:201F800010B483B040F28843C2F200031B6803B310BB40F28C42C2F20002586A148840EA54
:201FA0000440019000BF00BF00BF00BF00BF586A148840EA04400090019C00988442ECD17D
:201FC000DDED017AB8EEE70A81ED000A4FF0010004E04FF0000001E04FF0000003B010BCAB
:201FE000704700BF40F28843C2F200031B689BB1A8B91A686FF300021A6059624FEA1141E1
:020000040802F0
:2020000040F28C40C2F2000001801A6842F0010119604FF0010070474FF0000070474FF032
:202020000000704743F67403C4F20203186847F20402C4F20002136840F28E42C2F20002D4
:202040004FF00001117013F0010F04D010464FF0040202703EE04FEA106212F0600F07D0BA
:2020600040F28E41C2F200014FF020030B7031E002F00401C9B239B140F28E40C2F20000AC
:202080004FF04002027025E0C3F3400343EAD06010F0010F07D040F28E41C2F200014FF016
:2020A00080030B7016E002F01001CBB23BB140F28E40C2F200004FF0010202700AE002F07C
:2020C0000202D0B230B140F28E41C2F200014FF002030B7043F67401C4F202010B6843F017
:2020E0008070086047F20001C4F200010A6842F008030B6041F2E860C2F20000016840F2B3
:202100009042C2F200021160704700BF40F28E43C2F200031878704708B547F61021C1F66D
:20212000FF714FF00C0214F0C1FC4FF00C0008BD2DE9F04385B00C4615461F4600EB800115
:2021400049F2DC22C0F6030252F82120D6B2122800F2BA80122C02D9122D00F2B880032E5F
:2021600000F2B88000EB800149F2DC23C0F6030303EB81010B7C002B40F0AF80122C0BD039
:2021800004EB840149F2DC23C0F6030303EB81010B7C022B40F0A480122D0BD005EB8501CD
:2021A00049F2DC23C0F6030303EB81010B7C012B40F09980122C0AD004EB840149F2DC23F7
:2021C000C0F6030353F821108A4240F08F80122D0AD005EB850149F2DC23C0F6030353F8EC
:2021E00021108A4240F085805FFA82F949F25842C0F6030252F8298000EB800049F2DC2EA6
:20220000C0F6030E0EEB80010879D1F808C04FF0000300934FF003020192C9680291614654
:20222000FFF7ACFD122C13D004EB840449F2DC23C0F6030303EB84042079A1684FF0000317
:2022400000934FF003020192E4680294FFF796FD122D13D005EB850549F2DC22C0F6030219
:2022600002EB85052879A9684FF0010300934FF003020192EC680294FFF780FDB9F1020F70
:202280000ED0B9F1030F14D0B9F1010F19D143F64400C4F20200016841F48053036010E023
:2022A00043F64003C4F20203186840F480421A6007E043F64000C4F20200026842F40041FE
:2022C0000160C7B13E7016E04FF0000813E04FF0000810E04FF000080DE04FF000080AE0AB
:2022E0004FF0000807E04FF0000804E04FF0000801E04FF00008404605B0BDE8F08300BF04
:20230000012807BF4DF68063C0F2802346F64073C0F24013994238BF0B4649F2EC62C0F6FD
:20232000030252F82010B1FBF3F3802B0ED8402B0FD8202B10D8102B11D8082B12D8042B06
:2023400013D8022B94BF0020012070474FF0070070474FF0060070474FF0050070474FF0E7
:20236000040070474FF0030070474FF00200704710B542F20803CEF204031A6842F0100022
:20238000186042F22940C0F602004FF00F014FF03602FEF78FFF43F64001C4F202010C6880
:2023A00044F010030B6041F20004C4F2000449F26842C0F603021068206049F2FC61C0F694
:2023C0000301886913F026F815A3D3E9002313F065FA4FF000024FF00003C3F6F07313F04C
:2023E00017F913F083F841F22C03C4F20003188041F22800C4F200004FF00002028049F28D
:202400006C41C0F60301086841F20C03C4F200031860228842F00101218010BDAFF3008004
:202420002D431CEBE2362A3F684620F007018D4601B541F21003C4F200034FF000021A609B
:2024400005F020FCBDE801408546704770B50446B0F5CC7F2FD940F23233984216D940F20A
:202460006560844215D940F6CB418C4214D941F69712944213D943F22F36B44212D946F291
:202480005F639C4298BF06250ED90FE04FF001050AE04FF0020507E04FF0030504E04FF07E
:2024A000040501E04FF00505072D06D1FEF73AFE4FF0070501E04FF00005FEF789FE064679
:2024C00004EB84044FEAC40049F27041C0F6030151F83520B0FBF2F39CB2012C05D9B4F5B2
:2024E000805F04D3FEF71EFE01E04FF0020443F20000C4F2000045F25551016049F27042D9
:20250000C0F6030202EBC5052B7943F20401C4F200010B6043F20802C4F2000214604AF69E
:20252000AA2303603046FEF75DFE70BD08B543F20003C4F200034CF6CC421A604FF0C800F9
:20254000FFF784FF08BD00BF43F20003C4F200034AF6AA221A60704710B5044643F21003F9
:20256000C4F20003186810F0010F74D04FF0320006F032FE43F21001C4F200010A6812F0C6
:20258000010F68D04FF0320006F026FE43F21003C4F20003186810F0010F5CD04FF032003A
:2025A00006F01AFE43F21001C4F200010A6812F0010F50D04FF0320006F00EFE43F21003B1
:2025C000C4F20003186810F0010F44D04FF0320006F002FE43F21001C4F200010A6812F0C6
:2025E000010F38D04FF0320006F0F6FD43F21003C4F20003186810F0010F2CD04FF032006B
:2026000006F0EAFD43F21001C4F200010A6812F0010F20D04FF0320006F0DEFD43F21003E2
:20262000C4F20003186810F0010F14D04FF0320006F0D2FD43F21001C4F200010A6812F0C6
:20264000010F08D04FF0320006F0C6FD43F21003C4F200031B682046FFF7F8FE10BD00BF06
:2026600002469CF8043043B1DCF8000040B140F29441C2F2000141F82200DCF8000050B99D
:2026800040F29443C2F2000353F8220049F64042002808BF104670474FF00000704700BF9B
:2026A00070B50D4649F20C53C0F6030353F82040002C45D000EB800040F2D046C2F20006F3
:2026C00006EBC00630464FF0000104F061FA122D07D142F20431C4F201010A6842F48003DB
:2026E0000B60606B65F304006063E36C4FF0050006F072FDA16841F08042A260236813F001
:20270000020FFBD0E46C122D16D142F20430C4F2010001686FF39651016042F20002CEF23F
:20272000040213684FEA03504FEA105140F2194291420CBFA4006400304604F037FB01E042
:202740004FF0FF34204670BD10B52DED028B08EE101A49F2D044C0F6030404EB8004F7EE84
:20276000007AB4EEE78AF1EE10FA09DC084613F0A7FA00289FED210A18BFB0EE408A01E00D
:20278000B7EE008A2378012B1CD16078FFF7AAFB90ED0B1A6478F8EE411A21EE888A18EEFD
:2027A000100A12F0DDFE4FF000024FF00003C3F6E07312F02FFF12F099FE01462046FFF727
:2027C000A1FB18E0022B16D16478DFED0D0A28EE208A18EE100A12F0C3FE4FF000024FF06F
:2027E0000003C3F6E07312F015FF12F07FFE01462046FFF75DF9BDEC028B10BD0000000039
:2028000000F07F4510B54FF000044FF000002146FFF79AFF4FF001002146FFF795FF40F264
:202820000C03C4F202031A681A6040F20C40C4F202000168016040F60C03C4F202031A6850
:2028400049F2AC40C0F60300816822EA010249F21850C0F6030081680A431A6040F60C430F
:20286000C4F202031A681A6041F20C00C4F202000168016041F20C43C4F202031A681A60A7
:2028800041F60C00C4F202000168016041F60C43C4F202031A681A6042F20C00C4F202003E
:2028A0000168016040F20003C4F202031A681A6040F20040C4F202000168016040F6000335
:2028C000C4F202031A6849F2D840C0F60300816822EA010249F24450C0F6030081680A43F9
:2028E0001A6040F60043C4F202031A681A6041F20000C4F202000168016041F20043C4F24D
:2029000002031A681A6041F60000C4F202000168016041F60043C4F202031A681A6042F298
:202920000000C4F202000168016010BD08B506280ED849F27453C0F60303195CFF290AD042
:2029400049F23C52C0F60302105CFFF7A9FE08BD4FF0FF3008BD4FF0FF3008BD10B50446B0
:20296000FFF7E4FF07EE900AB8EE677A49F27453C0F60303185D11280BD147F62A21C1F6E1
:20298000FF710A8801EE102AF8EEC11AC1EE870A03E09FED030AC7EE000A10EE900A10BD6B
:2029A00000F07F454FF00000704700BF38B50D46044600B30E2801D9FEF7B4FB49F2FC6323
:2029C000C0F6030353F8240055B1B0FBF5F14FEA114202F10103B0FBF3F0B0FBF5F502E0AD
:2029E0004FF000052A4649F23871C0F6030151F824309A62DD6238BD10B582B000918DF8AB
:202A00000420022840F0E2804FF00000FFF744FE48B1EC464FF00000FFF722FE01464FF059
:202A20000000FFF7C3FF4FF00100FFF735FE48B1EC464FF00100FFF713FE01464FF001007C
:202A4000FFF7B4FF4FF00200FFF726FE48B1EC464FF00200FFF704FE01464FF00200FFF790
:202A6000A5FF4FF00300FFF717FE48B1EC464FF00300FFF7F5FD01464FF00300FFF796FFFC
:202A80004FF00400FFF708FE48B1EC464FF00400FFF7E6FD01464FF00400FFF787FF4FF06B
:202AA0000500FFF7F9FD48B1EC464FF00500FFF7D7FD01464FF00500FFF778FF4FF00600AF
:202AC000FFF7EAFD48B1EC464FF00600FFF7C8FD01464FF00600FFF769FF4FF00700FFF7C8
:202AE000DBFD48B1EC464FF00700FFF7B9FD01464FF00700FFF75AFF4FF00800FFF7CCFDFF
:202B000048B1EC464FF00800FFF7AAFD01464FF00800FFF74BFF4FF00900FFF7BDFD48B1E7
:202B2000EC464FF00900FFF79BFD01464FF00900FFF73CFF4FF00A00FFF7AEFD48B1EC46B8
:202B40004FF00A00FFF78CFD01464FF00A00FFF72DFF4FF00B00FFF79FFD48B1EC464FF0B5
:202B60000B00FFF77DFD01464FF00B00FFF71EFF4FF00C00FFF790FD48B1EC464FF00C00F2
:202B8000FFF76EFD01464FF00C00FFF70FFF4FF00D00FFF781FD48B1EC464FF00D00FFF711
:202BA0005FFD01464FF00D00FFF700FF4FF00E00FFF772FD48B3EC464FF00E00FFF750FDC2
:202BC00001464FF00E00FFF7F1FE1EE049F2D043C0F6030313F82010012916D149F2D042DB
:202BE000C0F6030202EB8000447804EB840348F67C61C0F6030151F82340EC462046FFF76C
:202C00002FFD01462046FFF7D1FE02B010BD00BF30B587B040F2D045C2F2000549F26854C5
:202C2000C0F603042846214603F09AFF05F12800214603F095FF05F15000214603F090FF3B
:202C400043F64403C4F202031A6842F480701860196841F400751D6049F20054C0F6030425
:202C6000226842F20433C4F201031A6049F20850C0F60300016842F20405C4F201052960F4
:202C800042F20414C4F20104216049F2A842C0F60302136842F20C00C4F20100036042F2C3
:202CA0000C11C4F201010B6049F27055C0F603052C6842F21002C4F20102146042F21013B8
:202CC000C4F201031C6049F26C50C0F60300016842F22C05C4F20105296042F22C14C4F2D1
:202CE0000104216049F20452C0F60302136842F20800C4F20100036042F20811C4F201012C
:202D00000B604FF002004FF000010A46FFF774FE4FF000054FF000002946FFF715FD4FF0D6
:202D200001002946FFF710FD4FF00100FFF7B4FC50B149F23874C0F60304636849F2FC4251
:202D4000C0F60302106818604FF00200FFF7A4FC50B149F23871C0F603018D6849F2FC44E2
:202D6000C0F6030423682B604FF00300FFF794FC50B149F23872C0F60302D06849F2FC4167
:202D8000C0F603010D6805604FF00400FFF784FC50B149F23874C0F60304236949F2FC423C
:202DA000C0F60302106818604FF00500FFF774FC50B149F23871C0F603014D6949F2FC44EE
:202DC000C0F6030423682B604FF00600FFF764FC50B149F23872C0F60302906949F2FC4173
:202DE000C0F603010D6805604FF00700FFF754FC50B149F23874C0F60304E36949F2FC4249
:202E0000C0F60302106818604FF00800FFF744FC50B149F23871C0F603010D6A49F2FC44F9
:202E2000C0F6030423682B604FF00900FFF734FC50B149F23872C0F60302506A49F2FC417E
:202E4000C0F603010D6805604FF00A00FFF724FC50B149F23874C0F60304A36A49F2FC4254
:202E6000C0F60302106818604FF00B00FFF714FC50B149F23871C0F60301CD6A49F2FC4406
:202E8000C0F6030423682B604FF00C00FFF704FC50B149F23872C0F60302106B49F2FC418A
:202EA000C0F603010D6805604FF00D00FFF7F4FB50B149F23874C0F60304636B49F2FC4261
:202EC000C0F60302106818604FF00E00FFF7E4FB50B149F23871C0F603018D6B49F2FC4413
:202EE000C0F6030423682B604FF001000146FEF701FD4FF001004FF00001FEF7D9FD4FF0FB
:202F00000004009401940294039404944FF00100014602462346FEF705FD48F63C45C0F61B
:202F20000305287EE9690094019402944FF002022346FEF723FF20464FF00101FEF7DAFC9D
:202F400020462146FEF7B4FD0094019402940394049420464FF0010122462346FEF7E2FCC5
:202F6000287AE9680094019402944FF002022346FEF704FFFFF746FC07B030BD10B5044610
:202F80004FF000004FF01101FFF78AFB47F62A23C1F6FF73198807EE901AB8EE670A06EE28
:202FA000900AB8EE667AC0EE070AC4ED000A4FF0010010BD30B472B649F27C53C0F6030398
:202FC0001A684EF63470CEF20000026049F28051C0F603010A684EF68853CEF200031A60D1
:202FE00049F28450C0F60300016842F20802CEF20402116049F28C53C0F60303186842F2A1
:203000000C01CEF20401086043F60003C4F202031A6842F48030186019460B6813F4003F87
:20302000FBD043F64000C4F20200026842F08051016047F20003C4F20003186840F480425B
:203040001A6049F29851C0F60301086843F60803C4F20203186049F29052C0F603021168E0
:2030600043F60040C4F20200016049F29453C0F603031A6843F60401C4F202010A6043F6C4
:203080000000C4F20200036843F0807202600146086810F0007FFBD043F60803C4F2020386
:2030A0001A684FF0020161F301021A601846036803F00C02082AFAD143F64401C4F202017D
:2030C000086840F480430B6043F63000C4F20200026842F48011016047F20003C4F2000376
:2030E0001A6842F48071196047F20403C4F200031A6842F400711960036843F4802202606D
:2031000043F61440C4F20200016848F22873C0F603031B6849F28852C0F6030210686FEA4C
:20312000000259400A4206D048F22870C0F603004178CC2904D12A4B2A49994221D344E0E9
:2031400043F60841C4F2020142F63B20C0F61900086046F67F60C4F65D400860134043F604
:203160001442C4F202021360136843F00201116043F60C40C4F20200026812F4803FFBD172
:20318000D9E7194C194D281B20F003054FF0000340F20002C1F200024BF6B401C0F603016E
:2031A00005F10404C5F380005D589D5003F10403A3420CD109E05858985003F1040358584E
:2031C000985003F10403A342F5D130BC70470028F1D05858985003F10403A342EBD1F4E7C6
:2031E00040E00308B4B80308B8B8030843E0030843F63003C4F202031A6842F4001018601D
:20320000196841F480021A60704700BF2DE9F0011546002A66D040F6E423C2F2000353E895
:20322000002F02F1010243E80024012CF7D049F2A452C0F60302146846F20846C4F202067A
:20324000346049F2A057C0F603073A6846F22843C4F202031A604FF6FF7846F2304CC4F248
:20326000020C46F23447C4F2020746F22C46C4F202061C46454534BF2B464346CCF80010B9
:2032800038603360226842F001022260ED1A4FEA8303C918C018226812F0010FFBD1002DAE
:2032A000E8D140F6E423C2F2000353E8002FA2F1010243E80024012CF7D053E8002FB2F111
:2032C000004F0DD14FF0000243E80024012CF4D04EF60450CEF20000016841F0805101601C
:2032E000BFF32F8FBDE8F001704700BF70B41646002A37D046F21045C4F202052C6814F0BF
:20330000010FFBD149F29C52C0F60302146846F20842C4F20202146046F21842C4F2020275
:20332000116046F21C41C4F20201086046F21440C4F20200066049F2A852C0F60302116853
:2033400046F21040C4F202000160026842F0010101603BB146F21040C4F20200036813F033
:20336000010FFBD170BC704743F61043C4F20203186800280DDA43F60441C4F2020140F24F
:203380002312C4F267520A6048F6AB13CCF6EF530B6043F61040C4F20200016801F00042D7
:2033A000002A14BF02200020704700BF43F61043C4F202031868002807DB43F61041C4F247
:2033C00002010A6842F000430B60704700F17840B0F5801F2CBF0020012070472DE9F04FBC
:2033E00083B006460D46FFF7F1FF002856D02846FFF7ECFF002854D0AE4255D8FDF7E8FE35
:203400000190FFF7B1FF0446002841D106F178434FEA933049F2AC52C0F6030212F80080C5
:2034200041F28830FFF798F84FF0020943F6104BC4F2020B43F60C47C4F2020749F2F05AAA
:20344000C0F6030AFFF780F8494668F3C60169F3092141F48033CBF80030386810F4803FC6
:20346000FBD15AF82820B61808F101085FFA88F8B542E7D24FF06400FFF76EF849F2EC5116
:20348000C0F60301086843F61043C4F202031860FFF78CFF0198FDF7A5FE07E04FF0020466
:2034A00004E04FF0020401E04FF00204204603B0BDE8F08FF8B507460C4616460846FFF794
:2034C00085FF002860D006F1FF302018FFF77EFF00285CD040F6E423C2F2000353E8002F8D
:2034E00002F1010243E800210129F7D0FFF73CFF054628BB49F22061C0F603010A6843F619
:203500001040C4F20200026086B107F1FF37A61943F60C41C4F202010B6813F4803FFBD1D9
:2035200017F8012F04F8012BB442F5D149F22464C0F60304206843F61041C4F202010860B5
:20354000FFF734FF40F6E423C2F2000353E8002FA2F1010243E80024012CF7D053E8002FA1
:20356000B2F1004F0DD14FF0000243E80024012CF4D04EF60450CEF20000016841F0805137
:203580000160BFF32F8F04E04FF0020501E04FF002052846F8BD00BF40F25453C2F2000397
:2035A000186849F22862C0F60302116801604FF00003036049F22C62C0F6030211684160EE
:2035C00049F2D463C0F603031A68C2614FF00D01016249F23063C0F603031A680260704743
:2035E00040F24C53C2F200031868704770B48568C668446806FB05404118196040F24C503B
:20360000C2F20000006881420CD2521890420CD340F25050C2F200000268891819604FF089
:20362000010004E04FF0000001E04FF0000070BC704700BF2DE9F0410546FEF785FF4FF05A
:203640001E044FF0000840F25456C2F200064FF00107052D26D8DFE805F0030A0F14191ED1
:203660003268936983F00200C0F340011BE03068416901F0010116E032685369C3F34001D8
:2036800011E030684169C1F3C0110CE032685369C3F3801107E03368986980F0010101F003
:2036A000010100E0414689B933685A6912F4807F10D1586910F4806F10D1384605F08CFD8A
:2036C000013CC6D14FF00000BDE8F0814FF00100BDE8F0814FF00000BDE8F0814FF00000D7
:2036E000BDE8F0812DE9F04184B014461D46072900F2AD80072A00F2AD8001EB810249F233
:203700003463C0F6030303EB8202137C002B40F0A48004EB840249F23463C0F6030303EBE5
:203720008202137C012B40F09B8049F23463C0F6030301EB810653F8262004EB840653F8A9
:2037400026309A4240F08F8040F24857C2F200073870022A15D0032A25D0012A34D143F628
:203760004000C4F20200066846F40012026040F25453C2F2000345F20047C4F200071F60EB
:2037800022E043F64000C4F20200066846F48002026040F25453C2F2000345F60007C4F2E2
:2037A00000071F6010E043F64000C4F20200066846F40002026040F25453C2F2000345F68B
:2037C0000047C4F200071F6049F23468C0F6030801EB810108EB8102107991684FF0000722
:2037E00000974FF001060196D36802934FF003023346FEF7C3FA04EB840408EB840420798B
:20380000A16800970196E26802924FF003023346FEF7B4FAFFF7C0FE45B340F25050C2F201
:2038200000000A99016040F24C52C2F200020B9B136040F25850C2F2000049F2D861C0F62D
:2038400003012A463B4607F08DF9304610E04FF000000DE04FF000000AE04FF0000007E015
:203860004FF0000004E04FF0000001E04FF0010004B0BDE8F08100BF38B5044640F254532C
:20388000C2F200031D68A86910F0020F63D0FFF783FEA96911F0020F5DD03BE040F25455D9
:2038A000C2F200052B684FF0A0021A614FF00200FFF7C0FE2868816911F0010F08D045695A
:2038C00015F4806F00F03882036843F4007202604FF0050003F052FD4FF0000516E040F2DE
:2038E0005450C2F2000001684FEA14230B614FF00300FFF79FFE38B140F25452C2F20002DF
:203900001068E4B2046101E04FF00005281C18BF012038BD4FF0000038BD4FF0000038BD76
:203920004FF0000038BD4FF0000038BD4FF0000038BD4FF0000038BD4FF0000038BD4FF044
:20394000000038BD4FF0000038BD4FF0000038BD4FF0000038BD40F25452C2F200021368CD
:203960004FF000005861196860F3492119601A6842F4807018604FF00100FFF75BFE0028C1
:20398000CBD040F25455C2F200052B684FF0A00119614FF00200FFF74DFE2868826912F00C
:2039A000010F08D0436913F4806F00F0C881016841F4007202604FF0050003F0DFFC40F28E
:2039C0005450C2F2000003684FF0000159611A6861F349221A60186840F4807119604FF012
:2039E0000100FFF727FE00289AD040F25455C2F200052B684FF0A0021A614FF00200FFF75F
:203A000019FE2868816911F0010F08D0436913F4806F00F09781026842F4007101604FF0D1
:203A2000050003F0ABFC40F25450C2F2000003684FF0000159611A6861F349221A601868BD
:203A400040F4807119604FF00100FFF7F3FD00283FF469AF40F25455C2F200052B684FF0C9
:203A6000A0021A614FF00200FFF7E4FD2868816911F0010F08D0436913F4806F00F0658136
:203A8000026842F4007101604FF0050003F076FC40F25450C2F2000003684FF0000159611C
:203AA0001A6861F349221A60186840F4807119604FF00100FFF7BEFD00283FF437AF40F2C9
:203AC0005455C2F200052B684FF0A0021A614FF00200FFF7AFFD2868816911F0010F08D04F
:203AE000436913F4806F00F03381026842F4007101604FF0050003F041FC40F25450C2F210
:203B0000000003684FF0000159611A6861F349221A60186840F4807119604FF00100FFF731
:203B200089FD00283FF405AF40F25455C2F200052B684FF0A0021A614FF00200FFF77AFDBF
:203B40002868816911F0010F08D0436913F4806F00F00181026842F4007101604FF0050038
:203B600003F00CFC40F25450C2F2000003684FF0000159611A6861F349221A60186840F4EC
:203B8000807119604FF00100FFF754FD00283FF4D3AE40F25455C2F200052B684FF0A00250
:203BA0001A614FF00200FFF745FD2868816911F0010F08D0436913F4806F00F0CF80026863
:203BC00042F4007101604FF0050003F0D7FB40F25450C2F2000003684FF0000159611A6863
:203BE00061F349221A60186840F4807119604FF00100FFF71FFD00283FF4A1AE40F2545597
:203C0000C2F200052B684FF0A0021A614FF00200FFF710FD2868816911F0010F08D04369A9
:203C200013F4806F00F09D80026842F4007101604FF0050003F0A2FB40F25450C2F20000B1
:203C400003684FF0000159611A6861F349221A60186840F4807119604FF00100FFF7EAFC0A
:203C600000283FF46FAE40F25455C2F200052B684FF0A0021A614FF00200FFF7DBFC2868AB
:203C8000816911F0010F07D0436913F4806F6BD0026842F4007101604FF0050003F06EFB63
:203CA00040F25450C2F2000003684FF0000159611A6861F349221A60186840F4807119603C
:203CC0004FF00100FFF7B6FC00283FF43EAE40F25455C2F200052B684FF0A0021A614FF0F3
:203CE0000200FFF7A7FC2868816911F0010F07D0436913F4806F3AD0026842F400710160A9
:203D00004FF0050003F03AFB40F25450C2F2000003684FF0000159611A6861F349221A608D
:203D2000186840F4807119604FF00100FFF782FC00287FF4B3AD0BE64FF0010519E04FF048
:203D40000A0516E04FF0090513E04FF0080510E04FF007050DE04FF006050AE04FF005052D
:203D600007E04FF0040504E04FF0030501E04FF0020540F24850C2F20000017801F1FF33A7
:203D8000DAB2012A3FF6B8ADA9E500BFF8B50D461446002A6FD080B2FFF76EFD002865D0D2
:203DA0004FF00300FFF746FC00285FD040F25453C2F200031868026842F4807101604FF0F1
:203DC0000100FFF737FC002850D040F25453C2F20003186814F1FF3118BF0121026861F375
:203DE0008A2202604FF0A10303614FF00200FFF721FC00283AD040F25450C2F200000168F5
:203E00008A6912F0010F31D04B6913F4806F2DD14FF0040640F25457C2F200073046FFF7A7
:203E200009FC18B304F1FF34012C27D1FDF7D0F939680A696FEA020305F8013B0A686FF329
:203E40008A220A60FDF7CEF9E8E72B681B6902E04FF004060E4D3046FFF7ECFB0028F4D1E5
:203E60000B4B1868016841F400720260D4F1010038BF0020F8BD4FF00100F8BD3868016969
:203E80006FEA010205F8012B002CC7D1E0E700BF5405002030B583B015461C461A4601ABF9
:203EA000FFF7A4FB48B1019829462246FFF76EFF00280CBF1820002001E04FF01F0003B064
:203EC00030BD00BF2DE9F84F93460D4600295DD004464FF0030840F25459C2F2000901E046
:203EE000002E40D01FFA8BF0FFF7C6FC00283DD00BF0070715F0010F4CD14046FFF79AFBB7
:203F0000002836D0072F1AD8DDB13CB1D9F8000014F8011B6FEA0103036104E0D9F8006001
:203F20004FF0FF02326107F10107BA4605F1FF3635464046FFF77EFB002845D119E02E4668
:203F400000E02E46D9F80000026842F4007101600BF1080B2BF0070B4FF00500FFF76AFBEF
:203F60000028BDD107E04FF0010004E04FF0000001E04FF0000040F25453C2F20003196810
:203F80000A6842F400730B60BDE8F88F4FF00100BDE8F88F4046FFF74DFB0028E9D0072F28
:203FA000CDD82CB9D9F800304FF0FF021A6106E0D9F8000014F8011B6FEA0103036107F123
:203FC000010705F1FF3598E7072FB8D82CB9D9F800504FF0FF022A6106E0D9F8000014F8D6
:203FE000011B6FEA0103036107F1010706F1FF3583E700BF30B583B015461C461A4601ABAF
:020000040802F0
:20400000FFF7F4FA48B128462146019AFFF75AFF00280CBF1820002001E04FF01F0003B0C7
:2040200030BD00BF08B541F2EC60C2F2000041F6EC12C2F20002131A4FF0FF314FEAA3027F
:20404000FDF780F841F6EC10C2F2000042F2EC11C2F200010A1A4FEAA2024FF0FF31A2F124
:204060002002FDF76FF802F075F940F26850C2F2000044F20001C4F202014FF480524FF081
:20408000030311F0A1F9FDF72BFC4FF0000008BDBFF36F8F704700BF49F27473C0F603035C
:2040A000185C00EB400149F6A002C0F6030252F821305B68704700BF38B549F27473C0F62B
:2040C00003031B5C03EBC30440F28052C2F2000202EB840282F8211014693CB140F2805565
:2040E000C2F200051346D2699B69A04738BD00BFF8B506460F4649F27473C0F603031D5C2F
:2041000005EBC50040F28054C2F2000404EB8004D4F810C0BCF1000F07D0E2698A4204D09F
:2041200030464FF00001A369E047E76163695BB105EBC50040F28052C2F2000202EB800298
:20414000304639469269984794F8201079B127696FB105EBC50540F28053C2F2000303EB96
:204160008505304694F82110E269AB69B847F8BD49F27473C0F60303185C00EB400149F6B2
:20418000A002C0F6030252F82130D86840F08001D960704749F27473C0F603031A5C02EB05
:2041A000420349F6A002C0F6030252F823301A6812F0800F1ABF596001200020D96841F029
:2041C0008002DA60704700BF49F27473C0F60303185C00EB400349F6A002C0F6030252F847
:2041E0002300036813F0800FFBD04160704700BFF8B5044600EB400249F6A003C0F60303FB
:2042000053F8226035686FEA0500306005F0010215F0020F1CBF42F00202D2B215F0040F8B
:2042200018BF42F0080215F0080F18BF42F0040215F4807F05D0316911F4804F18BF42F0EC
:20424000100215F0200F00D1E2B104EBC40740F28053C2F2000303EB870087688FB17168C1
:2042600004EBC40040F28053C2F2000303EB800349F2E870C0F60300005DC9B29B69B84737
:2042800000E07368F26812F0800F1CD015F0800F19D0F1686FF3C711F16004EBC40040F246
:2042A0008053C2F2000353F8203063B140F28052C2F2000202EB800249F2E870C0F6030050
:2042C000005D9169984715F0400F17D004EBC40140F28053C2F2000303EB810253686BB1B5
:2042E000084640F28051C2F2000101EB800249F2E870C0F60300005D91699847F8BD00BF54
:20430000684620F007018D4601B54FF00600FFF76FFFBDE801408546704700BF684620F0C0
:2043200007018D4601B54FF00500FFF761FFBDE801408546704700BF684620F007018D4692
:2043400001B54FF00400FFF753FFBDE801408546704700BF684620F007018D4601B54FF067
:204360000300FFF745FFBDE801408546704700BF684620F007018D4601B54FF00200FFF753
:2043800037FFBDE801408546704700BF684620F007018D4601B54FF00100FFF729FFBDE86E
:2043A00001408546704700BF2DE9F84F81468B4690461E469DF828A049F27473C0F6030311
:2043C0001D5C05EB450249F6A000C0F6030050F822409DF82C70012F14BF00270127082E32
:2043E00006D0072E02D1B8F1000F01D1FCF79AFE0AF1FF31CBB2012B01D9FCF793FE49F25D
:204400007872C0F6030252F82500B0FBFBF1A1604FF0000267F38612BAF1010F04D0002FFF
:204420000CBF0223002301E04FF0000363F30D3267F38E3222614FF06C00B8F1020F14BFDC
:204440000023012363F3492018F1000818BF4FF0010868F38A20082E18BF4FF0000868F372
:204460000C3040F40051E1604846FFF715FEBDE8F88F00BFF0B585B00D461E4649F2747305
:20448000C0F60303195C01EB410449F6A007C0F6030757F8247049F60C03C0F60303185CB3
:2044A00000EB400149F29474C0F6030404EBC1040AB1FCF737FE75B9207B21699DF82C2005
:2044C00000924FF001030193626902924FF003023346FDF753FC207861689DF82830009333
:2044E0004FF001020192A36802934FF003023346FDF744FC49F2DC70C0F603000168012D7F
:2045000014BF0025012565F3C301796105B0F0BD2DE9F843054649F27473C0F60303185C37
:2045200000EBC00240F28054C2F2000404EB820449F6A001C0F6030100EB40064FEA86030E
:2045400001EB030851F80390FCF742FE064694F82000B8B14FF00007C9F80C703846394674
:2045600098F90420FCF7A6FE28463946FFF7A4FDE3681BB12846E169A26998474FF0000271
:2045800084F820203046FCF72DFEBDE8F88300BF2DE9F04F85B005468B469246994649F254
:2045A0007473C0F603031E5C40F28058C2F2000806EBC6074FEA870708EB070406EB46005E
:2045C00049F6A001C0F6030101EB8006FCF700FE039043F64003C4F202031A6849F2F070F7
:2045E000C0F60300016822EA010249F2E070C0F6030001680A431A6043F64403C4F20203DB
:204600001A681A6049F2F871C0F6030105EB8503C818C95C4278837890F803E0CDF800E0FE
:20462000007901902846FFF725FF9DF8382000929DF83C1001912846594652464B46FFF7CA
:20464000B3FE109B48F807301298A060119A62601399E160149BA361B0684FF00F0196F9DA
:204660000420FCF727FE4FF0010084F820000398FCF7B8FD05B0BDE8F08F00BF49F2747325
:20468000C0F60303185C00EBC00340F28050C2F2000000EB830319615A61704749F60C03DB
:2046A000C0F60303185C00EB400149F61002C0F6030202EB01107047082806D9102807D9B6
:2046C00020288CBF4020202070474FF0080070474FF01000704700BF022809D0032804D02B
:2046E000012814BF0020012070474FF0030070474FF00200704700BF40F60013C5F2000313
:20470000186840F60802C5F200021168C1F34103022B12BF6FF30200032363F3020040F49B
:2047200000406FF3995040F60012C5F20002106040F60401C5F200010B6843F48070086088
:20474000704700BF49F60413C0F603031A6840F61030C5F200000260704700BF10B441F253
:204760007C03C2F200031A5CE0B14FF0000340F61861C2F200014FF04C0404FB0212D1687B
:2047800021F0030202F1040262F312034FF0010161F3DC4349F61012C0F6030202EB401093
:2047A00081690B6010BC704770B440F22003C5F200031868C0F34342022A01D0062A29D10F
:2047C00000F00F0149F6A415C0F6030555F82160C0F30A1505F1030398081BD041F20001C8
:2047E000C5F2000100F1FF3404F001040A68334672604FF0010282420ED10AE00C6803F1F0
:20480000040343F8044F0C685C6002F102028242F4D1356070BC7047002CEFD00C6803F188
:2048200004035C6002F101028242E7D1F1E700BF70B449F69013C0F6030353F82060326885
:20484000002A3CD049F61011C0F6030101EB401102F103024FEA9202CB691B689A420CD98E
:2048600040F63402C5F2000211684FF0010303FA00F008431060184623E006F10403C2B1DD
:2048800002F1FF3000F00105086953F8044B0460501E18D10DE00C691A4652F8045B25604A
:2048A00000F1FF300C695B68236002F104030138F1D14FF0000131604FF0010001E04FF0F7
:2048C000000070BC7047002DE5D00A6953F8044B14600138DFD1ECE708B54FF0010303FAD9
:2048E00000F040F27E62C2F200021388184210D023EA000340F27E60C2F200000380CA6B9F
:2049000052B1086A4FF0000103F0CAFE4FF0000008BD4FF0000008BD4FF0010008BD00BF5B
:2049200070B540F21403C5F200031C6849F6F800C0F6030001680C4200F0BB8140F60C6254
:20494000C2F200021378012B40F2B38140F21800C5F20000016849F6A012C0F603021368F3
:20496000194200F0A68140F61800C5F20000016811F0010F56D040F60815C5F200052A687F
:2049800040F60830C5F2000003682A60036041F27C01C2F20001087840F61861C2F2000151
:2049A0004FF04C0505FB001503F00100E96A0143E962C3F3C000296B0143296303F00803A4
:2049C000D8B258BBD2B212F0010F0ED01DE0EA6A22B105F1100000F063FF2BE02B6B002B7E
:2049E000F7D1686B0028F4D124E012F0900FEED040F63403C5F20003186820F0010119609A
:204A00004FF00000FFF714FFE1E76E6B4FF000002946FFF761FF30436863D8E74FF000016C
:204A2000E963CFE740F61802C5F20002136813F4803FA0D140F61801C5F200010A6802F04E
:204A4000020398B2002856D040F62815C5F200052A6840F62830C5F2000003682A6003605B
:204A600041F27C01C2F20001487840F61861C2F200014FF04C0505FB001503F00100E96AC1
:204A80000143E962C3F3C000296B0143296303F00803D8B258BBD2B212F0010F0ED01DE0A1
:204AA000EA6A22B105F1100000F0FAFE2FE02B6B002BF7D1686B0028F4D128E012F0900FE0
:204AC000EED040F63403C5F20003186820F0020119604FF00100FFF7ABFEE1E76E6B4FF026
:204AE00001002946FFF7F8FE30436863D8E74FF00001E963CFE740F61801C5F200010A68A2
:204B00004FEA124303F0020081B200299CD140F61801C5F200010A6802F0040398B2002865
:204B200056D040F64815C5F200052A6840F64830C5F2000003682A60036041F27C01C2F24D
:204B40000001887840F61861C2F200014FF04C0505FB001503F00100E96A0143E962C3F3BF
:204B6000C000296B0143296303F00803D8B258BBD2B212F0010F0ED01DE0EA6A22B105F1E8
:204B8000100000F08DFE2FE02B6B002BF7D1686B0028F4D128E012F0900FEED040F634035E
:204BA000C5F20003186820F0040119604FF00200FFF73EFEE1E76E6B4FF002002946FFF773
:204BC0008BFE30436863D8E74FF00001E963CFE740F61801C5F200010A684FEA124303F013
:204BE000040081B200299CD140F61801C5F200010A6802F0080398B258B940F61801C5F211
:204C000000010A684FEA124303F0080081B200294FD040F66815C5F200052A6840F668304E
:204C2000C5F2000003682A60036041F27C01C2F20001C87840F61861C2F200014FF04C05CC
:204C400005FB001503F00100E96A0143E962C3F3C000296B0143296303F00803D8B210B146
:204C60004FF00001E963D2B212F0010F08D06E6B4FF003002946FFF72FFE304368630EE061
:204C800012F0900F0BD040F63403C5F20003186820F0080119604FF00300FFF7C9FDEA6A0D
:204CA0001AB92B6B0BB9686B18B105F1100000F0F7FD14F0100F01D0FFF776FD14F4805FFD
:204CC0000DD040F60F61C2F200014FF001020A7040F6E053C2F20003186802F0B9F914F494
:204CE000005F01D0FFF708FD14F4006F14D040F60E60C2F200004FF00101017041F2790375
:204D0000C2F200034FF000021A7040F6E050C2F20000006802F09CF9002C14DA40F60E6149
:204D2000C2F200014FF000030B7041F27900C2F200004FF00102027040F6E051C2F20001D1
:204D4000086802F085F940F21403C5F200031C6070BD00BF684620F007018D4689B500AF82
:204D6000FFF7DEFDBD46BDE889408546704700BF2DE9F04140F61866C2F200064FF04C036D
:204D800003FB0066304650F8205F49F61018C0F603084FEA451708EB07044FF000014FF038
:204DA0001C0211F0A7FE35624FF00100B06258F807204FF00003136061690B60A0684FF09E
:204DC000FF02026061680B60A0690360E1680A6049F6A412C0F6030252F82500036049F65C
:204DE0009011C0F6030151F825201360BDE8F08100B583B04FF00003019340F21001C5F289
:204E000000010A68B0F1FF3F08BF102060F3891242F0200040F21003C5F200031860194633
:204E200040F63F52C0F20302019800F1010001900B6813F0200F02D001989042F4D94FF0EA
:204E4000030004F0C9F903B000BD00BF2DE9F8434FF04C0303FB00F040F61861C2F2000139
:204E60004418256A4FF0010606FA05F649F61012C0F6030202EB45174058002867D0A3689F
:204E8000FBB1D7F80080D8F8001011F4004F18D1D8F80020914663F30A09007AFFF71CFC42
:204EA00060F3934949F4004965F3995949F08050C0F3404363F39A60C8F800002846FFF740
:204EC00097FFE168F1B17A68106810F4004F19D12846FFF743FCD7F80480D8F80070E36839
:204EE00063F30A072168087AFFF7F6FB60F3934747F4004242F01047C7F3404060F39A6798
:204F0000C8F8007049F6A413C0F6030353F825104FF000020A60A06858B140F61C03C5F267
:204F20000003196846EA010290B2196860F30F011960E3685BB140F61C00C5F20000026851
:204F400046EA1246B6B2016866F31F410160BDE8F88300BF70B582B04FF00002019240F2A2
:204F60001003C5F20003196841F00100186001921A6812F0010F19D0019940F63F53C0F215
:204F80000303994212D840F21000C5F2000040F63F52C0F20302019901F101010191036844
:204FA00013F0010F02D001999142F4D94FF0030004F012F94FF00000019040F21002C5F2C6
:204FC00000021368002B1DDB019940F63F50C0F20300814216D84FF0030640F21005C5F226
:204FE000000540F63F54C0F20304304604F0F4F8019A02F1010201922B68002B02DB01997B
:20500000A142F2D902B070BD00B583B04FF00003019340F21000C5F20000026842F010019F
:20502000016040F63F52C0F20302019B03F101030193016811F0100F02D0019B9342F4D9D0
:205040004FF0030004F0C8F803B000BD50B149F60011C0F603010A6840F21803C5F2000366
:205060001A60704749F6FC03C0F603031A6840F21800C5F200000260704700BF38B54FF07E
:20508000000440F60063C5F200031C6040F60002C5F20002106840F0030164F3820164F36F
:2050A0000A11116040F22405C5F200052B684FF0400262F30F032B60204662F31F402146C6
:2050C00062F31F4162F30F0140F22805C5F2000529604FF0800363F30F0040F20412C5F2EC
:2050E000000210604FF0C00161F30F0040F20815C5F2000528604FF4807363F30F0040F27B
:205100000C12C5F2000210604FF0FF30FFF770FEFFF77AFF40F61000C5F20000046040F670
:205120001401C5F200010C604FF0FF3540F61803C5F200031D6040F61C02C5F200021460BA
:205140002046FFF715FE4FF00100FFF711FE4FF00200FFF70DFE4FF00300FFF709FE4FF0DB
:205160000400FFF705FE4FF00500FFF701FE4FF00600FFF7FDFD4FF00700FFF7F9FD40F260
:205180001800C5F20000046040F21401C5F200010D604FF00100FFF759FF38BD40F27E63DA
:2051A000C2F2000319884FF0010202FA00F0084000280CBF02200320704700BF40F600132A
:2051C000C5F200031B68C3F3076202F08000C1B209B143F0804343F4001040F60012C5F298
:2051E00000021060704700BF2DE9F8430546164649F61018C0F6030808EB401849F690137A
:20520000C0F6030353F820704FF0010909FA00F90C46A9B9386840B940F27E63C2F200039B
:20522000188819EA000F5AD10AE040F27E61C2F200010A8819EA020F02D02846FFF7D8FD30
:2052400006F1030107F1040388081CD000F1FF3202F0010CA4F1040151F8042F43F8042B37
:2052600001383ED10FE001F1040249681C4644F8041B00F1FF3002F1040152685A6004F110
:2052800004030138EFD13E6040F27E63C2F20003198849EA0109A3F8009065B940F6101029
:2052A000C5F2000002684FF0010161F3D44266F30602026009E0D8F8140002684FF00103E5
:2052C00063F3DC4266F312020260D8F80030186840F004421A6016B12846FFF7A9FABDE8A8
:2052E000F883BCF1000FBED051F8042F43F8042B0138B8D1C7E700BF70B5044649F6A4136F
:20530000C0F6030353F82060334653F8045BAA4238BF1546084619462A4611F0C7FB4FF086
:20532000000030602046FFF719FA49F61011C0F6030101EB441463681A6842F004401860D5
:20534000284670BDF8B5054640F61863C2F200031868002871D040F61861C2F20001CA6CCF
:20536000002A71D040F61864C2F20004D4F89860002E6DD040F61867C2F20007D7F8E430D6
:20538000002B69D040F61860C2F20000D0F83011002965D040F61862C2F20002D2F87C41F3
:2053A000002C61D040F61866C2F20006D6F8C871002F5DD040F61863C2F20003D3F8140276
:2053C000002859D040F61861C2F20001D1F86022002A55D0464E4FF00807FBF7A3FE2C7A63
:2053E000002C53D040F27C62C2F200021088014610F0020F55D04FF0010404F1010441FA0A
:2054000004F212F0010FF8D14FF0010101FA04F1084340F27C63C2F20003188044B96889F1
:20542000FFF74AF9B060A889FFF746F9F06042E06A89B260A989F1603DE040F61866C2F23E
:2054400000064FF000071EE02A4E4FF001071AE0294E4FF0020716E0284E4FF0030712E0E3
:20546000274E4FF004070EE0264E4FF005070AE0254E4FF0060706E0244E4FF0070702E090
:205480001B4E4FF00807072FA9D9A6E740F27C63C2F20003188840F0010119804FF000049A
:2054A000BDE740F0020440F27C63C2F200031C804FF00104BCE741F27C00C2F20000075508
:2054C000374647F8205B38464FF000014FF01C0211F010FB34626B68B36306F110004FF0A9
:2054E00006012A683B4600F0BBF92046F8BD00BF78100020640E0020B00E0020FC0E0020D2
:20550000480F0020940F0020E00F00202C100020022907D140F60003C5F200031A6860F31B
:205520000A121A60704700BF10B54FF0000440F63403C5F200031C6040F60400C5F20000C3
:20554000026842F0010101602046FFF711FC4FF00100FFF70DFC4FF00200FFF709FC4FF029
:205560000300FFF705FC4FF00400FFF701FC4FF00500FFF7FDFB4FF00600FFF7F9FB4FF05B
:205580000700FFF7F5FB4FF0FF30FFF731FC40F27E63C2F200031C8040F61800C5F2000022
:2055A0004FF0FF32026049F60C11C0F60301086840F61C03C5F20003186049F6F402C0F621
:2055C0000302116840F61400C5F20000016049F60813C0F603031A6840F61001C5F2000154
:2055E0000A6020464FF00201FFF792FFFFF7AAF82046FFF72BFC4FF00100FFF727FC4FF05F
:205600000200FFF723FC4FF00300FFF71FFC4FF00400FFF71BFC4FF00500FFF717FC4FF044
:205620000600FFF713FC4FF00700FFF70FFC10BD08B5FFF779FF08BD704700BFF0B585B00B
:20564000054641F28830FCF787FF002D62D043F63401C4F202010C6844F080060E604FF03A
:20566000000400944FF0030601964FF00A07029720464FF00B0132462346FCF77FFB009437
:205680000196029720464FF00C0132462346FCF775FB40F20C06C5F20006336843F04002D3
:2056A0003260FFF757FC40F23800C5F200004FF42411016044F6206003F08EFDFCF744FFA7
:2056C000336843F0400064F3082064F349204FF0050262F38D2064F35D7040F0804131608F
:2056E00044F6206003F078FDFCF72EFFFFF7C6FC40F20803C5F2000340F28110186044F644
:205700005550C0F602004FF00F014FF04302FBF7D1FD13E04FF000004FF00F014FF0430294
:20572000FBF7C8FD4FF0000340F23802C5F20002136040F21800C5F2000003602846FFF710
:205740007BFF4FF06400FCF707FF05B0F0BD00BF2DE9F04182B049F6B417C0F6030745F694
:205760003106C0F6020640F2A415C2F200054FF00408CDF8008038464FF0800132462B46D9
:2057800001F0B2FD40F28064C2F200042060CDF8008038464FF08101324605EB080301F033
:2057A000A3FD6060CDF8008038464FF08201324605F1080301F098FDA060CDF80080384642
:2057C0004FF08301324605F10C0301F08DFDE060CDF8008038464FF08401324605F11003C6
:2057E00001F082FD2061CDF8008038464FF08501324605F1140301F077FD6061CDF8008040
:2058000038464FF08601324605F1180301F06CFDA061CDF8008038464FF08701324605F168
:205820001C0301F061FDE06102B0BDE8F08100BF08B505464FF000060BE0FBF7C9FC2C68AF
:20584000616829606660FBF7CDFC22680AB1A06890472B68B3F1FF3FEFD101F0C7FBF8E78A
:205860000260B3F1FF3F18BF8360FF290ED141F2E863C2F200031A6822B192F829304FEA7D
:20588000530101E04FF007010173704701F07F010173704710B14FF000020260704700BFEB
:2058A00038B50446FBF794FC0546A4B1636893B9227B40F2A410C2F2000050F82210616006
:2058C00040F82240227B40F28063C2F2000353F8220001F0BDFB2846FBF784FC38BD00BF1B
:2058E00010B5044640F66C00C2F200004FF000014FF0240211F0FEF8D4B140F2C460C2F218
:2059000000004FF000014FF0480211F0F3F840F23C70C2F200004FF000014FF0240211F09A
:20592000E9F840F23473C2F200034FF002021A7010BD00BF38B549F6F813C0F6030353F85F
:20594000205040F2C411C2F2000151F8204049F64822C0F60302105CFCF7A4FA2840A042C7
:2059600014BF0020012038BD49F64823C0F603031A5C40F23C71C2F2000151F8222049F6E4
:20598000F813C0F6030353F8200002420CBF00200120704770B440F6E423C2F2000353E87B
:2059A000002F02F1010243E800210129F7D049F64822C0F60302155C40F66C01C2F2000158
:2059C00051F8254049F6F816C0F6030656F8202024EA020041F8250053E8005FA5F10105DB
:2059E00043E80056012EF7D053E8005FB5F1004F0DD14FF0000543E80056012EF4D04EF6C7
:205A00000450CEF20000016841F080510160BFF32F8F14420CBF0020012070BC704700BF32
:205A200049F65C23C0F60303185C704710B50446FCF738FA40F20823C2F2000353F82410FA
:205A4000484010BD10B504464FF00100FFF748FF49F6C013C0F6030353F8342040F238711D
:205A6000C2F200010A6003EBC404606840F26073C2F20003186010BD00B585B04FF000005F
:205A8000FFF7E0FF4FF00003009340F26872C2F2000201924FF04000029049F63C20C0F6A5
:205AA00003004FF0020145F64D32C0F6020201F007FB40F66803C2F20003186005B000BDF8
:205AC0002DE9F001804600283CD04FF000034FEA8302086850F823404D6855F8236086EAB5
:205AE0000407886850F8235084EA050C4CEA07076FEA070CC86850F8235026EA050707EAC9
:205B00000C0705EA0C0C66EA0C06354040F82350CD6855F82300384345F823000D6955F8A6
:205B20002300384345F823004D690DB145F8237048688558886885504868845003F1010355
:205B40004345C4D1BDE8F001704700BF2DE9F84340F23878C2F2000840F26476C2F2000667
:205B600040F2A064C2F200044FF0000540F26077C2F20007D8F8000000EB800001F0FEFB0A
:205B80003368002B40F0CF80204629464FF0240210F0B0FFC7E04FF0090049F6E011C0F602
:205BA0000301FFF78DFF40F23473C2F200031B783BB103F1FF31CBB240F66C00C2F2000059
:205BC000056040F23072C2F20002116821B940F23070C2F2000005603BB103F1FF33DBB2F9
:205BE00040F66C02C2F20002556040F23071C2F20001086820B940F23072C2F200021560C6
:205C00003BB103F1FF33DBB240F66C01C2F200018D6040F23070C2F20000026822B940F2A3
:205C20003071C2F200010D603BB103F1FF33DBB240F66C00C2F20000C56040F23072C2F2FF
:205C40000002116821B940F23070C2F2000005603BB103F1FF33DBB240F66C02C2F200020B
:205C6000156140F23071C2F20001086820B940F23072C2F2000215603BB103F1FF33DBB23F
:205C800040F66C01C2F200014D6140F23070C2F20000026822B940F23071C2F200010D603E
:205CA0003BB103F1FF33DBB240F66C00C2F20000856140F23072C2F20002116821B940F2FA
:205CC0003070C2F2000005603BB103F1FF33DBB240F66C02C2F20002D56140F23071C2F255
:205CE0000001086820B940F23072C2F2000215603BB103F1FF33DBB240F66C01C2F2000164
:205D00000D6240F23070C2F20000026822B940F23071C2F200010D6040F23470C2F20000CA
:205D20000370356026E7D4F800902846FFF77EFE40EA09012160D4F804904FF00100FFF7C7
:205D400075FE40EA09026260D4F808904FF00200FFF76CFE40EA0900A060D4F80C904FF0FA
:205D60000300FFF763FE40EA0903E360D4F810904FF00400FFF75AFE40EA09012161D4F8D1
:205D800014904FF00500FFF751FE40EA09026261D4F818904FF00600FFF748FE40EA0900B6
:205DA000A061D4F81C904FF00700FFF73FFE40EA0903E361D4F820904FF00800FFF736FE8A
:205DC00040EA09012162306800F1010030603A689042FFF4CFAEDEE600B585B04FF000031E
:205DE000009340F6D802C2F2000201924FF04000029049F66C30C0F603004FF0060145F691
:205E00001962C0F6020201F05BF940F69003C2F20003186005B000BD2DE9F04F85B040F6DE
:205E200048231E46C2F2000640F600200746C2F2000740F6B401C2F20001019101F0D6F88A
:205E40003268002AFAD061E1E359002B53D02846FFF7ECFD01996258605090434BD0E3596D
:205E600010EA030247D0039991F800E049F67439C0F603094FEA451840F69401C2F2000143
:205E80004FF6FF7C49F66C2AC0F6030A40F6DC1BC2F2000B00957046C2F10003134022EA5E
:205EA000030218B954F80B502B4221D15FEA136E04D01AF80E3003F118030EE01D0C04D01E
:205EC0001AF8053003F1100307E05FEA132E1ABF1AF80E3008331AF80330434419F803506F
:205EE00031F815E0E6451CBF0EF1010E21F815E0002AD1D1009D05F1010504F10404092DCA
:205F0000A2D1029C621E029240F0F7800399087800F10100C3B20B700B2B03D14FF000046A
:205F20000C7002E0002B40F0E58040F62422C2F20002116891B16FEA01003B6803403B607B
:205F400040F6DC15C2F200052C682040286040F62421C2F200014FF000020A6040F6242090
:205F6000C2F20000436893B16FEA03057C682C407C6040F6DC12C2F2000251680D4055605C
:205F800040F62420C2F200004FF00003436040F62425C2F20005AC6894B16FEA0400BA68DE
:205FA0000240BA6040F6DC13C2F2000399680840986040F62425C2F200054FF00004AC60E1
:205FC00040F62420C2F20000C26892B16FEA0203F9681940F96040F6DC15C2F20005EC6881
:205FE0002340EB6040F62420C2F200004FF00002C26040F62423C2F20003196991B16FEA11
:020000040802F0
:2060000001053C692C403C6140F6DC10C2F2000002691540056140F62423C2F200034FF05D
:206020000001196140F62425C2F200056C6994B16FEA04007A6902407A6140F6DC13C2F25D
:20604000000359690840586140F62425C2F200054FF000046C6140F62420C2F20000826919
:2060600092B16FEA0203B9691940B96140F6DC15C2F20005AC692340AB6140F62420C2F258
:2060800000004FF00002826140F62423C2F20003D96991B16FEA0105FC692C40FC6140F661
:2060A000DC10C2F20000C2691540C56140F62423C2F200034FF00001D96140F62425C2F2B9
:2060C00000052C6A94B16FEA04003A6A02403A6240F6DC13C2F20003196A0840186240F6AA
:2060E0002425C2F200054FF000042C624FF4FA70029002E04FF4FA7502954FF0010001F032
:206100003DF93268002A3FF499AE07E04FF4FA75029540F6D814C2F2000403944FF0000427
:20612000254691E610B54FF0000440F64823C2F200031C6040F6DC10C2F2000021464FF025
:206140000902FAF7FFFF40F60020C2F2000021464FF00902FAF7F6FF40F62420C2F2000076
:2061600021464FF00902FAF7EDFF40F6B400C2F2000021464FF00902FAF7E4FF40F69400A4
:20618000C2F2000021464FF0200210F0B3FC40F6D810C2F20000047010BD00BF70B549F69E
:2061A0004823C0F603031B5C49F6F812C0F6030252F8202040F64820C2F20000046840F6BF
:2061C0000025C2F2000555F82300104206D104F1010640F64825C2F200052E6049B140F632
:2061E000DC11C2F2000151F82350154341F8235009E040F6DC11C2F2000151F8235025EAB1
:20620000020541F82350104340F60021C2F2000141F8230040F62421C2F2000151F8230074
:2062200020EA020241F8232034B940F69003C2F20003186800F00CFF70BD00BF30B449F6DD
:206240004823C0F603031B5C49F6F812C0F6030252F8202040F60020C2F2000050F823009D
:20626000104229D040F64824C2F20004256805F10105256071B140F62421C2F2000151F8D0
:206280002340144341F8234040F6D811C2F20001097889B96FEA020240F6DC11C2F20001DC
:2062A00051F82340144041F82340024040F60020C2F2000040F8232030BC704730B40346AB
:2062C00040F6E422C2F2000252E8000F00F1010042E80004012CF7D040F69400C2F20000F1
:2062E00030F8132039B140F69401C2F200014FF0000421F8134040F6E423C2F2000353E8FB
:20630000004FA4F1010443E80045012DF7D053E8004FB4F1004F0DD14FF0000443E8004520
:20632000012DF4D04EF60450CEF20000016841F080510160BFF32F8F104630BC704700BF1F
:2063400040F6D813C2F200031878D0F1010038BF002070472DE9F84FDFF834814B4FC8EB0F
:2063600007004FEAD00707F101074FF0000540F2982AC0F6000A40F26039C0F6000931E073
:2063800044464FF000066FEA060B0BEB070101F0010B58F8043CAB4229D135E054F8043CB1
:2063A000AB4205D154F8080C8047FCF7CDF80BE0FF2B09D9FF2D07D154F8040C4FF007019D
:2063C00054F8082C00F09CFF06F1010604F1080454F8041CA94240D14CE005F10105B5F579
:2063E000807F02D0CA45CBD3F7E7BDE8F88FFF2B0FD9FF2D0DD158F8040C4FF0070158F802
:20640000082C00F07DFF04E058F8082C9047FCF79BF806F1010604F10804BE42DDD0BBF1BF
:20642000000FBBD054F8040CA8420AD0FF280DD9FF2D0BD14FF0070154F8082C00F060FF77
:2064400004E054F8081C8847FCF77EF806F1010604F10804BE42A1D1BFE7FF290FD9FF2D5D
:206460000DD154F8040C4FF0070154F8082C00F047FF04E054F8082C9047FCF765F806F163
:20648000010604F10804BE4288D1A6E767030008A0020008027840F6B123C2F200031B7824
:2064A0009A4206D34FF000020270087800F1010008700A7840F6B223C2F2000318788242F2
:2064C00024BF00200870704710B5A0F10803052B3DD8DFE803F01F3C2C3C038340F650203B
:2064E000C2F200004FF020014FF0540210F002FB40F6A420C2F200004FF0FF314FF00C028C
:2065000010F0F8FA40F6B820C2F20000026802F1010202604FF0000140F64C23C2F2000369
:20652000197040F64D20C2F20000017056E040F64C21C2F200014FF000030B7040F64D201C
:20654000C2F20000027802F1010202703CE040F64C22C2F20002127840F64D21C2F200014C
:206560000B7840F6B121C2F20001097801FB032340F65021C2F20001C95C81421DD040F6D1
:206580005024C2F20004E0544FEA531040F6A421C2F2000103F01F034FF0010404FA03F302
:2065A00051F820401C4341F8204040F6B820C2F20000016801F10101016002F1010240F68E
:2065C0004C23C2F200031A7040F64C20C2F2000040F64D21C2F20001FFF75CFF4FF00000CC
:2065E00010BD00BF70B4039D049C064628B140F6B420C2F200000078307029B140F6BC20C4
:20660000C2F20000007808702AB140F6B021C2F20001087810702BB140F6BD22C2F2000298
:20662000117819702DB140F64C23C2F20003187828702CB140F64D22C2F200021178217094
:2066400070BC704706281DD8002808BF052040F6B423C2F20003187049F69443C0F6030302
:2066600013F8101040F6B122C2F20002117003EB4000417840F6B223C2F2000319704FF03E
:20668000010070474FF00000704700BF08B540F6BC23C2F200034FF001021A704FF00500F4
:2066A000FFF7D0FF4FF00C004FF00001FFF70CFF08BD00BF08B540F64C22C2F2000210706E
:2066C00040F64D23C2F20003197010461946FFF7E1FE08BD034628B140F6B120C2F20000A8
:2066E0000078187029B140F6B223C2F20003187808702AB140F6B821C2F200010B68136071
:2067000040F65020C2F20000704700BF2DE9F00140F65027C2F200073F1853284BD8002A1B
:2067200049D03B4607F1010702F1FF3257FA82F74FF0000640F6A424C2F200044FF0010591
:206740006FEA030C0CEB070202EA050C13F8018B01F1FF3111F8012F90452FD13DE013F8E5
:2067600001CB01F1010049788C450ED003F8011C4FEA521102F01F0605FA06FC54F8216051
:206780004CEA060644F821602E4602F10102D2B2542A07D013F801CB00F10101407884456C
:2067A00042D150E03EB140F6B823C2F20003196801F101011960BDE8F001704703F8012C7C
:2067C0004FEA501600F01F0805FA08F854F8262048EA020244F826202E4600F10100C2B2E0
:2067E000542ADFD0BB42DDD0BCF1000FB7D013F801CB11F8010F84450ED003F8010C4FEAA7
:20680000521002F01F0605FA06FC54F820604CEA060644F820602E4602F10102D2B2542AC8
:20682000C0D0BB429BD1BDE703F8010C4FEA521002F01F0605FA06FC54F820604CEA0606F2
:2068400044F820602E4602F10102D2B2542AA9D0BB4284D1A6E700BF003018BF012040F69B
:20686000BC23C2F200031870003118BF012140F6B020C2F200000170003218BF012240F643
:20688000BD23C2F200031A70704700BF40F6B323C2F200034FF000021A7070474FF0540089
:2068A000704700BF40F6B323C2F200034FF001021A707047034628B10868834214BF0020D2
:2068C000012070474FF00000704700BF10B440F6E423C2F2000353E8002F02F1010243E8E8
:2068E00000210129F7D00468C4B16268824202D19268626002E043688168996023688342C9
:2069000002D15B68236002E0826841685160A26802F1FF31A1604FF00004046040F6E42326
:20692000C2F2000353E8002FA2F1010243E80024012CF7D053E8002FB2F1004F0DD14FF0E4
:20694000000243E80024012CF4D04EF60450CEF20000016841F080510160BFF32F8F10BC95
:20696000704700BF38B504460D464FF000014FF0100210F0BFF8E56038BD00BFF8B50446DF
:206980000F46C6688D192946FFF794FF00283CD140F6E423C2F2000353E8002F02F101024D
:2069A00043E800210129F7D04FF0000068606168A96001B14D60226802B925606560BC51C6
:2069C000A36803F10103A36040F6E423C2F2000353E8002FA2F1010243E80024012CF7D07A
:2069E00053E8002FB2F1004F0DD14FF0000243E80024012CF4D04EF60450CEF2000001681B
:206A000041F080510160BFF32F8FF8BD2DE9F04104468846C6688D199719C2B940F6E42353
:206A2000C2F2000353E8002F02F1010243E800210129F7D002686A6005604FF00000A86022
:206A4000616809B9656020E06B689D601DE03946FFF730FF00283FD02846FFF737FF40F66E
:206A6000E423C2F2000353E8002F02F1010243E800210129F7D0B868A8606F60BD6021681E
:206A8000B9420EBF2560A9684D6048F80640A26802F10102A26040F6E423C2F2000353E834
:206AA000002FA2F1010243E80024012CF7D053E8002FB2F1004F0DD14FF0000243E8002404
:206AC000012CF4D04EF60450CEF20000016841F080510160BFF32F8FBDE8F081C368C9180F
:206AE000486808B1C01A70474FF00000704700BF036813B1C068181A70474FF000007047B1
:206B000008B5C368C918FFF7D5FE08BD08B5C0680818FFF7DBFE08BD08B540F6C020C2F2FE
:206B200000004FF01C01FFF71DFF08BD70B5054600F108063046FFF7DBFF0446686050B15A
:206B400030462146FFF7E2FF4FF00100A861204600F07EFA70BD4FF00003AB6170BD00BF03
:206B600038B504460D464FF000014FF028020FF0C1FF204640F8085B4FF01C01FFF7F2FEE0
:206B800040F6C020C2F200002146FFF7F7FE38BD2DE9F0410746884641F2E863C2F200034D
:206BA0001868002800F0FE8040F6E424C2F2000454E8002F02F1010244E800210129F7D02A
:206BC000796831B141F2E862C2F20002136899422ED141F2E860C2F2000004687C60B969D1
:206BE00001F10101B96140F6E423C2F2000353E8002FA2F1010243E80024012CF7D053E815
:206C0000002FB2F1004F0DD14FF0000243E80024012CF4D04EF60450CEF20000016841F002
:206C200080510160BFF32F8F4FF00100BDE8F081B8F1FF3F24D140F6E423C2F2000353E851
:206C4000002FA2F1010243E80024012CF7D053E8002FB2F1004F0DD14FF0000243E8002462
:206C6000012CF4D04EF60450CEF20000016841F080510160BFF32F8F4FF00000BDE8F0813A
:206C800007F108052846FFF733FF0246F0B141F2E866C2F20006306892F8294090F82910E9
:206CA0008C4208D912E0336892F8290093F82940A04204D90AE041F2E866C2F2000628469F
:206CC0001146FFF70BFF02460028ECD1284641F2E861C2F200010968FFF798FE40F6E42654
:206CE000C2F2000656E8002FA2F1010246E80024012CF7D056E8002FB2F1004F0DD14FF015
:206D0000000246E80024012CF4D04EF60450CEF20000016841F080510160BFF32F8FB8F1F1
:206D2000000F04D008EB880000F028FB01E000F05DF940F6E424C2F2000454E8003F03F156
:206D4000010344E80032012AF7D041F2E866C2F2000628463168FFF7D9FE54E8003FA3F1C1
:206D6000010344E80032012AF7D054E8003FB3F1004F0DD14FF0000344E80032012AF4D0E4
:206D80004EF60450CEF20000016841F080510160BFF32F8F78683268904214BF00200120FF
:206DA000BDE8F0814FF00100BDE8F08110B5044641F2E863C2F200031868002860D0626881
:206DC000904201D0FAF7AEF940F6E423C2F2000353E8002F02F1010243E800210129F7D0E7
:206DE000A16901F1FF30A06118B340F6E423C2F2000353E8002FA2F1010243E80024012C2C
:206E0000F7D053E8002FB2F1004F0DD14FF0000243E80024012CF4D04EF60450CEF2000098
:206E2000016841F080510160BFF32F8F4FF0000010BD2046FFF77AFE40F6E423C2F2000342
:206E400053E8002FA2F1010243E80024012CF7D053E8002FB2F1004F0DD14FF0000243E849
:206E60000024012CF4D04EF60450CEF20000016841F080510160BFF32F8F4FF0010010BD5C
:206E80004FF0010010BD00BFF8B5054640F6E423C2F2000353E8002F02F1010243E800218E
:206EA0000129F7D040F6C020C2F20000FFF720FE0446E0B140F6C027C2F200076068A8429E
:206EC00003D12046FFF732FE0AE004F1080630462946FFF715FE18B130462946FFF716FEBF
:206EE00038462146FFF7FAFD04460028E6D140F6E423C2F2000353E8002FA2F1010243E878
:206F00000024012CF7D053E8002FB2F1004F0DD14FF0000243E80024012CF4D04EF6045006
:206F2000CEF20000016841F080510160BFF32F8FF8BD00BF08B549F6A043C0F60303195CD1
:206F4000012906D011B102290BD105E0FDF7A6FB08BD02F001F908BDFAF7E4F84FF000006C
:206F600008BD4FF0000008BD4EF60453CEF200031A6842F080501860704700BF4FF0010236
:206F800080F8282040F6E023C2F2000390F8291002FA01F2188802431A80704710B440F661
:206FA000DC23C2F200031A68C2B1904213D104E088420FD102F1140203E040F6DC22C2F20E
:206FC000000243691BB19C698169611899614369136003E00A4651690029E9D14FF00002A5
:206FE00082614FF0FF31416110BC704710B5FAF7EFF8044641F2E863C2F20003186890F8F6
:207000002820032A1BD0FAF7E3F841F2E863C2F2000319684FF0000281F8282091F82920BA
:20702000096940F6D033C2F2000343F82210FAF7D9F82046FAF7D6F8FFF796FF10BD4FF003
:20704000020180F828102046FAF7CCF810BD00BF38B5044690B3036883B3FAF7B9F80546CE
:2070600094F8280010BB2046FFF788FF41F2E861C2F200010B6843B194F8292093F829008D
:2070800020F00101531A002B15DA40F6E422C2F20002106838B140F0004140F6E423C2F2A2
:2070A0000003196007E0FFF75FFF04E0022804BF032084F828002846FAF794F838BD00BFE2
:2070C0002DE9F04F85B006460F46934698460F9DDDF84090FAF77CF8824640F62833C2F20B
:2070E00000031968504881420FD240F20002C2F2020252F82C4C54B14C4B1C468B4207D977
:2071000053F82C090028F8D102E0474C00E0464CA14206D1A1F12C0140F62832C2F2000258
:20712000116020464FF000014FF02C020FF0E2FC4FF0FF3161611EB949F6A456C0F60306EE
:207140002660B8F1000F08D00E9B042B08D9184600F103004FEA900604E04FF0000601E035
:207160004FF000060DBB42F2EC19C2F2000940F6D025C2F20005296847F2DD50C0F6020079
:207180000090CDF80480029648464FF000025B46FAF756FB2A68A260E0604FEA80015318D3
:2071A0002B60C1EB0900606020E028464FF0FF314A46F9F7C7FF4AF2ED52CDF6CE622A60B4
:2071C000E56005EB8905656047F2DD51C0F602010091CDF804800296284629464FF0010276
:2071E0005B46FAF72DFBA5EB800363606FEA0702C2F3C01101EB470707F0FF0784F82970CB
:2072000040F6E823C2F2000353F82700206143F827405046F9F7E6FF2046FFF719FF20469C
:2072200005B0BDE8F08F00BFD4FF0120A8FF012030B585B04FF0000141F2E863C2F200036B
:207240001960284C40F20005C2F202052A1B20464FEAA202F9F776FF40F6D020C2F2000088
:207260000460A5F12C0540F62831C2F200010D6041F6EC13C2F200034FF0B504CBF26B1411
:207280001C6003F14C004FF0FF3243F8042F43F8042F43F8042F8342F9D14FF00004009412
:2072A00040F62C31C2F2000101914FF02803029349F6B050C0F603004FF0070147F25D32EE
:2072C000C0F602022346FFF7FBFE40F6CC32C2F20002106040F6E820C2F20000C46305B074
:2072E00030BD00BFF021002010B584B0069C00944FF0000401940294FFF7E2FE04B010BDBD
:2073000000B585B04FF00003009301930293FFF7D7FE05B000BD00BF38B541F2E863C2F26A
:2073200000031868C0B1F9F753FF054641F2E864C2F200042068FFF721FE216891F829209D
:20734000086940F6D033C2F2000343F822002846F9F748FFFFF708FE38BD00BF38B541F2FA
:20736000E865C2F2000540F6E824C2F200042B6822681A61FFF7D0FFF9E700BF38B541F2F1
:20738000E863C2F200031968002900F0918020B9FFF7C2FF4FF001029AE0B0F1FF3F04D140
:2073A000FFF724FE4FF0000292E040F6E424C2F2000454E8002F02F1010244E80021012934
:2073C000F7D040F6DC22C2F200021568002D7AD0AB6998426FD3C01A05F114016D691DB14F
:2073E000AB698342F7D96AE041F2E865C2F200052B689861086858611846F9F797FE40F693
:20740000E424C2F2000454E8003FA3F1010344E80032012AF7D054E8003FB3F1004F0DD1FD
:207420004FF0000344E80032012AF4D04EF60450CEF20000016841F080510160BFF32F8F29
:20744000FFF7D4FD54E8003F03F1010344E80032012AF7D028684169B1F1FF3F04D0FFF7BE
:207460009DFD4FF0000201E04FF0010240F6E423C2F2000353E8004FA4F1010443E8004586
:20748000012DF7D053E8004FB4F1004F0DD14FF0000443E80045012DF4D04EF60450CEF29E
:2074A0000000016841F080510160BFF32F8F0FE04FF001020CE040F6DC21C2F20001AC6976
:2074C000221AAA6190E740F6DC21C2F200018BE7104638BDF8B5044600287AD0F9F778FE7A
:2074E000064640F62833C2F2000319683948814211D240F20002C2F2020252F81C5CA542BB
:2075000063D0354B1D468B4205D9A3F12C03D86BA042F7D15AE094F8293040F6E822C2F2E7
:20752000000252F82300A04206D1016940F6E822C2F2000242F823102046FFF72FFD204668
:20754000FFF7A2FC94F82900236940F6D031C2F2000141F8203041F2E862C2F20002106836
:20756000A04229D0A06838B3E76800EB870540F6D027C2F200073B685A1B29464FEAA2022B
:207580004FF00003FBF7B2FEE1683868A0EB81033B6040F62832C2F2000211680D4B994282
:2075A0000AD29A68954203D8E068A2EB80029A60A3F12C038B42F4D84FF00001216084F851
:2075C00028103046F9F70EFEF8BD024D21692961A1E7F8BDD4FF0120A8FF012000BFF047FA
:2075E00072B641F2E864C2F200042068FFF772FF4FF000032360FAF773F900BF40F6DC2327
:20760000C2F20003196849B1886950B100F1FF328A61D2F1010038BF002070474FF0000068
:2076200070474FF00000704770B540F6DC23C2F200031C68A4B1A06990B940F6DC25C2F276
:2076400000054FF0FF3660692946F9F76FFD66612046FFF7FDFC2C6814B1A1690029F2D0B3
:2076600070BD00BFF0B472B640F6E023C2F200031C882CB940F6CC33C2F2000318685FE02E
:2076800049F6A44CC0F6030C40F6D035C2F2000540F6E826C2F20006C4F1000323401A0AC5
:2076A0001ABF1CF8021008311CF8031011F0010F0AD141F0010055F8200038B190F8282027
:2076C000012A38D81F4602E01F4600E01F4655F82120B2B192F828307BB140F6E020C2F295
:2076E0000000048010462BE090F8283033B140F6E022C2F20002148022E010460069002876
:20770000F2D156F82100824207D1BC43C4D140F6E021C2F200010C80ACE745F8210011F09D
:20772000010FD4D114EA4703D1D04FEA4707BFB241F00101CBE740F6E021C2F200010C8056
:2077400062B6F0BC704700BF70B541F2E863C2F200031B6883420FD193F82820012A9CBF14
:20776000022283F8282093F8291040F6D030C2F2000040F8213070BD40F6D422C2F20002DC
:20778000136041F2E861C2F20001086090F8292040F6D033C2F2000343F8220090F82810FF
:2077A00001299CBF022180F828108268AAB9C1684AF2ED53CDF6CE630868984201D0F9F780
:2077C000B1FC41F2E862C2F2000211684868CB6898427ED2F9F7A6FC70BD40F6D823C2F29F
:2077E00000031B68984274D093B3586842F2EC14C2F20004251A4FEAA501D96041F6EC1267
:20780000C2F2000290420AD34FF0B503CBF26B1341F6EC10C2F2000004689C4201D0F9F7DF
:2078200081FC40F6D825C2F200052A6840F6D024C2F2000420685168D2684FF00003FBF7BC
:2078400055FD296823688B60C86803EB8002226041F2E861C2F200010B6840F6D820C2F227
:2078600000000360DA68002A33D0586899684FF00103FBF73BFD41F2E866C2F20006356830
:20788000A868EC6800EB840440F6D026C2F200063268131B21464FEAA3024FF00003FBF7EA
:2078A00025FDE9683068A0EB8102326040F62833C2F200031968074B99420AD29A68944273
:2078C00003D8E868A2EB80029A60A3F12C038B42F4D870BDD4FF012000B585B040F66C501B
:2078E000C2F200004FF00001FFF73CF840F61440C2F200004FF00001FFF734F84FF0000388
:20790000009340F62C42C2F2000201924FF05000029049F6B850C0F60300194647F62D42BB
:20792000C0F60202FFF7CCFB40F61043C2F20003186005B000BD00BF08B5FFF7D9F803461A
:2079400048B1C06850B100F1FF31D960D1F1010038BF002008BD4FF0000008BD4FF00000C9
:2079600008BD00BF70B505460E46144640F6E423C2F2000353E8002F02F1010243E80021C5
:207980000129F7D0FFF7B4F80246002839D0C06884422DD3241A28461146FFF79FF8024615
:2079A00000282ED0C068A042F4D921E040F6E423C2F2000353E8002FA2F1010243E8002486
:2079C000012CF7D053E8002FB2F1004F0DD14FF0000243E80024012CF4D04EF60450CEF2A0
:2079E0000000016841F080510160BFF32F8F70BDF460D1680B1BD36028463146FFF706F85F
:207A0000D4E7F46028463146FEF7B8FFCEE700BFF8B50646FFF76CF80446F8B1C368EBB93D
:207A200030462146FFF75AF80546F9F7D1FB074630462146FFF76AF83846F9F7D3FB2269D1
:207A40001AB130462146FFF78DFF04F11400FDF727FF1DB12C46E8680028E1D0F8BD00BFFC
:207A600008B540F62843C2F200031A6802F101021A6040F61440C2F20000FFF75DFF28B196
:207A800040F61440C2F20000FFF7C2FF08BD00BF08B5014640F66C50C2F20000FFF730F8A5
:207AA00020B140F66C50C2F2000008BD40F61440C2F2000008BD00BF70B5044640F6E4231C
:207AC000C2F2000353E8002F02F1010243E800210129F7D0FFF7DCFF05462146FFF710F8D1
:207AE000002845D040F6E420C2F2000050E8002F02F1010240E800210129F7D028462146EF
:207B0000FEF7ECFF18B1C168E2688B18C360F9F75FFB064628462146FEF7F8FF3046F9F7C6
:207B200061FB4FF0FF35E56040F6E423C2F2000353E8002FA2F1010243E80025012DF7D0F8
:207B400053E8002FB2F1004F0DD14FF0000243E80025012DF4D04EF60450CEF200000168A7
:207B600041F080510160BFF32F8F4FF0010501E04FF0000504F11400FDF78CFE40F6E42304
:207B8000C2F2000353E8002FA2F1010243E80024012CF7D053E8002FB2F1004F0DD14FF072
:207BA000000243E80024012CF4D04EF60450CEF20000016841F080510160BFF32F8F284681
:207BC00070BD00BF2DE9F04105460F4614469846FFF772FF064694B19DF82030002B14BFBF
:207BE00020460020286105F114004146069A079BFDF736FE384629462246FFF7B3FE304609
:207C0000BDE8F08170B584B00E4615460093089C01949DF82430029340F66C51C2F2000154
:207C200032462B46FFF7CEFF04B070BD00B583B04FF0000300934FF00100019040F67C5027
:207C4000C2F2000041F288314FF0FF0247F66123C0F60203FFF7D6FF40F66C54C2F200044F
:207C6000FFF7E2FC2046FFF7D3FEFFF7BFF9F7E740F62443C2F2000318681A689042FBD183
:207C8000704700BF10B540F62443C2F200031A6802F101021A60FFF7B1FC044640F66C5084
:207CA000C2F20000FFF748FE204310F0FF0F06D040F61040C2F200000068FFF7C9F910BD66
:207CC00008B549F6DC50C0F603004FF0060148F2FD02C0F60202FFF713FB40F6E053C2F269
:207CE0000003186008BD00BF38B504460D4640F61863C2F20003586AA0420AD040F6186166
:207D0000C2F200014C620A681AB115B14948FDF7C7FD40F61863C2F20003186F84420AD025
:207D200040F61861C2F200010C67CA6C1AB115B14148FDF7B5FD40F61863C2F20003D3F843
:207D4000BC0084420CD040F61861C2F20001C1F8BC40D1F898201AB115B13848FDF7A0FD89
:207D600040F61863C2F20003D3F8080184420CD040F61861C2F20001C1F80841D1F8E420F2
:207D80001AB115B12E48FDF78BFD40F61863C2F20003D3F8540184420CD040F61861C2F2D3
:207DA0000001C1F85441D1F830211AB115B12548FDF776FD40F61863C2F20003D3F8A00121
:207DC00084420CD040F61861C2F20001C1F8A041D1F87C211AB115B11B48FDF761FD40F621
:207DE0001863C2F20003D3F8EC0184420CD040F61861C2F20001C1F8EC41D1F8C8211AB130
:207E000015B11248FDF74CFD40F61863C2F20003D3F83802A0420CD040F61861C2F2000176
:207E2000C1F83842D1F814221AB115B10848FDF737FD38BD280E0020740E0020C00E00202C
:207E40000C0F0020580F0020A40F0020F00F00203C1000202DE9F04707460D46914608989E
:207E6000DDF828800C683E68D8F800108A19944202D80219964203D304192C60BDE8F087AA
:207E8000341B061BB14234BF8A46B246099931B1D9F800000818191952460EF007FED8F8B2
:207EA0000030CAEB0302C8F800203E6806EB0A013960D9F8000000EB0A03C9F800302E686D
:207EC000A41954442C60BDE8F08700BF70B584B09CF81960157A947B4FF007038CF81030D5
:207EE0004FF005028CF8112006F00F0260F3C7128CF812204FF0000065F301008CF813006F
:207F00004FF0000261F30A02ACF814208CF81640DCF80C100093DCF804300193CDF808C062
:207F200001F104000CF108020CF11003FFF792FF04B070BD2DE9F04F8FB0074605911446FB
:207F40004FF000030793136012896068131A8B4238BF05930599002900F0AA8040F610655A
:207F6000C2F200052D6815B34FEAC5054FF000024FF0FF01134641F28C00C2F20000A5F106
:207F80000806C6F3C00E1658F6798E4240F0958096E01658F6798E421CBF0133314602F1BE
:207FA00008028658F6798E4240F09F80A0E04FF0000303EB43024FEAC20000F110000890C2
:207FC0004FF48071ADF824104FF00402ADF826208DF828300DF129004FF000014FF00702D8
:207FE0000EF088FD04F1040B04944FF010030093019705A802905846214607AA08ABFFF747
:020000040802F0
:2080000029FF0599002951D04FF001028DF821200DF132004FF000014FF006020EF06AFD2C
:2080200040F61063C2F20003186800283ED04FF0FF014FF0000441F28C09C2F2000949F6E4
:20804000EC58C0F6030840F6106AC2F2000A59F83450ED798D4223D08DF820404FEA051677
:208060000DF1220008EB06014FF008020EF01EFD06F108010DF12A0041444FF008020EF090
:2080800015FD4FF018020092019705AB02935846049907AA08ABFFF7DDFE059830B12946A9
:2080A00004F10104DAF80020A242D0D8079801E04FF0FF300FB0BDE8F08F03F10103314608
:2080C00002F10802AA423FF474AFBEF1000F3FF460AF1658F6798E421CBF0133314602F13B
:2080E0000802AA427FF455AF63E703F10103314602F10802AA427FF44CAF5AE72DE9F0417B
:208100004FF00100FDF79AFA49F66C60C0F60300FDF718F940F60C63C2F200034FF0010230
:208120001A7040F60860C2F20000016841B940F60864C2F20004FEF759FF2568002DFAD0D5
:2081400040F60F67C2F2000740F60C64C2F2000440F60E66C2F2000641F27905C2F200058C
:2081600040F6E458C2F200083B783BB14FF000023A704FF002002070FDF75AFA317859B17B
:208180004FF000033370227862F07F0020704FF001000146FFF7A8FD297851B14FF00000FB
:2081A0002870237803F07F0222704FF00101FFF79BFD98F8000010B9FEF718FFD4E740F661
:2081C0000C61C2F200014FF002030B704FF00000FDF734FABDE8F08108B540F60863C2F235
:2081E0000003186040F6E050C2F200000068FEF72FFF08BD70B505460E4640F61463C2F275
:2082000000031868032801D9F8F78CFF40F61462C2F20002116840F6E854C2F2000444F81B
:20822000316004EBC104656001F10101116070BD70B505460C461646032801D9F8F772FF1F
:2082400041F28C03C2F2000353F8350008B1F8F769FF41F28C01C2F2000141F8354001EB06
:20826000C5056E6040F61063C2F200031A6802F101021A60206930B1FDF764F804F104045D
:2082800020690028F8D170BD08B540F61863C2F20003196881425AD040F61862C2F200023E
:2082A000D36C834234D040F61861C2F20001D1F8982082422FD040F61863C2F20003D3F8DB
:2082C000E41081422AD040F61862C2F20002D2F83031834225D040F61861C2F20001D1F875
:2082E0007C21824220D040F61863C2F20003D3F8C81181421BD040F61862C2F20002D2F843
:208300001432834216D0F8F70DFF4FF0080013E04FF0010010E04FF002000DE04FF0030097
:208320000AE04FF0040007E04FF0050004E04FF0060001E04FF0070040F61861C2F2000131
:208340004FF04C0202FB001090F8200008BD4FF00000F1E72DE9F04F8FB0089007910A929F
:208360004FF0000309931360546813891B1B8B4238BF07930799002900F04A81082C69D8C7
:2083800040F61064C2F20004D4F800E040F61465C2F200052E680EEBCE0707EBC60404F152
:2083A00009044FF0000141F28C07C2F20007CB598BB1DD68641903F110051B695BB15E894D
:2083C0000EB104F107049B890BB104F1070455F8043F002BF3D101F108012029E7D140F64D
:2083E0000861C2F200010D682F7E6E7EEB8A03F10103C3F347054FF000010C914FF00903BA
:208400008DF82C304FF002018DF82D10ADF82E408DF830E04FF001018DF831104FF0000188
:2084200067F3451166F3861161F07F018DF833108DF834500093019007A8029002F104009E
:20844000114609AA0BABFFF705FD079A002A00F0DD80E0E04FF009001060DCE05BF836404F
:20846000002C00F0CE80059D286800284BD07A68B2420CD04FF0000310F0010F3ED1DFE04B
:2084800007EBC3025268B24240F0E38001E04FF0000357F83300D2B290F8048090F805C062
:2084A00090F806E0C579016819B143F01000C3B201E04FF000034FF008008DF82C004FF0CB
:2084C0000B018DF82D108DF82E208DF82F808DF830C08DF831E08DF832508DF833300A992A
:2084E0000090089A019207AB029301F1040009AA0BABFFF7AFFC079828B987E003F101058F
:208500002B468542BCD104F1100523697BB129464FF00002588908B102F101029B890BB1B4
:2085200002F1010251F8043F002BF3D101E04FF000025FFA86FCD2B294F804E06079A179E6
:2085400023681BB146F02003DBB201E04FF000038DF82CA04FF004088DF82D808DF82EC07A
:208560004FF0000C8DF82FC08DF830208DF831E08DF832008DF833108DF834300A99CDF801
:2085800000A0089A019207A8029001EB080009AA0BABFFF75FFC0799002937D0A3686BB120
:2085A0000A99E26800920898019007AA029201EB080009AAFFF74EFC079B3BB3246904B30B
:2085C0004FF001084FF000092046FFF75DFE8DF83500618939B10DF11C0C40462246FFF7BC
:2085E00075FC079991B1A18939B10DF11C0C48462246FFF76BFC079840B155F8044F002C3F
:20860000E2D106F10106042E7FF428AF099814E04FF0FF3011E04FF0000641F28C0BC2F276
:20862000000B40F61464C2F2000405944FF0090A40F6E857C2F2000710E70FB0BDE8F08FD4
:2086400003F1010307EBC3014A68B2427FF456AF1FE705F1010307EBC3014A68B2427FF47F
:208660004DAF16E708B541F27C03C2F200031A5C40F61861C2F200014FF04C0000FB021069
:20868000436AD3F1010238BF002242634FF00001C1630164416400F11000FDF701F908BD86
:2086A0002DE9F04790B081468A4641F27C03C2F200031A5C40F61860C2F200004FF04C04C6
:2086C00004FB020404F148064FF001084FF00007354640463146F8F729FD28B14FF002001D
:2086E0003146F8F723FD36E0BAF1000F05D148464146FCF753FD032827D0256C75B168466F
:20870000A168E26BA8470546B0F1FF3F14D06064484669462A46FCF767FD0EE0616CA56876
:208720008D4228BF0D464846E16B2A46FCF75CFDE36B5A19E26300E03D46606CA168884292
:208740003CBFE7632764451B656438463146F8F7EDFC0228BCD010B0BDE8F087F8B50546C9
:208760000E46174641F27C03C2F200031A5C40F61860C2F200004FF04C0404FB02044FF034
:208780000000FCF763FCE76326644FF00001616428464FF00101FFF783FF4FF00100FCF754
:2087A00055FCF8BDF8B505460F46164641F27C03C2F200031A5C40F61860C2F200004FF08A
:2087C0004C0404FB0204A168B1420DD241F6EC13C2F200039F4207D342F2EC12C2F20002D9
:2087E000974201D2F8F79EFC4FF00000FCF72EFCE7634FF000002064666428464FF0010162
:20880000FFF74EFF4FF00100FCF720FCF8BD00BF08B5FCF771FD08BD70B586B005460C4677
:20882000164602A8F9F778FC01462EB102A82A46234600F09BFD07E04FF00103009302A836
:208840002A46234600F044FE06B070BD70B58AB00378212B00F0938004D86BB1012B40F0AD
:20886000D88186E0A12B00F0A781C02B00F0B481802B40F0CE8195E04178052903D00929BA
:2088800040F0CA8146E0408840F60C62C2F200021378022B02D0032B33D118E000F1FF3140
:2088A0008AB27E2A30D8C0B241F27803C2F2000318704FF00201FCF72BFE40F60C60C2F2B9
:2088C00000004FF0030101704FF00100C3E170B941F27802C2F20002107040F60C60C2F29E
:2088E00000004FF0020303704FF00100B3E17F280DD841F27801C2F2000108704FF0010048
:20890000A9E14FF00200A6E14FF00200A3E14FF00200A0E1827840F60C63C2F20003197897
:20892000022923D972B940F60C63C2F200034FF0030119704FF001000146FFF7D5F94FF033
:20894000010088E1012A18BF022040F0848140F60C60C2F200004FF0040202704FF0000008
:208960000146FFF7C1F94FF0010074E14FF0020071E140780B280CBF012002206BE1838888
:20898000032B00F24C8141F28C04C2F2000404EBC3035B68002B00F045819847002808BF48
:2089A000022058E142781AB1062A40F03E8121E0C18802291BD14FF00000ADF8040040F639
:2089C0000862C2F2000212680346517E61F30003ADF80430127E62F341030AA921F8243D5F
:2089E0004FF00202FFF7DEFE4FF0030033E14FF0020030E18278C1888CB2C378022B2ED0D3
:208A0000032B3DD0012B40F0D48040F6A055C2F20005284649F6C851C0F603014FF01202B4
:208A20000EF044F840F60860C2F2000001688A892A81CB896B81088AA8818A7C2A71CB7CA0
:208A40006B71097DA9714FF000002946122C34BF22461222FFF7A6FE4FF00300FBE041F235
:208A6000B402C2F2000211814FF00000506048F25531C0F60201FFF771FE4FF00300EAE01F
:208A8000D2B940F6A054C2F2000404F1020049F6C451C0F603014FF002020EF007F84FF0E5
:208AA000040222704FF0030565704FF000002146FFF778FE2846CEE0012A06D140F6086331
:208AC000C2F20003196809682FE0022A06D140F60862C2F200021068416826E0032A06D15A
:208AE00040F60863C2F20003196889681DE002F00F0022F00F03102B08D15A4B1968884286
:208B00000EDA594A52F8300001680EE0202B07D1032805D8554951F8300008B1016804E0B1
:208B2000EE2A04D04FF0020095E009B93EE05049B1F1FF3F40F0888001A84FF020014FF0BA
:208B40000102FFF769FE0AAD2A184FF0000002F8240C01A978E000F10206428003F101029F
:208B6000134611F8015F5DB100F10400758002F1010311F8012F002A6FD101E04FF000037E
:208B800040F6A051C2F200014FF003054D7003F101034FEA4303DAB20A704FF00000A24255
:208BA00028BF2246FFF7FEFD284654E04FF0020051E04FF002004EE08388032B38D841F276
:208BC0008C04C2F2000404EBC3035B689BB39847002808BF02203EE04378212B2ED1C1882A
:208BE00041F2B403C2F2000319814FF000025A608088042825D1104647F63571C0F6020123
:208C000041F2B402C2F20002FFF7A8FD4FF0030021E04FF002001EE04FF002001BE04FF01D
:208C2000020018E04FF0020015E04FF0020012E04FF002000FE04FF002000CE04FF0020033
:208C400009E04FF0020006E00A78002A96D009484FF000037FE70AB070BD1E2B7FF47BAF2C
:208C60008EE700BF140E0020E80D00208C100020E09D0308A00D002010B50446436993B159
:208C80004FF00000606140F60C61C2F200010A78032A08D141F27803C2F2000318784FF0C0
:208CA0000301FCF735FC206958B34FF000002061E06040F60D61C2F20001087041F2AC0147
:208CC000C2F200014FF00802FFF7A2FD082853D141F2AC02C2F20002137813F0800F06D122
:208CE00041F2AC00C2F20000C188002944D141F2AC00C2F200004FF000010A46FFF7A6FD9E
:208D00002DE0E168002937D04FF00000E06040F60D62C2F20002137840F6A051C2F200018C
:208D2000C3F14002FFF774FD034628B340F60D60C2F2000001785A18D2B2027041F2AC0398
:208D4000C2F20003D888904216D141F2AC00C2F2000040F6A051C2F20001FFF777FD012841
:208D600004D0022808D1FCF729FA10BD4FF0000001460246FFF716FD10BD00BF08B541F2E6
:208D8000C003C2F200031B693BB14FF0000141F2C002C2F200025269984741F2C000C2F2BD
:208DA00000004FF00001017041608160C1600161416108BD41F2C000C2F20000816149F6CE
:208DC0002C71C0F603018A5C42778377037F6FF3070303774FF000014162704730B583B089
:208DE00041F2C004C2F200042070089D6560099DA5600A9DE5600B9D25610C9D65619DF801
:208E0000184000949DF81C400194FFF7D3FF03B030BD00BF41F2C003C2F200035B6AB3F1A3
:208E2000FF3F09D141F2C001C2F200014FF000034B624FF0010070473F2B0BD841F2C00249
:208E4000C2F20002106AC15403F1010353624FF0010070474FF00000704700BF704700BFFE
:208E600070B541F2C004C2F2000404F1180049F61C71C0F603014FF007020DF017FE4FF0F2
:208E8000000049F62471C0F60301FFF7B3F949F2BD06C0F602064FF0000049F6CC61C0F685
:208EA00003013246FFF7C4F949F63075C0F603054FF0010029463246FFF7BAF92869FFF78A
:208EC000E3F984F8280041F2EC00C2F200004FF0070148F6E562C0F602024FF00003FCF784
:208EE000BFFC70BD38B541F22013C2F200034FF001021A7041F2C004C2F2000494F8280051
:208F00004FF000010A46FFF74DFC606868B141F2C004C2F200044FF0FF3565626368207855
:208F200061699847616A0029F7D041F2C000C2F200004FF000024262836833B141F2C0017E
:208F4000C2F2000108784969984738BD2DE9F047A2B0804643680BB9806828B14FF0000181
:208F6000C8F80810FFF7BEFFD8F80C20002A3ED04FF00007C8F80C70D8F8000012A94FF0E6
:208F80004002FFF745FC074641F2C003C2F20003D86860B35FB341F2C004C2F200044FF00B
:208FA000000507F1FF3606F0010A20789DF848102A466369E668B0474FF001094F456CD15E
:208FC00015E0E668207812AA12F809102A466369B04709F10109E668207812AB13F80910D9
:208FE0002A466369B04709F101094F45E9D1D8F8140000284ED04FF0000441F22011C2F267
:2090000000010C70C8F8144041F2FC00C2F20000FEF752FD41F2C002C2F20002546253687C
:20902000002B30D041F2C005C2F2000502AC2C622C46656A6268207861699047606A854243
:20904000F7D105B3D8F8000002A92A46FFF7AAFB4FF000010091019141F2FC00C2F20000C4
:209060004FF04B014FF0FF0248F6E563C0F60203FEF7C8FD0EE041F2C002C2F20002107809
:209080005169984706E041F2C003C2F200039B68002BF0D122B0BDE8F087BAF1000F90D0AD
:2090A000E668207812A911F809102A466369B04709F101094F4584D199E700BF10B544780D
:2090C0000378212B02D0A12B19D10CE0202C02D0222C08D119E0072A1AD10F480DF0E6FCC5
:2090E0004FF0010010BD212C0CD14FF000000A494FF00702FFF756FB4FF0030010BD4FF0CA
:20910000000010BD4FF0000010BD4FF0010010BD4FF0020010BD00BFD810002008B541F2A4
:209120002013C2F20003187870B941F2C001C2F200014A6A72B941F2C003C2F2000393F8CC
:209140002800FFF78FFA08BD41F2EC00C2F20000FCF7A6FB08BD00BF49F69C60C0F60300C4
:20916000704700BF70B4037801298CBF4478002402298CBF85780025DCF8000048B34FEAE5
:2091800093064AF25C00C0F60300365C16704FEA031343EA141303F03F031B5C5370012991
:2091A00007D94FEA840444EA951303F03F04205C01E04FF03D009070022907D905F03F05E5
:2091C0004AF25C03C0F60303E95C01E04FF03D01D17070BC704700BF82B04FF015010CE03F
:2091E0000191019B03F1FF32019233B100BF019B03F1FF320192002BF8D100F1FF30B0F1DD
:20920000FF3FEDD102B0704770B4C4B24FEA10204AF2F006C0F6030649F65C75C0F6030527
:2092200011F8013B1AB94BB944EA00200BE06340F45C4440E85C013AF2D1F5E76340F45C51
:209240004440E85CECE770BC704700BF10B444F6FB43C0F2861311F8014B02B9ACB380EA71
:2092600004404FEA400010F0807F18BF58404FEA400010F0807F18BF58404FEA400010F063
:20928000807F18BF58404FEA400010F0807F18BF58404FEA400010F0807F18BF58404FEA59
:2092A000400010F0807F18BF58404FEA400010F0807F18BF58404FEA400010F0807F18BFCA
:2092C0005840002AC7D0013AC5D120F07F4010BC704700BF82B001909DF806304FF0000086
:2092E00063F307009DF8052062F30F209DF8042062F317409DF8072012F0800F14BF63F0FB
:209300007F0103F07F0161F307004FEA4201CAB262F31F6013F0800F18BF42F0010262F340
:209320001F6002B0704700BF84B0C0F307438DF80C30C0F307228DF80D20C3B24FEA1060E8
:209340004FEA500210F0010F14BF63F07F0103F07F018DF80E1013F0800F18BF62F07F027A
:209360008DF80F20039804B0704700BF2DE9F04F83B005460F4614461E46019201F1FF33D7
:2093800013F1050F44D8032E43D9A6F10400C0F380080DF1040C2846FFF7E4FE05F1030524
:2093A000A7F1030104F10404A6F10406A7F1040717F1050F67D92CE00DF1040C284639466D
:2093C0002246FFF7CFFE05F1030B5D46A7F1030104F1040A5446A6F104094E46A7F10407A7
:2093E00017F1050F15D80F460DF1040C58465246FFF7B8FE0BF10305A7F103010AF104047C
:20940000A9F10406A7F1040818F1050F59D900E0FFE799B396B30DF1040C28466A46FFF738
:20942000A1FE022E11D0032E02D0012E26D11AE0019929B19DF8002022704FF0010301E07A
:209440004FF0000304F1010401E04FF00003019830B102A9CA1812F8080C207003F1010300
:2094600004F1010401E04FF00003019921B102AAD31813F8080C207004F101040199601A0F
:2094800003B0BDE8F08F0F46032EC2D9B8F1000F92D00DF1040C28462246FFF763FE05F189
:2094A0000305A7F1030104F10404A6F10406A7F1040717F1050FACD80F46032E3FF67CAF41
:2094C000A7E7A7F10307032E3FF676AFA1E700BFF0B49DF81040ECB14FEA41079F421CD214
:2094E000DD1B1DD056194FF030046FEA0203F31803F0010302F8014BB24240F0928007E0E2
:20950000134603F8014B547003F10102B242F7D13B4607E04FF0000504E04FF0000501E07F
:209520004FF0000500293CD003F1FF34002B3AD000F1010341182846521B04F1FF3515F0FF
:20954000020F10D032E0A4F1020603F101031F46012C29D03446B44613F8016C4FEA161697
:20956000092E42D944E01E4613F8015C4FEA1515092D8CBF37353035155414B900F10100CC
:2095800012E013F8016C06F00F05092D8CBF373530351618757000F1020528468B42D2D11C
:2095A00002E0284600E02846F0BC70471E4613F8015C4FEA1515092D94BF303537351554B8
:2095C000002CDBD013F8016C06F00F05092D94BF303537351618757000F102008B42E3D052
:2095E00003F10103A4F10204BDE706F1300601E006F137065655BCF1000FBFD013F8016C84
:2096000006F00F06092E94BF303637361018467005F102008F42C7D003F10103A4F1020411
:20962000A1E7002B3FF46CAF02F8014BB2427FF467AF6DE7DCF8143093F8452083F844202B
:20964000DCF8141091F8463081F84530DCF8141091F8472081F84620DCF8143083F8470084
:20966000704700BFDCF8143093F8470093F8462083F84720DCF8141091F8453081F84630D2
:20968000DCF8141091F8442081F84520704700BF41F2DC32C2F20002136840F20001C0F636
:2096A0000101C85CC918497803F10203136041EA00207047DCF80430DCF8082002EBD300B0
:2096C000CCF8080003F007014FF0010303FA01F2CCF80420704700BF2DE9F04F83B0044660
:2096E0008A4693461E46CDF804C04FF00007B846B9463DE025463046D047034600283DD0FE
:20970000B9F1000F0CD1202829D0092829D00A2829D00D2829D0022D4FF0010988BF022509
:20972000A3F13002D1B2092910D9A3F14100C1B2052903D8A3F13703D9B207E0A3F161023D
:20974000D0B205281AD8A3F15703D9B24FEA0717FCB241EA040708F101082C4606E02C46E8
:2097600004E02C4602E02C4600E02C463046D847FF2CBFD004F1FF35002CBCD1DDF804C023
:209780003846FFF757FF019B5A69D8F1010838BF4FF0000882F8508003B0BDE8F08F00BFB0
:2097A00041F2B023C2F200031B684B634BB19A68824209D0DB684B631BB19A688242F9D1D3
:2097C00002E04FF01E0070474FF00000704700BF884204D8884234BF0220002070474FF043
:2097E00001007047D0F80431D0F80021934214BFC05C0020704700BFD0F80431FF2B14BF77
:2098000001330023C0F80431704700BF10B4DCF81420D16C0B46044658B14FEA016343EA17
:20982000116301F47F4043EA002301F47F0143EA1123DCF8040030B199B24FEA134060F3F7
:209840000F0361F31F435CB94FEA036141EA136103F47F4041EA002103F47F0341EA132313
:20986000D36410BC704700BFDCF80030FA2B05D841F22C12C2F20002D05C70474FF0000020
:20988000704700BFDCF8003003F10103CCF80030DCF8140090F8512002F1010280F85120A2
:2098A000704700BF70B404460846A1B199188C4211D22518AA420ED294423ABFC4EB020633
:2098C000F6B20026A94205D20019821AD31AF118C8B200E0304670BC704700BFF0B583B003
:2098E00041F28423C2F200034FF00E021A7041F26C20C2F2000004683CB3154641F28427F7
:20990000C2F200074FF0000621680B6873B10DF107000DF1060198479DF807009DF80610F7
:2099200032463B78FFF7BEFF4519EDB26468002CEAD141F28422C2F200021078A84204D2C2
:2099400041F28421C2F200010D7041F28423C2F200034FF008025A7041F2A424C2F20004A6
:2099600024683CB3154641F28427C2F200074FF000062068036873B10DF107000DF1060112
:2099800098479DF807009DF8061032467B78FFF789FF4519EDB26468002CEAD141F2842130
:2099A000C2F200014A78AA4204D241F28420C2F20000457041F28423C2F200034FF0060157
:2099C000997041F27C24C2F2000424683CB30D4641F28427C2F200074FF000062268136842
:2099E00073B10DF107000DF1060198479DF807009DF806103246BB78FFF754FF4519EDB222
:209A00006468002CEAD141F28420C2F200008178A94204D241F28422C2F20002957041F287
:209A20008423C2F200034FF00100D87041F2E034C2F2000424683CB3054641F28427C2F2E9
:209A400000074FF0000621680A6872B10DF107000DF1060190479DF807009DF806103246FC
:209A6000FB78FFF71FFF4519EDB26468002CEAD141F28423C2F20003D878A84204D241F2DB
:209A80008421C2F20001CD7003B0F0BD41F2D833C2F20003196840F20000C0F60200401A15
:209AA000704700BF034610B182688A4218D041F28023C2F20003186860B182688A4203D1E0
:209AC0000BE083688B420AD040680028F9D14FF0000305E04FF0000302E0034600E00346B2
:209AE0001846704710B540F2A064C1F200044FF4117303FB0044D4F80811B1F1FF3F03D0FE
:209B0000D4F8042191420DD123689A6A4FF0FF019047002834D0D4F8080100F10100C4F84F
:209B2000080110BD91422BD86318197941F27922C2F2000213787BB9FD290FD923689A6A8C
:209B40004FF0FE019047D8B141F27920C2F200004FF00101017010BD6FEA01012268936A86
:209B6000C9B2984760B1D4F8080100F10100C4F8080141F27921C2F200014FF000020A70B1
:209B800010BD00BF70B5064640F2A065C1F200054FF4117404FB00F42B194FF00101C3F8DE
:209BA0000C112A59936998472859016A3046884770BD00BF38B540F2A061C1F200014FF4F6
:209BC000117202FB00F28C18D4F80831D4F80451AB420DD08958E3188A6A1979904738B15D
:209BE000D4F80801FF2814BF01300020C4F8080138BD00BF38B540F2A064C1F200044FF4AF
:209C0000117202FB00F2A318D3F80451D3F808118D4206D14FF00001C3F80C11A25893695F
:209C2000984738BD10B440F2A063C1F200034FF4117202FB003000F58870D0F80031FF2B9E
:209C400014BF5A1C0022D0F80441A2421CBFC154C0F8002110BC7047F8B541F2D834C2F2BC
:209C6000000424688568C768466807FB05604518611911D2CE180B48864210D8012B04D17F
:209C8000635D13704FF00000F8BD10461A460CF00DFF4FF00000F8BD4FF01F00F8BD4FF089
:209CA0001F00F8BD0100020810B541F28823C2F200031A7840F2A060C1F200004FF411742C
:209CC00004FB0204F7F784FA4FF0FF31C4F810124FF00003C4F8183204F58874F7F782FA1F
:209CE00010BD00BFF8B506464FF00203037044F20000C0F60000C28B4FF6FF718A4221D07D
:209D00003F4C404BA34222D203F110033E4DEF1A4FEA17124FF6FF7502F1010002F00107B0
:209D20001C46D98BA9424FD115E01C46D98BA94211D002F1010203F110031C46D98BA9421D
:209D400057D108E044F20004C0F6000403E044F20004C0F600044FF6FF7021464FF00D02BF
:209D6000FFF752FA4FF6FF73984208BF0020E28982421BD0A4F1100544F20000C0F6000079
:209D800085421AD34FF6FF7029464FF00D02FFF73BFA4FF6FF71884208BF002034F8024C93
:209DA00084420AD12C464FF0010201E04FF00002607BFF2806D1327004E04FF002033370E6
:209DC0004FF000042046F8BD4FF0000202F1010203F110038242BED0002FA6D01C46D98B2A
:209DE000A942B8D002F1010203F1100382429CD1B1E702F1010203F11003824295D1AAE772
:209E000000800008004000080F80000870B5C0B005460E4620F0FF04684621464FF04002FE
:209E2000F9F7F4F900AB53FA85F031464FF010020CF03CFE684621464FF48072F9F73AFB6B
:209E400040B070BD38B5054640F2A064C1F200044FF4117303FB0044D4F81C02FDF73AFBA4
:209E600041F28820C2F200000178A94206D141F28823C2F200034FF0FF021A704FF000007A
:209E8000C4F81C0238BD00BF10B54FF00000FBF727FD41F26C23C2F200031C6834B12068B0
:209EA000016901B188476468002CF8D110BD00BF10B50446072827D8032894BF4FF4FA73FF
:209EC000322303FB01F140F2A063C1F2000303EBC000C0F8141969B1FDF7CAFE002808BFFA
:209EE000012040F2A063C1F2000303EBC404C4F8100910BD40F2A061C1F2000101EBC40463
:209F00004FF00002C4F8102910BD00BF38B50446072851D840F2A063C1F2000303EBC00057
:209F2000D0F8145935B340F2A061C1F2000101EBC402D2F81039EBB1FDF79AFE002808BF41
:209F4000012040F2A061C1F2000101EBC402D2F81039C01A85420CD240F2A065C1F20005C6
:209F600005EBC4014FF00005C1F81459C1F8105900E02D1A05F104054CF6CD42CCF6CC4259
:209F8000A2FB05234FEA9300032C0AD800F1630348F21F51C5F2EB11A1FB03324FEA5210FF
:209FA00038BD00F109014CF6CD42CCF6CC42A2FB01304FEAD00038BD4FF0000038BD00BFD1
:209FC00070B506466446DCF814305D6AFDF750FE6169CA6A0AB9C86208E0801A05EB85055E
:209FE00006FB05F6B04224BF0020C8626369D96AD1F1010038BF002070BD00BF10B540F27A
:020000040802F0
:20A00000A063C1F200034FF4117404FB003303F58873D3F80841002C5FD15AB14FF0FF31B0
:20A02000C3F8001141F22C23C2F200034FF00000187010BDD3F80021B2F1FF3F06D1FF29BB
:20A040004BD14FF00002C3F8002110BDFF291ED141F22C21C2F200014FF000040C70012AC4
:20A0600010D94FF00102C3F8082140F2A063C1F200034FF4117101FB0030D0F81C02FCF71C
:20A08000E7FF10BD4FF00000C3F8000110BDFE2907D141F22C23C2F200034FF00101197043
:20A0A00010BD41F22C20C2F20000007848B16FEA0101C9B241F22C20C2F200004FF00004E3
:20A0C0000470FF2A05D8995402F10102C3F8002110BD4FF0FF32C3F8002110BD08B540F272
:20A0E000A063C1F200034FF4117202FB0030D0F80811D0F8043100F1040099420AD94FF0E4
:20A100000002C0F8002141F2B420C2F200004068FCF79EFF08BD00BFF8B5654641F27023CF
:20A12000C2F200031C7804F00802D7B227B1DCF8146096F8516007E014F0110F06BFDCF84A
:20A14000144094F85260002601EB800411F820304FEA9312012A08D0022A10D111F82070F7
:20A16000C7F3C20303FB06F70BE06A6992F8513011F82070C7F3C20202FB03F701E04FF06E
:20A18000000711F8200000F00701042950D8DFE811F0940140003B002200050041F2DC3103
:20A1A000C2F200010B6840F20007C0F60107FA1892F802E0D0784FEA006040EA0E405278DF
:20A1C00040EA0220FF5C03F104030B603843FFF7ABF868602CE041F2DC32C2F20002136818
:20A1E00040F20000C0F60100C11891F801C0C05C4FEA004040EA0C208978084303F1030322
:20A2000013603F186F6013E0FFF742FAC2196A600EE041F2DC33C2F20003186840F2000141
:20A22000C0F601010A5CBF186F6000F10100186063784FEA9310012807D002280ED1617857
:20A24000C1F3C20202FB06F70AE06F6997F851306078C0F3C20101FB03F701E04FF000074F
:20A26000627802F00703042B50D8DFE813F0260140003B002200050041F2DC31C2F2000129
:20A280000B6840F20007C0F60107FA1892F802E0D0784FEA006040EA0E40527840EA022067
:20A2A000FF5C03F104030B603843FFF73DF8A8602CE041F2DC32C2F20002136840F200007F
:20A2C000C0F60100C11891F801C0C05C4FEA004040EA0C208978084303F1030313603F18A9
:20A2E000AF6013E0FFF7D4F9C219AA600EE041F2DC33C2F20003186840F20001C0F6010162
:20A300000A5CBF18AF6000F101001860A3784FEA9310012807D002280ED1A178C1F3C202F6
:20A3200002FB06F70AE06F6997F85130A078C0F3C20101FB03F701E04FF00007A27802F09A
:20A340000703042B4ED8DFE803F0B83E3920030041F2DC31C2F200010B6840F20007C0F63B
:20A360000107FA1892F802E0D0784FEA006040EA0E40527840EA0220FA5C03F104030B602C
:20A380001043FEF7D1FFE8602CE041F2DC32C2F20002136840F20000C0F60100C11891F894
:20A3A00001C0C05C4FEA004040EA0C208978084303F1030313603F18EF6013E0FFF768F948
:20A3C000C219EA600EE041F2DC33C2F20003186840F20001C0F601010A5CBF18EF6000F189
:20A3E00001001860E3784FEA9310012802D002280FD108E06E6996F85130E078C0F3C2010C
:20A4000001FB03F607E0E178C1F3C20202FB06F601E04FF00006E27802F00703042B4CD8C7
:20A42000DFE803F04B031318300041F2DC33C2F20003186840F20001C0F601010A5CB61821
:20A440002E6100F101001860F8BDFFF721F982192A61F8BD41F2DC32C2F20002136840F2BF
:20A460000000C0F60100C1184C78C05C4FEA004040EA04208978084303F10303136036189E
:20A480002E61F8BD41F2DC31C2F200010B6840F20004C0F60104E2189678D0784FEA006036
:20A4A00040EA0640527840EA0220E25C03F104030B601043FEF738FF2861F8BD08B50328CD
:20A4C0001ED8DFE800F0020910174BF27820C0F603000EF0DDF808BD4BF27C20C0F60300E5
:20A4E0000EF0D6F808BD4BF29020C0F603000EF0CFF808BD4BF2A820C0F603000EF0C8F81F
:20A5000008BD00BF2DE9F8430546884616461F4641F28823C2F2000393F8009041F2E86061
:20A52000C2F20000016841F26822C2F200021368994201D0FFF7B8FB072D6ED81F2E6CD8B0
:20A5400040F2A064C1F200044FF4117000FB094441F2B420C2F200004FF00001FCF718FB01
:20A56000217965F34711072D14BF00250125AA1962F304012171CBB22DB184F805804344AD
:20A580004FF0020001E04FF0010006F1FF3E5FFA8EFE46B302463F1A0EF0010C3D5C04F10D
:20A5A000040635545B1902F101020EF1FF31C9B2FF2934D114E0BD5C04F10406B5545B193E
:20A5C00002F1010201F1FF3101F0FF01BD5CB5545B1902F1010201F1FF31C9B2FF29EAD166
:20A5E00000F1010070442218137100F10100C4F804014FF0FF33C4F8083121680B6A41F2AD
:20A600008820C2F2000000789847FCF7EFFC41F2B420C2F20000FCF7C9FBBDE8F8834FFACE
:20A620008CF5002DC7D0BD5C04F10406B5545B1902F1010201F1FF31C9B2FF29BBD1CFE743
:20A6400038B5054641F23024C2F200042046FCF7ADFBF7F779FF2846FCF790FE20464FF088
:20A660000001FCF795FA38BD10B586B00DF10700FFF738FB044618B19DF8073023B90FE08F
:20A6800044F20004C0F60004E2894FF6FF7082422BD048F20001C0F600018C4209D32AE042
:20A6A000304821464FF00D020BF0AAFD002848D0EAE74FF6FF7248F20000C0F600006FEABB
:20A6C0000403C118C1F3001104F11004E389934239D10AE004F110031C46D989914204D024
:20A6E00003F11004E389934239D148F20002C0F60002944207D344F20004C0F60004204609
:20A700002146F8F76BFE02A816494FF00D020CF0CDF94FF0FF008DF815004FF6FF7002A92A
:20A720004FF00D02FEF770FD4FF6FF71884212BFADF816000021ADF81610204602A9FFF76B
:20A7400065FB06B010BD8442D5D20029C2D004F11004E1899142C8D08442BBD3CBE7844244
:20A76000B8D3C8E7321100202DE9F04F85B0884691461D46E2464FF0000426464FF0020B87
:20A780002DE007462846C047034670B324B9202822D0092802D11FE0012C05D12B2B0DD02E
:20A7A0002D2B0DD05C4601E0022C01D12E2B09D0A3F13002D0B2092817D805E05C4603E0DD
:20A7C0005C4601E04FF003040E2E05D804A98A1902F8103C06F101062846C8473846FF28E1
:20A7E000CFD000F1FF370028CCD1012C12D98EB104ACA6194FF0000406F8104C6846214656
:20A800000BF058FDDAF81410C864DAF8142082F8504005E0DAF814304FF0010083F85000B0
:20A8200005B0BDE8F08F00BF10B586B040F20000C0F601003449F8F7D1FD00284BD1334BA0
:20A84000334A9A421DD240F20001C0F601010B68B3F1FF3F42D102F104032E4AD01A20F0F1
:20A860000302991812F0040F3FD118468B420CD003F104021B68B3F1FF3F3ED04FF000004A
:20A8800031E040F20000C0F6010040F20003C0F60203984225D10DF10700FFF723FA04469C
:20A8A000B0B19DF80710022912D002A821464FF010020CF0FBF89DF815006FF307008DF895
:20A8C0001500204602A9FFF7A1FA4FF001000AE04FF0010007E04FF0000004E04FF000000E
:20A8E00001E04FF0000006B010BD184603F104030268B2F1FF3FB8D0C0E702F10403106870
:20A90000B0F1FF3FB1D0B9E7FFFF01080000020800000108030002082DE9F0030346002896
:20A9200042D040F20022C0F6000292F8468092F847C041F28420C2F20000457892F848708E
:20A94000047841F2A826C2F20006306896F8049076794FF000021A7083F8018083F802C013
:20A96000DA704FF0FB0C83F804C04FF0060C83F805C09C71DD714FF004051D725D729F7265
:20A98000DC721A734FEA10245C73987383F80F901E745A744FF01D0098744FF00202DA7422
:20A9A0004FF0FE001875587529B141F28423C2F200031A680A60BDE8F0037047034628B138
:20A9C00041F2A822C2F200021068186041F2A821C2F200010879704770B505460E461446CD
:20A9E0004FF000002946FFF75DF808B1F6F79AFB41F28023C2F200031A686260A5602660C7
:20AA00001C6070BD08B539B141F26C23C2F200031A68426018601EE041F26C23C2F200035A
:20AA20001B6883420FD1586841F26C21C2F20001086010E042685A6041605A688242F9D00D
:20AA400013461BB907E033B14FF000015A688242F0D01346F5E7FEF741FF08BD08B539B1A2
:20AA600041F2A423C2F200031A68426018601EE041F2A423C2F200031B6883420FD15868F2
:20AA800041F2A421C2F20001086010E042685A6041605A688242F9D013461BB907E033B165
:20AAA0004FF000015A688242F0D01346F5E7FEF715FF08BD08B539B141F27C23C2F20003DD
:20AAC0001A68426018601EE041F27C23C2F200031B6883420FD1586841F27C21C2F20001E6
:20AAE000086010E042685A6041605A688242F9D013461BB907E033B14FF000015A688242EC
:20AB0000F0D01346F5E7FEF7E9FE08BD08B539B141F2E033C2F200031A68426018601EE061
:20AB200041F2E033C2F200031B6883420FD1586841F2E031C2F20001086010E042685A607B
:20AB400041605A688242F9D013461BB907E033B14FF000015A688242F0D01346F5E7FEF75D
:20AB6000BDFE08BD01604360826041F2B023C2F200031A68C2601860704700BF70B582B0C9
:20AB800006464FF000038DF807300D4601B10B7041F26C20C2F20000046874B121684B68AB
:20ABA00043B130460DF107012A46984710B19DF8070013E06468002CF0D10D2E05DC0F2E74
:20ABC00003D83046FAF7D0FE08E02DB14FF005022A704FF0000001E04FF0000002B070BD81
:20ABE00070B582B006464FF000038DF807300D4601B10B7041F26C20C2F20000046874B130
:20AC000021688B6843B130460DF107012A46984710B19DF807001BE06468002CF0D10D2EAD
:20AC20000DDC0F2E0BD83046FAF7B4FE8DF8070010B13046FAF7F4FE9DF8070008E02DB1EA
:20AC40004FF005022A704FF0000001E04FF0000002B070BD70B582B006464FF000038DF86C
:20AC600007300D4601B10B7041F26C20C2F20000046874B12168CB6843B130460DF10701ED
:20AC80002A46984710B19DF8070013E06468002CF0D10D2E05DC0F2E03D83046FAF74AFE79
:20ACA00008E02DB14FF005022A704FF0000001E04FF0000002B070BD70B582B006464FF0CE
:20ACC00000038DF807300D4601B10B7041F2A420C2F2000004685CB121688B682BB1304643
:20ACE0000DF107012A46984758B96468002CF3D1072E0CDC0A2E0AD83046F7F7B9F88DF861
:20AD000007009DF80700003018BF012008E02DB14FF006022A704FF0000001E04FF0000062
:20AD200002B070BDF0B583B005460E464FF000038DF8073041F2A420C2F200000468E4B113
:20AD40004FF000072168CA681AB1284631469047F0B923689B6833B128460DF106010DF1DF
:20AD60000702984700E038469DF8071099B9646814B10028E6D004E018B9072D0DDC0A2D17
:20AD80000ED82846314606F0ABF94FF0000009E04FF0000006E0084604E04FF0060001E0A9
:20ADA0004FF0060003B0F0BD70B582B005460E464FF000038DF8073012B11946FFF7B2FF31
:20ADC00041F2A420C2F2000004686CB121684B68284631460DF10702984710B19DF80700DB
:20ADE00012E06468002CF1D1072D08DC0A2D09D828463146F7F75EF84FF0000004E04FF0EC
:20AE0000060001E04FF0060002B070BD08B54FF0000001464FF00102FFF7C6FF08BD00BF63
:20AE200070B582B005460E464FF000038DF8073041F27C20C2F2000004689CB121684B68A6
:20AE4000284669460DF10702984728B10EB1009830609DF8070014E064681CB19DF807204A
:20AE6000002AEBD0052D07D84EB12846F7F776FD30604FF0000004E04FF00F0001E04FF0ED
:20AE8000000002B070BD00BF70B582B005460E464FF000038DF8073041F2E030C2F2000029
:20AEA000046884B121684B68284631460DF10702984710B19DF8070010E064681CB19DF86F
:20AEC0000720002AEED03DB94FF000003146F7F73BFC4FF0000001E04FF00E0002B070BD46
:20AEE00070B582B005460E464FF000038DF8073041F2E030C2F200000468A4B121688B682A
:20AF00005BB1284669460DF10702984728B10EB1009830609DF8070014E064681CB19DF8A4
:20AF20000720002AEAD045B956B14FF00000F7F739FD30604FF0000004E04FF0060001E0C5
:20AF40004FF0000002B070BD2DE9F04F2DED048B8BB007461546914259D289464FF0000BDB
:20AF60004FF000089FED908B9FED919B6FEA0106B01800F00106CDF804B0022F4CD150E015
:20AF8000CDF804B0022F05D15FFA89F001A9FFF7A7FF04E05FFA89F001A9FFF741FF04EB94
:20AFA00044060AA88119A1F1200601F8209C01F81F8C01980AF0D4FA53EC182B0AF06EFCA3
:20AFC00053EC192B0AF026FB0AF090FA83B2FF2B28BFFF23B37004F101040A2C04D005F1CA
:20AFE000FF324A450AD14CB104EB44044FF007003946E2B202ABFFF785FA444609F1010979
:20B000004E46CDF804B0022F40F089808DE00BB0BDEC048BBDE8F08FC8B201A9FFF700FF1C
:20B0200003E0C8B201A9FFF75BFF0AAC04F8209D84F8018001980AF093FA53EC182B0AF0B1
:20B040002DFC53EC192B0AF0E5FA0AF04FFA81B2FF2934BF0B46FF23A3704FF0000404F11C
:20B06000010405F1FF324A450DD10AE004EB44044FF007003946E2B202ABFFF743FA444653
:20B0800001E0002CF2D109F101094D45BFD9002E3FF476AFCDF804B0022F05D05FFA89F0DB
:20B0A00001A9FFF7BDFE04E05FFA89F001A9FFF717FF04EB44060AA8861906F8209D86F806
:20B0C000018001980AF04CFA53EC182B0AF0E6FB53EC192B0AF09EFA0AF008FA81B2FF294D
:20B0E00034BF0B46FF23B37004F101040A2C0AD104EB44044FF007003946E2B202ABFFF789
:20B1000001FA444605E005F1FF324A4501D1002CEED109F101094D453FF632AF77E75FFAEF
:20B1200089F001A9FFF77CFE04E05FFA89F001A9FFF7D6FE04EB44000AA90B18A3F1200A8B
:20B1400003F8206C03F81F8C01980AF009FA53EC182B0AF0A3FB53EC192B0AF05BFA0AF046
:20B16000C5F982B2FF2A28BFFF228AF8022004F101040A2C0AD104EB44044FF00700394601
:20B18000E2B202ABFFF7BEF9444605E005F1FF30B04201D1002CEED109F101094D453FF6B3
:20B1A000EFAE34E7AFF300800000000000E06F40000000000000E03F2DE9F04F95B040F637
:20B1C000C410FCF7DBF84FF002004FF0000141F28423C2F20003DA78FFF7B6FE4FF0000B7D
:20B1E000DA46D9464FF001074CF6CD44CCF6CC4401944FF07D00FCF7C1F88DF82F90C84655
:20B200004E464C4613E045F0800504F10804E4B20CABF05CA84202D00CA97554B84606F192
:20B2200001069DF82F50002D50D1202E4ED020460DF12F01FFF7A2FC051C18BF012504F1FE
:20B240000100C0B20DF12F01FFF798FC10B145F00205EDB204F10201C8B20DF12F01FFF791
:20B260008DFC08B145F0040504F10302D0B20DF12F01FFF783FC08B145F0080504F1040338
:20B28000D8B20DF12F01FFF779FC08B145F0100504F10500C0B20DF12F01FFF76FFC08B1D4
:20B2A00045F0200504F10601C8B20DF12F01FFF765FC08B145F0400504F10702D0B20DF188
:20B2C0002F01FFF75BFC00289DD19EE7B8F1000F02D1BAF1000F0AD14FF002004946F2B242
:20B2E0000CABFFF70FF94FF03200FCF747F841F28422C2F2000292788AB1019EA6FB0A4395
:20B300004FEA131404EB8400BAEB800F07D138464946FFF719FE4FF03200FCF72FF8BBF1FD
:20B32000000F40F09B8003A849464FF020020BF0E1FB41F28421C2F200018D78ADB34E46BB
:20B340006FEA0902531903F0010009F0070407FA04F29DF80C1042EA01038DF80C3006F195
:20B360000106AE42C0F299801FE014AA02EBD60306F0070407FA04F013F8441C40EA0102FA
:20B3800003F8442C06F1010614AC04EBD60006F0070107FA01F210F8443C42EA030400F81A
:20B3A000444C06F10106AE42DFDB4FF007004FF011014FF01E0203ABFFF7A4F84FF03200AE
:20B3C000FBF7DCFF03A849464FF020020BF092FB41F28425C2F20005EE78A6B348466FEA42
:20B3E00009018A1902F0010309F0070407FA04F59DF80C1045EA01028DF80C2000F1010026
:20B40000864236DC1FE014AD05EBD00200F0070407FA04F312F8441C43EA010502F8445CA6
:20B4200000F1010014AA02EBD00500F0070407FA04F315F8441C43EA010205F8442C00F1AC
:20B4400001008642DFDC4FF007004FF012014FF01E0203ABFFF756F84FF0060BBAF1000F75
:20B4600004D10BF1FF3B4FF0280AC2E60AF1FF3ABFE6002BC7D014AB03EBD00500F0070490
:20B4800007FA04F215F8441C42EA010305F8443C00F101008642B6DCD5E700283FF465AF24
:20B4A00014A800EBD60206F0070407FA04F312F8441C43EA010002F8440C06F10106AE4244
:20B4C000FFF653AF71E700BF2DE9F04F2DED028B87B008EE100A0C4617469946129E139931
:20B4E000B5EEC08AF1EE10FA54BF00250125A84604F1FF33D8B2082807D8092A05D8A24672
:20B5000001F1FF32944205D808E001F1FF339C4240F2CD8001F1FF34E4B2C8E018EE100A69
:20B520000AF0F2FB48B930464FF03F0122460BF0E1FA4FF000013155C4E018EE100A0AF06C
:20B5400059FD06EE900AF2EE047AF4EEE76AF1EE10FA0DDB4FF00100B0EE677A00F10100F4
:20B5600067EE877AF4EEE76AF1EE10FAF6DA03E04FF00100F2EE047A21464319A34200F36D
:20B580009680C0EB040EC5EB0E0202F1FF3E4AF2F04AC0F6030ADFED9C4AF6EE003AB2EE3F
:20B5A000044AC0EB040CC5EB0C0303F0010BBEF1000F00F38F808AE0BEF1000F04DDBE45F8
:20B5C000B4BF72463A4601E04FF000025AF8223003EE103AB8EE430A20EE027AB4EEE47A42
:20B5E000F1EE10FA48BF37EE237ABDEEC73A13EE10CABCFBF3FB06EE10BAB8EEC65AB4EE47
:20B60000E75AF1EE10FA0DDB00F1010C87EE006A67EE847A0EF1FF3E6046BEF1000200F362
:20B62000C380BEE013EE105AB5FBF3F403FB14542CB916EE107A002F08BF4FF00008B9F167
:20B64000000F07D0C8EB0103181A002A18BF0138831A01E04FF0000301F10101B8F1000F75
:20B6600004D04BF2CC27C0F6030703E048F2E077C0F6030722B14BF2D020C0F6030003E036
:20B6800048F2E070C0F603004BF2E425C0F60305009501978DED026A039004920594304618
:20B6A0004BF2D422C0F603020AF0EEFD0AE03046002D0CBF2B212D2122460BF01BFA4FF00E
:20B6C0000000305507B0BDEC028BBDE8F08F4FF0000203E0BE45B4BF72463A465AF822305E
:20B6E00000EE103AB8EE405A65EE260AF4EEE40AF1EE10FA48BF70EEA30ABDEEE03A13EEBE
:20B7000010CABCFBF3FC06EE10CAF8EEC65AF4EEE75AF1EE10FA85DB00F1010080EE852A5A
:20B7200067EE847A0EF1FF3E42199142BFDBBBF1000F3FF441AFBEF1000F02DC4FF00002F7
:20B7400003E0BE45B4BF72463A465AF8223001EE103AF8EE411A21EE822AB4EEE42AF1EEF0
:20B7600010FA48BF32EE232ABDEEC23A13EE10BABBFBF3FB06EE10BAF8EEC62AF4EEE72AAE
:20B78000F1EE10FAFFF64EAF00F1010082EE212A67EE847A0EF1FF3E43199942BFF60CAFEB
:20B7A00085E74FF0000202E0BA42A8BF3A465AF8223006EE903AF8EE660A20EE861AB4EE0F
:20B7C000E41AF1EE10FA48BF31EE231ABDEEC13A13EE10BABBFBF3FB06EE10BAF8EEC65A46
:20B7E000F4EEE75AF1EE10FAFFF61CAF0CF1010081EE202A67EE847A0EF1FF3E4219914209
:20B80000BFF6DAAE53E700BF0000004BF8B505460F46F5F7DDFC064640F2A062C1F2000260
:20B820004FF4117303FB05F01418115811B18A682846904784F820724FF00005C4F8105250
:20B84000C4F81452C4F80451C4F808513046F5F7C9FC04F5097029464FF00802F5F772FCF5
:20B86000F8BD00BF70B588B0054640F2A064C1F200044FF4117303FB004494F820020028E0
:20B8800047D041F28821C2F200010878FF2803D04FF00401FFF7BAFF28464FF00001FFF7EF
:20B8A000B5FF41F28826C2F2000635704BF2F020C0F603004FF0070140F6B912C0F603028B
:20B8C000FBF71EFDC4F81C02246830784FF0010200924FF00002019249F6E523C0F60203A3
:20B8E00002934AF2DD01C0F60201039149F6FD73C0F60203049349F64561C0F60201059117
:20B90000069264684FF416514FF00803A047FEF7CBF908B070BD00BF08B5B0F1FF3F04D01B
:20B9200040B90246F7F768F808BD4FF000000246F7F762F808BD00BF38B505F0C5FB41F28B
:20B940008923C2F200034FF001021A704FF000042546E0B229462A46FFF726FA40B904F195
:20B960000104E0B229462A46FFF71EFA002867D04FF0FF304FF00001FFF7CEFF4FF0000034
:20B980004FF00001FFF780FA41F2E031C2F200010C6834B12368DA6802B190476468002C56
:20B9A000F8D141F28020C2F2000004683CB121680B680BB1A06898476468002CF7D1FAF78E
:20B9C000B1FBFEF761FA40F2A062C1F2000292F82002042806D028B14FF000004FF0040178
:20B9E000FFF714FF40F2A061C1F2000191F86434042B06D02BB14FF001004FF00401FFF7DB
:20BA000005FF40F2A062C1F2000292F8A806042806D028B14FF002004FF00401FFF7F6FEB7
:20BA200040F2A061C1F2000191F8EC38042B06D02BB14FF003004FF00401FFF7E7FE38BD3B
:20BA400004F10104B4F5807F83D191E738B5054641F26824C2F200042068FBF73BFD4FF0D8
:20BA6000000323608DB14BF20030C0F603004FF007014BF68132C0F60202FBF741FC41F285
:20BA80007422C2F20002106038BD41F27424C2F200042068FBF71EFD4FF000002060FAF72D
:20BAA000F5FEFFF749FF08F0F5FE41F28821C2F200010878FF2803D04FF00401FFF7A6FE81
:20BAC00038BD00BF70B541F2B420C2F200004BF21031C0F60301FBF743F841F28823C2F2DB
:20BAE00000034FF0FF021A7040F2A064C1F200044FF0040684F820624FF00005C4F81C52D7
:20BB00002846FBF717FA206084F86464C4F860544FF00100FBF70EFAC4F8440284F8A866BA
:20BB2000C4F8A4564FF00200FBF704FAC4F8880484F8EC68C4F8E8584FF00300FBF7FAF9E3
:20BB4000C4F8CC0641F23020C2F200004BF21C31C0F60301FBF704F841F29420C2F2000053
:20BB60004AF61451C0F603012A462B46FEF7FAFFFDF7B4FE4FF00100FFF768FF70BD00BF68
:20BB80002DE9F04F2DED0A8BABB01CAF26AC4AF2F015C0F6030595E80F0084E80F00A7609C
:20BBA00049F66903C0F60203E36020462AA9F8F76FFA22AE95E80F0086E80F00B76049F61C
:20BBC0008500C0F60200F06030462146F8F760FA4FF000041B9441F23020C2F20000214622
:20BBE000FAF7D6FF41F2A821C2F200010C71FFF7A3FE08F04FFE4FF00200FFF733FE41F2DA
:20BC0000DC32C2F2000215680DBB0CF031FDF0B9F6F77CFA10F0C20F19D14FF00300FEF7F3
:20BC20004DFC4FF47A754FF032063046FBF7A6FBF6F78AFC05F1FF343046FBF79FFBF6F77E
:20BC400083FC651EF1D14FF00000FEF737FC41F27023C2F200034FF000041C604FF001003D
:20BC6000187040F2A066C1F2000606F515652846214641F254520AF03DFF41F22C10C2F2CF
:20BC8000000021464FF480720AF034FF06F5116021464FF040020AF02DFF41F2DC20C2F27E
:20BCA000000021464FF0FC020AF024FF21954FF00A01C6F8741920462946FDF771FD41F20E
:20BCC0008C22C2F20002146041F29023C2F200031C6041F2DC35C2F200054FF030042C6077
:20BCE00040F20004C0F6010494F82F0000F1010094F82E1000EB0122101941F2D833C2F2B3
:20BD000000031860FBF7B4FF0B902868215CFF2920D141F2A822C2F200024FF001031371C8
:20BD200010604FF0FF00507141F27421C2F200014FF000020A6041F28823C2F20003187847
:20BD40004FF4117202FB0063D3F81C02FBF780F904F0FBBD05F096F94FF000070A97BA4652
:20BD60003C46DFEDBF8A9FEDBF9ADFEDBFAA9FEDBF8ADFEDBF9A9FEDBFAA01E04FF00004FF
:20BD80002CB94FF00000FEF75BFC4FF0640404F1FF3441F27026C2F20006357805F0F70246
:20BDA0006FF30412327041F2DC33C2F200031868099041F2DC36C2F2000640F20007C0F669
:20BDC000010741F27028C2F200084AF63459C0F6030931687D5C01F10101316098F800209E
:20BDE00012F0010F0ED10AF1010A40F2FF339A4508D941F2A823C2F200034FF03601197173
:20BE000004F06CBD0DF1700C28464946FEF784F94AF2A870C0F6030050F825204AF2185BD3
:20BE2000C0F6030B42F0010108473268BB5C0C9302F1010232600F2B04F248850DF1700C6C
:20BE400018465946FEF768F94AF20020C0F603000C9950F82120E5E73268BB5C0C9302F13D
:20BE600001023260102B02D91D4604F030BD0DF1700C0C984BF23411C0F60301FEF74CF93F
:20BE80004AF6A830C0F603000C9950F82120C9E73268BB5C0C9302F1010232600F2B02D906
:20BEA0001D4604F014BD0DF1700C0C984BF23821C0F60301FEF730F94AF25860C0F6030021
:20BEC0000C9950F82120ADE73268BB5C0C9302F1010232602F2B02D91D4604F0F8BC0DF18A
:20BEE000700C0C984AF24021C0F60301FEF714F94BF27810C0F603000C9950F8212091E7A5
:20BF00003268BB5C0C9302F1010232603B2B02D91D4604F0DCBC0DF1700C0C984AF200318E
:20BF2000C0F60301FEF7F8F84AF62440C0F603000C9950F8212075E73268BB5C0C9302F138
:20BF4000010232603F2B02D91D4604F0C0BC0DF1700C0C984AF2F031C0F60301FEF7DCF836
:20BF60004AF25850C0F603000C9950F8212059E73268BB5C0C9302F101023260432B02D995
:20BF80001D4604F0A4BC0DF1700C0C984AF29861C0F60301FEF7C0F84BF27030C0F603009A
:20BFA0000C9950F821203DE7219F97F846600DF1700CFDF757FB219D331895F8500000F0A4
:20BFC00001015A181C9285F84720FF2A94BF0022012285F85020D3E6219F97F846600DF101
:20BFE000700CFDF73FFB35181C95219B83F84750FF2D94BF0025012583F85050C0E60DF142
:020000040802F0
:20C00000700CFDF72FFB30B1219991F84720101C18BF012001E04FF00000219F87F8470031
:20C02000AEE60DF1700CFDF71DFB219E96F84750284086F84700A3E61D9BA3F1FB031C9353
:20C0400012E11D98A0F1FB001C909AE11D99A1F1FB011C91CBE11D9AA2F1FB021C9267E2AA
:20C0600000000034FFFF7F4BFFFF7FCB00000000FEFFFFCAFEFFFF4A1D9EA6F1FB061C966B
:20C080004FF002031B93F3E11D98A0F1FB001C901E991B911DE21D9AA2F1FB021C9217E19E
:20C0A0001D9EA6F1FB061C9699E21D9BA3F1FB031C93D5E21D9FA7F1FB071C971E981B90E6
:20C0C00012E31D99A1F1FB011C911E9A1B924FF000068DF86A60C0E31D9BA3F1FB031C93E5
:20C0E0001E981B904FF001018DF86A10B5E31D9AA2F1FB021C9200F04DBC1D9DA5F1FB05C9
:20C100001C9500F0A2BC9DF874004FF00101FEF709FE8DF86B0000283FF432AE41F2A824B0
:20C12000C2F20004207104F0D9BB1D9E1C964FF001038DF86A301E46219890F847100B4216
:20C1400005D09DF870003146FEF7ECFD68B99DF86A304FEA43008DF86A001C9A02F1010249
:20C160001C9210F0FE03E7D10CE09DF86A60012E08D19DF86B4041F2A821C2F200010C7197
:20C1800004F0ACBB0DF1700CFDF76CFAF8E59DF8740004F069FFF3E50DF1700CFDF762FA8C
:20C1A0001C9041F2DC36C2F2000630681C9900EB41023260FDF76CFA1C9001F0DDBC1D9882
:20C1C000FA2808D941F2A826C2F200064FF01304347104F083BB41F22C12C2F20002135CDE
:20C1E0001C93DEE7219991F852001C90D9E7219A92F850301C93D4E74FF0000AC0E50DF1AF
:20C20000700CFDF72FFA1C90219F97F847101B91FDF7DEFA87F84700B2E5219D95F84700CC
:20C2200095F84610FDF7D4FA85F85000A8E50DF1700CFDF73FFA1E9B41F22C16C2F2000670
:20C24000F05C1D9920EA0102F25499E541F2DC20C2F200004FF000014FF0FB020AF04AFC6C
:20C260008EE54FF000031C930DF1A80C1CF8386DFDF7F8F90146304606F0CCFE8DF86B009D
:20C2800000283FF47DAD41F2A824C2F20004207104F024BB05F04CFD72E505F051FD8DF8A1
:20C2A0006B0000283FF46CAD41F2A821C2F20001087104F013BB41F2D837C2F200073D6811
:20C2C0001D98281805F028FD5AE54FF000021C921C9B40F2A066C1F200064FF4117101FBB8
:20C2E000036090F82022032A3FD140F2A067C1F2000701FB03F303F58876B919FB1803F120
:20C3000004034FF00000D1F80021FE2A94BF551C0025D1F80471BD4214BF0025012565F329
:20C320000000BA4214BF0022012262F34100D3F80051FE2D94BF013500250DF1A80C4CF868
:20C34000385DD3F80461B54214BF0025012565F38200D3F80811D1F1010338BF002363F30F
:20C36000C300C0B2FDF766F90AE541F2A824C2F200044FF04803237104F0B0BA4FF00000D4
:20C380001C901C9E40F2A062C1F200024FF4117101FB062393F8200203281CD140F2A06766
:20C3A000C1F2000701FB0675D5F81022D5F81412531AB3F5807F88BF03F580731C931C98B1
:20C3C000FF2884BFFF201C900DF1A80C1CF8380DFDF730F9D4E441F2A824C2F200044FF052
:20C3E0004806267104F07ABA4FF000061C961C9B40F2A062C1F200024FF4117101FB0320B5
:20C4000090F82062032E24D140F2A067C1F2000701FB037505F58876D6F80021D6F80411BB
:20C42000501AB0F5807F88BF00F580701C900DF1700CFDF717F98DF86A001C9B984238BF21
:20C440001C90D6F804711C9DEA19D1B2C6F8041196E441F2A824C2F200044FF0480323718C
:20C4600004F03CBA4FF000061C964FF002001B901C9B40F2A062C1F200024FF4117101FB8E
:20C48000032696F82002032815D140F2A067C1F2000701FB03750DF1700C1B9849F2E5718D
:20C4A000C0F6020149F2F972C0F6020205F58873FDF712F964E441F2A824C2F200044FF031
:20C4C0004803237104F00ABA4FF000021C921D991B911C9E40F2A060C1F200004FF411730E
:20C4E00003FB060292F82012032915D140F2A067C1F2000703FB06750DF1700C1B9849F294
:20C50000E571C0F6020149F2F972C0F6020205F58873FEF729F933E441F2A824C2F20004D2
:20C520004FF04806267104F0D9B94FF000001C901C9B40F2A062C1F200024FF4117101FB05
:20C54000032696F8200203283DD140F2A067C1F2000701FB037505F588750DF1700CFDF7FD
:20C5600081F88DF86A00D5F804211C924FF000011B91D5F800711346974207D0AE5C8642AE
:20C5800019D04FF001024FF0000E0CE04FF0FF001B9010E002F10106E95C814202D11C93DA
:20C5A0001B9208E03246FF2B14BF013373469F42F0D11C93EAE70DF1700C9DF86C00FDF7F3
:20C5C00039F8FFF7DDBB41F2A824C2F200044FF04803237104F082B94FF000031C931C9EED
:20C5E00040F2A062C1F200024FF4117101FB062090F82032032B27D140F2A065C1F200057C
:20C6000001FB065707F58875D7F81462D7F81022964212D00DF1700CFDF724F88319DFB211
:20C620001C970DF1700CE85DFDF704F84FF00005219E86F85050FFF7A3BB4FF00101219829
:20C6400080F85010FFF79CBB41F2A824C2F200044FF04806267104F041B94FF000021C92FD
:20C660001C9840F2A063C1F200034FF4117101FB003696F82022032A28D140F2A067C1F242
:20C68000000701FB007505F58876D6F80431D6F800118B4213D00DF1700CF05CFCF7CAFF16
:20C6A000D6F80471FF2F14BF01370027C6F804714FF00005219E86F85050FFF761BB4FF032
:20C6C0000102219880F85020FFF75ABB41F2A824C2F200044FF04800207104F0FFB84FF0F2
:20C6E00000031C931D991B9141F2D832C2F20002D2F800801B9F08EB070640F20000C0F647
:20C700000200864208D941F2A826C2F200064FF01F02327104F0E2B81C9B032B08D941F229
:20C72000A820C2F200004FF03703037104F0D6B8F1780D2908D941F2A824C2F200044FF098
:20C740003701217104F0CAB840F2A065C1F200054FF4117202FB035090F820323BB118F8BE
:20C76000071021B10FE04846FDF76AFF05E04CF24F354FF09609DDF82CB0FBF779FACBEBA5
:20C780000002AA42EFD918F80770032F3FF6F8AADFE807F002080F169DF87000FFF762F811
:20C7A000FFF7EEBA9DF87000314606F04DFCFFF7E7BA9DF87000314605F03CFAFFF7E0BA52
:20C7C0009DF87050B77828464FF00301FFF71EF84FF4117000FB05F340F2A061C1F200017A
:20C7E000C85800283FF4CCAA4AF62053C0F6030307EB470703EB0708F6784AF6EC32C0F61A
:20C80000030252F82610DA5D98F8013098F8027000974FF00006019649F6B537C0F602073C
:20C82000029749F6F537C0F60207039749F62547C0F60207049749F64567C0F60207059750
:20C84000069646682846B047FFF79ABA4FF000011C911D981B908DF86A101C9840F2A063AA
:20C86000C1F200034FF4117101FB003696F82022032A79D140F2A065C1F2000501FB005782
:20C8800007F5887941F2D833C2F200031968219EB26B01EB020B8B5CFF2B5CD0D8464FF0B6
:20C8A00001054FF0000B0994CDF830A0AA4698F8014004EB032741F2D833C2F200031E68A1
:20C8C000F219D9F804111C919DF86A0018B1F75D02F1010200E05F4602F1FF349DF86A50AE
:20C8E0002DB177B9099C5046DDF830A005E063783BB9099C5046DDF830A01C99C9F804112B
:20C900002BE01C99D9F800618E4218D014F8016F19F801501B9A3AB9304609F059FCC6B2AB
:20C92000284609F055FCC5B2AE4208D11C98FF2814BF013058461C9007F1FF37CEE70AF1F8
:20C94000010A18F8023FFF2BB1D1099CDDF830A04FF0000001E04FF000000DF1700CC0B23A
:20C96000FCF768FEFFF70CBA41F2A824C2F200044FF04800207103F0B1BF4FF000031C937F
:20C980001E9E1B964FF001028DF86A2065E74FF000021C921C9E40F2A060C1F200004FF4BC
:20C9A000117303FB060191F82022032A31D140F2A065C1F2000503FB065707F588750DF1B3
:20C9C000700CFCF74FFE8DF86A004FF000031C93D5F80471D5F800118F4212D0EA5D8242DD
:20C9E0000FD14FF00006FF2F14BF01373746B94202D1C5F8047104E0EB5D8342F3D0C5F8EB
:20CA000004710DF1700C4FF00000FCF713FEFFF7B7B941F2A824C2F200044FF048062671A3
:20CA200003F05CBFFBF724F90B9D401B0DF1700C4CF24F37B8428CBF00200120FCF7FAFD28
:20CA4000FFF79EB94FF000001C901C9E40F2A062C1F200024FF4117101FB062393F8205214
:20CA6000032D7FF48DA940F2A067C1F2000701FB067000F10406D0F80811D6F8002102F1BA
:20CA80000102914238BF01F580718B1AFF2B34BF1D46FF250DF1700CE8B2FCF7CBFDFFF7D4
:20CAA0006FB91D9F41F22C10C2F20000C65D06F1FF31C155FFF764B91D9BFA2B08D941F20B
:20CAC000A824C2F200044FF01300207103F006BF41F22C10C2F20000C25C02F1FF36F1B22B
:20CAE000C15400293FF44CA91E9B1C9301F044B81D9EFA2E08D941F2A824C2F200044FF0C1
:20CB00001306267103F0EABE41F22C11C2F200018A5D02F1FF33D8B28855002842F037841D
:20CB2000FFF72EB91D9BFA2B08D941F2A824C2F200044FF01303237103F0D0BE41F22C11C9
:20CB4000C2F20001CA5C02F1FF30C6B2CE54002E02F01D84FFF714B9219D95F8517007F1B6
:20CB6000FF3185F85110FFF70BB9219890F8472002F1FF3680F84760FFF702B9219BD86C4D
:20CB800009F038FA219DE864FFF7FAB8219F97ED137AD7ED127A37EE270A87ED130A2199F6
:20CBA000C86C09F091F830B14FF00205219981F85050FFF7E5B8219BD86C09F095F830B1CB
:20CBC0004FF00102219880F85020FFF7D9B84FF00006219F87F85060FFF7D2B89DF874002E
:20CBE000219901F14C01FEF71BF98DF86B0000283FF4C6A841F2A824C2F20004207103F03F
:20CC00006DBE9DF874002199C96CFEF73DF98DF86B0000283FF4B4A841F2A822C2F200026C
:20CC2000107103F05BBE2198C06C09F05DF820B9219EB06C09F058F830B14FF00300219E55
:20CC400086F85000FFF79CB8219BD3ED13BA93ED12BA7BEECB0A10EE900A09F0CBF90CEE9A
:20CC6000100A1BEE900A1BEE101A09F039F901464FF07E5009F034F901EE100A61EE281A85
:20CC8000B4EEE1CAF1EE10FA06D84FF00001219A82F85010FFF774B8219D95ED132AD5ED4A
:20CCA000122AB4EEE22AF1EE10FA05DD4FF0010785F85070FFF764B8B4EEE22AF1EE10FA92
:20CCC0004CBF0222032285F85020FFF759B8219B93ED133AF7EE003A33EE634A83ED134AC9
:20CCE0002198C06C09F000F830B14FF00307219981F85070FFF744B8219A92ED13BA7BEEDF
:20CD000049BA1BEE900A09F075F90BEE900A1BEE100A19EE101A09F0E3F801464FF07E50F7
:20CD200009F0DEF800EE100A60EE280AF4EEE0BAF1EE10FA1ED9219E96ED13BA3BEE091AE5
:20CD400011EE100A09F056F90BEE900A1BEE100A1AEE901A09F0C4F801464FF07E5009F008
:20CD6000BFF801EE900A21EEA82AF4EEC2BAF1EE10FA06D84FF00406219B83F85060FEF748
:20CD8000FFBF219BDF6C384609F034F90BEE100A384618EE101A09F0A3F801464FF07E5081
:20CDA00009F09EF802EE900A22EEA83AB4EEC3BAF1EE10FA06D84FF00000219A82F85000BE
:20CDC000FEF7DEBF2199D1ED133AF4EEC83AF1EE10FA05DD4FF0010581F85050FEF7D0BF6B
:20CDE000F4EEC83AF1EE10FA4CBF0222032281F85020FEF7C5BF219DD5ED124A95ED135AE5
:20CE0000C4EE855AC5ED135AC9E62199C86C08F057FF002840F0AE86FEF7B2BF219AD66C88
:20CE2000304609F0E7F80BEE100A304618EE101A09F056F801464FF07E5009F051F806EE1A
:20CE4000100A66EE286AB4EEE6BAF1EE10FA00F39186FEF795BF2198C06C08F031FF00281F
:20CE600000F08886FEF78CBF219B93ED137AD3ED127AB4EEE77AF1EE10FA80F27B86FEF70B
:20CE80007FBF219991ED130AD1ED120AB4EEE00AF1EE10FA00F36E86FEF772BF219A92ED69
:20CEA000131AD2ED121AB4EEE11AF1EE10FA40F26186FEF765BF219E96ED132AD6ED122A24
:20CEC000B4EEE22AF1EE10FA00F15486FEF758BF2198C66C304609F08DF80BEE100A30467C
:20CEE00018EE101A08F0FCFF01464FF07E5008F0F7FF03EE100A63EE283AB4EEE3BAF1EEF1
:20CF000010FA40F23786FEF73BBF219FF86CFCF7E1F9F8640DF1700C4FF00000FCF776FCBE
:20CF2000FEF72EBF1D9BF62B08D941F2A824C2F200044FF01203237103F0D0BC219DE86C25
:20CF400008F0BEFE38B9219AD2ED134AB6EE005A34EE85BA06E0219991ED13BAB6EE004A1D
:20CF60003BEE44BA1BEE100A08F0AAFE88B9B4EECABAF1EE10FA04DC1BEE100A08F0A4FEDA
:20CF800038B14FF00100219E86F850006FF000402CE01BEE100A08F093FE88B1B4EEE9BA06
:20CFA000F1EE10FA04D41BEE100A08F08DFE38B14FF00101219A82F850104FF0004015E0D7
:20CFC0001BEE100A08F090FE38B14FF00205219B83F850504FF0000008E0BDEECBBA1BEE42
:20CFE000100A4FF00006219F87F850604FEA006747EA106500F47F4345EA032100F47F021F
:20D0000041EA122041F2DC26C2F200061D9FF051FEF7B6BE1D99F62908D941F2A824C2F2F5
:20D0200000044FF01203237103F058BC41F2DC25C2F200056A584FEA026040EA126602F41B
:20D040007F4746EA072302F47F0143EA112505EE905AB8EEE56A219880ED136AB4EECA6A8C
:20D06000F1EE10FA04DCB4EEE96AF1EE10FA05D54FF0010680F85060FEF782BE4FF000024B
:20D0800080F85020FEF77CBE0DF1700C4FF00100FCF7BCFB219FF86CFCF746F92199C864D9
:20D0A000FEF76EBE219DD5ED136AB7EE007A76EE877AC5ED137A13E6219DE86C08F014FE7A
:20D0C00050B1219F4FF0000187F847104FF0040587F85050FEF754BE219890ED134AB4EED6
:20D0E000C84AF1EE10FA23DB9FEDD66AB4EEC64AF1EE10FA0FD5FCEEC46A16EE902A0DF118
:20D10000700CD0B2FCF796FA4FF00006219B83F85060FEF735BE0DF1700C4FF0FF00FCF7CF
:20D1200089FA4FF00205219880F85050FEF728BEB4EEC84AF1EE10FA7EF522AEDFEDC24AC2
:20D14000B4EEE44AF1EE10FA11DDB1EE445AFCEEC55A15EE903A0DF1700CD8B2FCF76AFABA
:20D160004FF00107219981F85070FEF709BE0DF1700C4FF0FF00FCF75DFA4FF00302219EB4
:20D1800086F85020FEF7FCBD1D98F92808D941F2A824C2F200044FF01300207103F09EBB56
:20D1A000219A92ED137AFDEEC77A17EE906A33B21C939FB2C6F3072141EA072541F22C12EF
:20D1C000C2F200021552FEF7DBBD1D9EF92E08D941F2A824C2F200044FF01306267103F049
:20D1E0007DBB219B93ED130AFCEEC00A10EE907ABDB21C954FEA152141EA052241F22C1092
:20D20000C2F200008253FEF7BBBD1D9F219B9F64FEF7B6BD1D9D2199CD64FEF7B1BD0DF12F
:20D22000700CFCF71FFA01EE100AF8EE411A219AC2ED131AFEF7A4BD1D98F92808D941F245
:20D24000A824C2F200044FF01300207103F046BB41F22C16C2F20006375A4FEA172343EA13
:20D260000725A9B202EE101AF8EE422A219AC2ED132A9FED763AF4EEC32AF1EE10FAFEF62C
:20D280007FADDFED733A32EEE34A82ED134AFEF777BD1D9EF92E08D941F2A824C2F200042D
:20D2A0004FF01306267103F019BB41F22C17C2F20007BB5B4FEA132545EA03218AB204EE7F
:20D2C000902AB8EE645A219880ED135AFEF758BD1D98072808D941F2A823C2F200034FF0DA
:20D2E0000801197103F0FABAFCF710FE05EE900AB8EE656A219F87ED136AFEF741BD219D8F
:20D30000D5ED136A95ED127A66EE877AC5ED137A45E4219A92ED130AF1EE400AC2ED130AB7
:20D32000FEF72EBD4FF000004FF001010A46FDF73BFD219890ED131AF1EE041A21EE212A57
:20D340004FF000060096019641F2E430C2F20000FCEEC22A12EE901A4FF0FF024AF60D63F0
:20D36000C0F60203FAF74EFCFEF70ABD1D9BF72B08D941F2A824C2F200044FF013022271A2
:20D3800003F0ACBA41F22C17C2F20007F858FBF7CBFF21998864FEF7F3BC1D98F72808D9F8
:20D3A00041F2A823C2F200034FF01301197103F095BA41F22C15C2F200052858FBF7B4FF47
:20D3C000219EF064FEF7DCBC1D9A072A08D941F2A824C2F200044FF00806267103F07EBA1E
:20D3E000219F97ED133AB4EEC83AF1EE10FA0DDBB4EEC93AF1EE10FA08D8FCEEC33ACDED18
:20D400001C3A4FF0000587F8505028E0B4EEC93AF1EE10FA07DD6FF07F421C924FF00100CB
:20D4200087F850001BE04FF000001C9013EE100A08F046FC70B14FF00201219B83F85010E8
:20D440000DE000BF00008043000080C300000047800080474FF00305219E86F850501D98B3
:20D460001C99FCF725FDFEF78BBC219FF86C08F03BFC00287EF484AC219991ED134AB4EE52
:20D48000C84AF1EE10FA04DD4FF07E52CA64FEF777BCB4EEC84AF1EE10FA7EF571AC4FF0DF
:20D4A0000003CBF68073CB64FEF76ABC2198856ACDB1FAF7DDFB219FB96AC1F104031818B0
:20D4C0004CF6CD42CCF6CC42A2FB00154FEA9506796AB6FBF1F304EE903AB8EE645A87ED99
:20D4E000135AFEF74DBC4FF6FF76C7F67F76C664FEF746BC1D9EF72E08D941F2A824C2F2C0
:20D5000000044FF01300207103F0E8B9219FF86CFBF7E0FE41F22C12C2F200029051FEF79F
:20D520002FBC219DD5ED125A95ED136A75EEC66AC5ED136AFFF733BB219BDE6C1C969F6CAC
:20D54000DF649E64FEF71CBC219AD06C08F0CCFB30B14FF00306219981F85060FEF710BC36
:20D560002198C06C08F0B0FB30B14FF00400219D85F85000FEF704BC219DEE6C304608F039
:20D5800039FD0BEE100A304618EE101A08F0A8FC01464FF07E5008F0A3FC07EE100A67EEB1
:20D5A000287AB4EEE7BAF1EE10FA06D84FF00007219A82F85070FEF7E3BB219991ED130A9C
:20D5C000B4EEC80AF1EE10FA05DD4FF0010381F85030FEF7D5BBB4EEC80AF1EE10FA4CBFE3
:20D5E0000222032281F85020FEF7CABB219BD3ED13BA93ED12BA3BEECBCA1CEE100A08F010
:20D60000F9FC0CEE100A1BEE900A1BEE101A08F067FC01464FF07E5008F062FC00EE900A9E
:20D6200020EEA81AB4EEC1CAF1EE10FA0DF1700C8CBF00200120FBF7FDFFFEF7A1BB219FFF
:20D64000FD6C284608F0D6FC0BEE100A284618EE101A08F045FC01464FF07E5008F040FCB7
:20D6600001EE900A21EEA82AB4EEC2BAF1EE10FA0DF1700C8CBF00200120FBF7DBFFFEF772
:20D680007FBB219AD2ED132A92ED123AF4EEC32AF1EE10FA0DF1700CB4BF00200120FBF7F6
:20D6A000C9FFFEF76DBB2198D0ED133AF5EEC03AF1EE10FA0DF1700CB4BF00200120FBF7DC
:20D6C000B9FFFEF75DBB219E96ED134AD6ED124AB4EEE44AF1EE10FA0DF1700CD4BF0020E1
:20D6E0000120FBF7A7FFFEF74BBB219991ED135AD1ED125AB4EEE55AF1EE10FA0DF1700C63
:20D700008CBF00200120FBF795FFFEF739BB219B93ED136AD3ED126AB4EEE66AF1EE10FA3E
:20D720000DF1700C54BF00200120FBF783FFFEF727BB219F97ED137AB5EEC07AF1EE10FA39
:20D740000DF1700C54BF00200120FBF773FFFEF717BB219DD5ED13BA95ED12BA7BEECB7A87
:20D7600017EE900A08F046FC0CEE100A1BEE900A1BEE101A08F0B4FB01464FF07E5008F0F3
:20D78000AFFB00EE100A60EE280AB4EEE0CAF1EE10FA0DF1700CD4BF00200120FBF74AFF99
:20D7A000FEF7EEBA219AD66C304608F023FC0BEE100A304618EE101A08F092FB01464FF07E
:20D7C0007E5008F08DFB01EE100A61EE281AB4EEE1BAF1EE10FA0DF1700CD4BF00200120ED
:20D7E000FBF728FFFEF7CCBA1D98F82808D941F2A824C2F200044FF01303237103F06EB826
:20D80000FAF736FA219B00F104004CF6CD41CCF6CC41A1FB00174FEA97055A6AB5FBF2F732
:20D820001D9D41F22C10C2F2000041194E78425D4FEA024545EA0620897840EA01061B9694
:20D84000BF1B27F07F421C9202EE102AF8EE422AC3ED132AFEF794BA219DE86CA864FEF7A9
:20D860008FBA219991F85160002E40F08381FEF787BA219A92F85130002B00F07B81FEF701
:20D880007FBA1D98FA2808D941F2A824C2F200044FF01303237103F021B841F22C11C2F207
:20D8A00000010E5C002E7EF46BAA1E9A1C9263E11D98FA2808D941F2A824C2F200044FF0F0
:20D8C0001303237103F00AB841F22C11C2F200010E5C002E3EF454AA1E9A1C924CE141F236
:20D8E000A820C2F200004FF00101017102F0F6BF1D9EF92E08D941F2A824C2F200044FF099
:20D900001206267102F0EABF41F2DC22C2F20002905D1E9B18427EF433AA1F991C912BE116
:20D920001D98F92808D941F2A824C2F200044FF01200207102F0D2BF41F2DC22C2F200022D
:20D94000115C1E9B19423EF41BAA1F9E1C9613E11D99FA2908D941F2A824C2F200044FF03C
:20D960001300207102F0BABF41F22C12C2F20002535C002B7EF404AA1E9E1C962DE11D9945
:20D98000FA2908D941F2A824C2F200044FF01300207102F0A3BF41F22C12C2F20002535CBF
:20D9A000002B3EF4EDA91E9E1C9616E11D99FA2908D941F2A824C2F200044FF013012171B9
:20D9C00002F08CBF41F22C12C2F20002565C1E9B9E427EF6D5A91F981C90CDE01D9EFA2EB3
:20D9E00008D941F2A824C2F200044FF01306267102F074BF41F22C12C2F20002905D1E9BAE
:20DA00009842FEF4BDA91F991C91B5E01D98FA2808D941F2A824C2F200044FF01300207188
:20DA200002F05CBF41F22C12C2F20002115C1E9B99427EF4A5A91F9E1C969DE01D99FA292C
:20DA400008D941F2A824C2F200044FF01301217102F044BF41F22C12C2F20002565C1E9BC2
:20DA60009E423EF48DA91F981C9085E01D9EFA2E08D941F2A824C2F200044FF0130626712C
:20DA800002F02CBF41F22C12C2F20002905D1E9B98423EF675A91F991C916DE01D98FA2827
:20DAA00008D941F2A824C2F200044FF01300207102F014BF41F22C12C2F20002115C1E9BD9
:20DAC0009942BEF45DA91F9E1C9655E0219A92F847101D9B99427EF453A91E9E1C967CE0A8
:20DAE000219890F847201D998A423EF449A91E9B1C9372E0219E96F847001D9A90427EF68D
:20DB00003FA91E991C9168E0219B93F847601D988642FEF435A91E9A1C925EE0219991F84F
:20DB200047601D9B9E42BEF42BA91E981C9054E0219A92F847101D9EB1423EF621A91E9B89
:20DB40001C934AE09DF874000DF16B01FDF748F88DF86A009DF86B1031B141F2A824C2F2B1
:20DB60000004217102F0BABE00283EF409A91E981C9001E01D9A1C921C9A40F20000C0F653
:20DB8000010090F82E1090F82F3043EA0126964208D241F2A824C2F200044FF0090222713D
:20DBA00002F09CBE41F2DC37C2F200073A60FEF7E7B80DF1700CFBF755FD1C900028D9D0AF
:20DBC000FEF7DEB80DF1700CFBF74CFD1C900028D0D1FEF7D5B81D9E1C96219E336A052B15
:20DBE00008D941F2A824C2F200044FF00A03237102F074BE03F1020241F2DC30C2F200009E
:20DC0000016846F8221003F10103219E3362B3E70DF1700CFBF726FD1C900028DBD0FEF742
:20DC2000AFB80DF1700CFBF71DFD1C900028D2D1FEF7A6B80DF1700CFBF714FD1C901D9B4C
:20DC400098427EF49DA81E991C9195E70DF1700CFBF708FD1C901D9A90423EF491A81E988C
:20DC60001C9089E70DF1700CFBF7FCFC1C901D9EB0427EF685A81E9B1C937DE70DF1700CE4
:20DC8000FBF7F0FC1C901D998842FEF479A81E9A1C9271E70DF1700CFBF7E4FC1C901D9EF6
:20DCA000B042BEF46DA81E981C9065E70DF1700CFBF7D8FC1C901D9B98423EF661A81E998B
:20DCC0001C9159E79DF874000DF16B01FCF756FF8DF86A009DF86B6036B141F2A824C2F2B3
:20DCE0000004267102F0FABD00283EF449A81E9A1C9241E79DF874000DF16B01FCF73EFF64
:20DD00008DF86A009DF86B3033B141F2A821C2F200010B7102F0E2BD00287EF431A81E9819
:20DD20001C9029E70DF1700CFBF7C4FC41F22C16C2F200061E9AB05C1D9B18423EF420A8FC
:20DD40001F991C9118E70DF1700CFBF7B3FC41F22C16C2F200061E9AB05C1D9B18427EF4CD
:20DD60000FA81F991C9107E70DF1700CFBF7A2FC41F22C16C2F200061E9AB05C1D9B18428A
:20DD80007DF4FEAF1F991C9127E70DF1700CFBF791FC41F22C16C2F200061E9AB05C1D9B4E
:20DDA00018423DF4EDAF1F991C9116E798F8005045F0080288F80020FEF70BB80DF1700CE9
:20DDC000FBF750FC8DF86A00219991F851601D9BF1181C911E9AC2F1FB06B14208D941F241
:20DDE000A824C2F200044FF01303237102F076BD4FF000071B971E9DEDB11C9941F22C1319
:20DE0000C2F200035A5C824236D005F1FF3241F22C16C2F20006731841F22C15C2F20005BD
:20DE2000C5F10107C1F10101C5EB010E12F0010F1AD002F0AEBD4FF0FF001B901CE013F868
:20DE4000019F02F1FF35484504D11C91CDF86CC01E9211E02A46F9180EEB030C13F8016F56
:20DE6000B04242F0A385F0E7F9180EEB030C002AE5D11C911E92DEE70DF1700C9DF86C00E9
:20DE8000FBF7D8FBFDF77CBF0DF1700CFBF7EAFB41F2582BC2F2000B8BF800004FF0010104
:20DEA0001C91CDF834B095E0219E96F851201D9813181C93F92B08D941F2A824C2F200048E
:20DEC0004FF01301217102F009BD1E981B900DF1700C26AF47F0010122AD45F001024FF076
:20DEE0000003FBF7F9FBFDF74BBF219E96F851201D9813181C93FA2B08D941F2A824C2F235
:20DF000000044FF01301217102F0E8BC1F9F1E98B84228BF38461B900DF1700C26AD45F082
:20DF2000010122AE46F001024FF00003FCF71CFCFDF726BF0DF1700CFBF794FB034641F239
:20DF4000582BC2F2000B58464FF010014BF22432C0F6030208F098F91C90CDF834B039E04C
:20DF60001E9A1C921F981B904FF000030D9331E04FF0FF361C960D962CE02199C86C9DF88E
:20DF800078109DF87C2041F25826C2F2000600964FF0100301934FF00103FDF795FA4FF0DC
:20DFA000FF321C920D9615E02198C06C9DF878109DF87C2041F25826C2F2000600964FF077
:20DFC000100301934FF00003FDF77EFA4FF0FF311C910D961D9800F10506F2B20C92A0F1A9
:20DFE000FB01032923D840F2A060C1F200004FF411760C9A06FB020191F82032032B08D0C4
:020000040802F0
:20E0000041F2A820C2F200004FF04806067102F065BC40F2A060C1F200004FF411770C9EE0
:20E0200007FB060707F104074FF0000605E0219F97F851301E184FF00007DDF870B0BBF1B7
:20E04000FF3F0CD14FF0FF0B4FF00009C84641F22C12C2F200020E920F950D9D05E0BBF160
:20E06000000FF1D14FF0000961E01D99A1F1FB01032910D8D7F80061FF2E14BF01364646FB
:20E08000D7F804319E4206D14046FCF7D9FAD7F804018642F8D0B5F1FF3F15D1219850F84A
:20E0A000343F1A68D2F800C0494610AA4FF00103E0478DF86B0080B10F9D41F2A824C2F2AE
:20E0C0000004207102F00ABC25B115F809108DF8401002E01B9A8DF840201C98B0F1FF3F13
:20E0E00002D19DF8401011B31D9BA3F1FB03032B07D8D7F800119DF840307B54C7F8006179
:20E1000011E0FA2E09D90F9D41F2A824C2F200044FF01306267102F0E1BB9DF840200E9889
:20E12000825506F1010609F10109D9459DD31D9FA7F1FB07032F04D80C98FBF723FDFDF76A
:20E140001FBE219D95F8512009EB020E85F851E0FDF716BE1D9AA2F1FB0003285AD802F117
:20E160000502D7B240F2A060C1F200004FF4117101FB070292F82032032B08D041F2A8247F
:20E18000C2F200044FF04803237102F0A7BB40F2A066C1F200064FF4117505FB076505F139
:20E1A00004051E9800F1FF311E9170B34FF0000841F2DC39C2F2000940F200029346C0F69E
:20E1C000010BD5F80061FF2E14BF01364646D5F804319E4206D14046FCF732FAD5F8040112
:20E1E0008642F8D0D9F80030D5F800211BF80310A95403F10103C9F80030C5F800611E9EBA
:20E2000006F1FF301E90002EDBD13846FBF7BAFCFDF7B6BD1E9B1C93219991F8510082182D
:20E220001B92C3F1FB06B24208D941F2A824C2F200044FF01306267102F050BBC71881F8AC
:20E2400051701C9A02F1FF351C95002A3DF498AD41F2DC33C2F200031E681B9F41F22C1126
:20E26000C2F20001C91940F20000C0F6010030184FF0000305F0010E10F803C001F803C009
:20E2800003F10103934242F075830DE010F8038001F8038003F1010310F803E001F803E0D4
:20E2A00003F101039342F1D1E819A91901F1010141F2DC32C2F2000211604FF0FF331C9390
:20E2C00000F101001B90FDF75BBD4FF000028DF86A20219E96F851001D9BC1181C911E9AB1
:20E2E0001B92C2F1FB00814208D941F2A824C2F200044FF01303237102F0F0BA41F22C176D
:20E30000C2F2000707EB01099DF87CB041F2D835C2F200052A68B66B9119975DFF2F52D0EB
:20E3200088464FF0010009900C9498F8014004EB072741F2D835C2F200052A68D6194FF0EF
:20E3400000011C919DF86A30002B02F0EB82D75D06F1010602F0E8BA9DF86A5015B15FB963
:20E360000C9C02E062783AB90C9C219E96F85120851886F8515029E014F8015F19F800B0EE
:20E3800046B9284607F024FFC5B2584607F020FF5FFA80FB5D4508D11C9800F101001C902A
:20E3A00007F1FF371B998142D6D2B346099B03F10103099318F8027FFF2FB6D10C9C4FF0B2
:20E3C0000000099002E04FF0000309930DF1700C0999C8B2FBF72EF9FDF7D2BC4FF0010172
:20E3E0008DF86A1075E70DF1700CFBF73BF9034641F2582BC2F2000B58464FF010014BF239
:20E400002C32C0F6030207F03FFF1C90CDF834B0E0E50DF1700CFBF725F9034641F2582B0B
:20E42000C2F2000B58464FF010014BF23432C0F6030207F029FF1C90CDF834B0CAE50DF1B0
:20E44000700CFBF70FF9034641F2582BC2F2000B58464FF010014BF23832C0F6030207F041
:20E4600013FF1C90CDF834B0B4E50DF1700CFBF7F9F8034641F2582BC2F2000B58464FF0A4
:20E4800010014BF24032C0F6030207F0FDFE1C90CDF834B09EE5219991F8513003F101037B
:20E4A00081F85130FDF76CBC1D9F41F22C15C2F20005EA5D02F10102EA55FDF761BC219817
:20E4C00090F8476006F1010680F84760FDF758BC9DF874000DF16B01FCF750FB0DF1700CBD
:20E4E000FBF7A8F89DF86B1000293DF449AC41F2A824C2F20004217102F0F0B99DF874003E
:20E500000DF16B01FCF7A6FB0DF1700CFBF792F89DF86B30002B3DF433AC41F2A822C2F2EB
:20E520000002137102F0DAB91D981C904FF000061B964FF001018DF86A109DF870000DF136
:20E540006B01FCF71BFB9DF86B309BB920B19DF86A201B9810431B909DF86A604FEA460142
:20E560008DF86A101C9B03F101031C9311F0FE0FE3D10AE09DF86A20012A06D141F2A82472
:20E58000C2F20004237102F0A9B90DF1700C9DF86C00FBF74FF8FDF7F3BB1D981C904FF0E5
:20E5A00000061B964FF001018DF86A109DF870000DF16B01FCF74EFB9DF86B309BB920B164
:20E5C0009DF86A201B9810431B909DF86A604FEA46018DF86A101C9B03F101031C9311F02E
:20E5E000FE0FE3D10AE09DF86A20012A06D141F2A824C2F20004237102F070B90DF1700C6F
:20E600009DF86C00FBF716F8FDF7BABB9DF874000DF16B01FCF7E4FA8DF86A009DF86B60FD
:20E6200036B141F2A820C2F20000067102F056B90DF1700CFAF7FEFFFDF7A2BB1D991C91B0
:20E640004FF000031B934FF001008DF86A00219A92F8476030420ED09DF870000DF16B01F0
:20E66000FCF7BEFA9DF86B1099B920B19DF86A001B9B03431B939DF86A204FEA42068DF8EE
:20E680006A601C9901F101011C9116F0FE00DED10AE09DF86A30012B06D141F2A824C2F2D8
:20E6A0000004217102F01AB91B9F219D85F84770FDF766BB9DF874000DF16B01FCF7FCFAE2
:20E6C0000DF1700CFAF7B6FF9DF86B60002E3DF457AB41F2A822C2F20002167102F0FEB877
:20E6E0001D991C91C8B20DF16B01FCF7E5FA1B909DF86B0030B141F2A824C2F2000420712D
:20E7000002F0ECB84FF001038DF86A301C9FFA181C92D0B20DF16B01FCF7CEFA9DF86A5090
:20E7200000FA05F01B9E06431B9605F101058DF86A501C9A02F101021C92E9B20729E8D916
:20E740000DF1700C9DF86C00FAF774FFFDF718BB0DF1700C219890F85100FAF76BFFFDF7B8
:20E760000FBBFDF70DBB41F28923C2F200034FF001071F70FDF704BB41F28925C2F200055A
:20E780004FF000062E70FDF7FBBA21984FF000014FF0540208F0AEF94FF00002219241F299
:20E7A0008C21C2F200010C6804F1FF30086002F001B841F28C22C2F2000211683F2908D9F3
:20E7C00041F2A824C2F200044FF03000207102F085B84FF001071C9740F2A065C1F200056A
:20E7E000D5F8A809002842F0AA8005E0D6F8AC20002A4ED11C9301E04FF001031D9840F295
:20E80000A066C1F200064FF0540505FB03F3F218C2F85009C2F854091E9982F8A2194FF04C
:20E820000A07C2F8747906F51567F81800F13400219901F134014FF0100208F037F91C9B63
:20E8400005FB037000F14400219901F144014FF0040208F02BF91C9805FB007000F1480061
:20E86000219901F148014FF0080208F01FF9219A92F851101C9F05FB076686F8A11941F211
:20E880008C25C2F200052B6803F101032B60FDF777BA03F101010B4606F15406D6F8AC7051
:20E8A000002F42F05780A5E71C93FDF769BA219B93F852601E967CE70DF1700CFAF7D2FE83
:20E8C0001E9076E71D9A219981F85120FDF758BA0DF1700C9DF87400FAF7ACFEFDF750BAB0
:20E8E000219EB36A002B3DF44BAAF9F7C1F921998A6A801A4E6A1D9B06FB03F303EB830120
:20E900008842BDF43DAA1E9A1C92FFF735B9F9F7AFF9219FB862FDF733BA41F2DC20C2F215
:20E92000000090F8FB201E9E9319FB2B08D941F2A820C2F200004FF01206067101F0CEBFCA
:20E940001D9BC2F1FB018B4208DD41F2A824C2F200044FF01302227101F0C0BF41F2DC255C
:20E96000C2F20005A81941F22C17C2F20007F91808F09CF8FDF704BA98F8003043F0100199
:20E9800088F80010FDF725BA219D95F84770002F0CBFFF22002285F84720FDF7F1B921989A
:20E9A00090F847606FEA060380F84730FDF7E8B90DF1700CFAF77EFE1E9D41F22C17C2F276
:20E9C00000077A5D1D9951407955FDF7D9B92198866B1D9B9A191C92A1E12199C86B8E6B93
:20E9E00083191C939BE121990A6C42B941F2A824C2F200044FF02000207101F06FBF02F16C
:20EA0000FF350D64FDF7BCB9219E336C03F101033364002B7DF4B4A941F2A821C2F2000151
:20EA20004FF020020A7101F059BF2198466B3368596841B941F2A820C2F200004FF01E0322
:20EA4000037101F04BBF0DF1700CFAF70BFE1C90219850F8342F166876681D991CAA4FF0AC
:20EA60000103B0478DF86B0000283DF489A941F2A824C2F20004207101F030BF0DF1700C7E
:20EA8000FAF7F0FD1C9038E10DF1700CFAF7EAFD219FF863FDF774B90DF1700CFAF7E2FDFB
:20EAA000219D2864FDF76CB9219850F8341F0A6816681D991CAA4FF00103B0478DF86B0009
:20EAC00030B141F2A824C2F20004207101F006BF0DF1A80C1CF8380DFAF7ACFDFDF750B9B5
:20EAE0002198436B0DF1700C187AFAF7A3FDFDF747B90DF1700C219F97F83C00FAF79AFD91
:20EB0000FDF73EB921990A6CFF2A08D941F2A826C2F200064FF02004347101F0DFBE0DF181
:20EB2000700CD0B2FAF786FDFDF72AB9219850F8345F2B689F68B84703EE100AF8EE433AF1
:20EB40002198C0ED133AFDF71BB9219991ED0E4AF8EE444AC1ED134AFDF712B9219A92ED32
:20EB6000105AF8EE455AC2ED135AFDF709B9219E96ED136AFCEEC66ACDED1C6ACFE0219B50
:20EB8000D3ED137A9FEDC17AF4EEC77AF1EE10FA08DB41F2A824C2F200044FF020002071CB
:20EBA00001F09CBEBCEEE70A83ED100AFDF7E8B8219850F8341F0A6816681D991CAA4FF052
:20EBC0000403B0478DF86B0030B141F2A823C2F20003187101F082BE1C98FAF7A5FB219DF4
:20EBE000A864FDF7CDB8219850F8341F0A6816681D991CAA4FF00403B0478DF86B0030B1C2
:20EC000041F2A824C2F20004207101F067BE1C98FAF78AFB219FF864FDF7B2B82198436B8B
:20EC200019684A6842B941F2A820C2F200004FF01E01017101F052BEC06CFAF74BFB1C9017
:20EC4000219850F8346F33685E681D991CAA4FF00403B0478DF86B0000283DF491A841F241
:20EC6000A824C2F20004207101F038BE1D9A2198C36BC3F1FB06B24208D941F2A824C2F2BD
:20EC800000044FF01300207101F028BE50F8347F39680E684FF0000141F22C17C2F2000733
:20ECA000BA18B0478DF86B0000283DF469A841F2A823C2F20003187101F010BE219850F833
:20ECC000342F11680E681D991BAA4FF00403B0478DF86B0030B141F2A824C2F20004207111
:20ECE00001F0FCBD1B9B98B2C3F3072242EA00218EB21C9613E01D9B1C931C982199FAF793
:20ED00004FFD8DF86B0000283DF43AA841F2A822C2F20002107101F0E1BD1D981C901C9E9E
:20ED2000B6F5803F08D341F2A824C2F200044FF01F03237101F0D2BD219DAE63FDF720B8C7
:20ED40001D9D219FFD63FDF71BB81D99219E3164FDF716B8219B9A6B1D98111A1C91DEE733
:20ED60001E9A219BD96B8818FB2808D941F2A823C2F200034FF012021A7101F0AFBD41F214
:20ED8000DC27C2F2000787F8FB10184650F8346F31680E681D99BA18DB6BB0478DF86B001E
:20EDA00000283CF4EDAF41F2A824C2F20004207101F094BD2198416B0E68766846B941F2EA
:20EDC000A826C2F200064FF01E02327101F086BD1D9AC36BC3F1FB018A4208D941F2A82038
:20EDE000C2F200004FF01303037101F077BD00F134004FF0000141F22C17C2F20007BA1809
:20EE0000B0478DF86B0000283CF4BAAF41F2A824C2F20004207101F061BDF7F791FA002852
:20EE20007CF4AEAF1D991C91FEF7A6BEF7F788FA00283CF4A5AF1D981C90FEF79DBE1D9BC4
:20EE40000F2B08D941F2A824C2F200044FF00506267101F043BDD8B24FF00001F7F72EFA2E
:20EE600000EE900AB8EE601A219F87ED131AFCF787BF1D9A0F2A0BD941F2A821C2F20001CB
:20EE80004FF00500087101F029BD00BF00008047D0B24FF00101F7F711FA01EE900AB8EE6D
:20EEA000612A219D85ED132AFCF76ABF1D9B0F2B08D941F2A824C2F200044FF005062671D3
:20EEC00001F00CBDD8B24FF00001F7F767F9FCF757BF1D9A0F2A08D941F2A821C2F20001D5
:20EEE0004FF00500087101F0F9BCD0B24FF00101F7F754F9FCF744BF1D9B0F2B08D941F2B5
:20EF0000A824C2F200044FF00506267101F0E6BCD8B24FF00001F7F791F9FCF731BF1D9A1D
:20EF20000F2A08D941F2A821C2F200014FF00500087101F0D3BCD0B24FF00101F7F77EF9A1
:20EF4000FCF71EBF9DF87400F2F7FAFF00287CF417AF41F2A823C2F200034FF028041C71EB
:20EF600001F0BCBC9DF87400219901F14C01F3F707F800287CF404AF41F2A826C2F2000637
:20EF80004FF02802327101F0A9BC2199D1ED132A9DF87400BCEEE23A13EE101AF3F722F85C
:20EFA00000287CF4EDAE41F2A820C2F200004FF02803037101F092BCFCF7E2BE0DF1700C45
:20EFC000FAF750FB30B9219F97F847502E1C18BF012601E04FF00106219A82F84760FCF7E8
:20EFE000CFBE9DF874600DF1700CFAF73BFB014630464FF00102FBF7D7FE8DF86B0000289C
:20F000003CF4BEAE41F2A824C2F20004207101F065BC0DF1700CFAF725FB01468DF86A0039
:20F020009DF87400FBF77EFE8DF86B0000283CF4A7AE41F2A821C2F20001087101F04EBC97
:20F040001D981C904FF001038DF86A301E46219A92F847100B420AD092F846109DF87000E1
:20F0600019403246FBF7A0FE8DF86B0068B99DF86A304FEA43008DF86A001C9A02F10102D8
:20F080001C9210F0FE03E2D10AE09DF86A60012E06D141F2A824C2F20004207101F01EBCAC
:20F0A0004FF000078DF86B700DF1700CFAF7DAFA0DF1700CFAF7D6FAFCF762BE9DF8740014
:20F0C0004FF001010A46FBF76FFE8DF86B0000283CF456AE41F2A821C2F20001087101F0D9
:20F0E000FDBB9DF874004FF000014FF00102FBF75BFE8DF86B0000283CF442AE41F2A8224D
:20F10000C2F20002107101F0E9BB0DF1700CFAF7A9FA219D95F84730184385F84700FCF741
:20F120002FBE1D980DF1A80C4CF8380DFAF748FF00287CF425AE41F2DC30C2F20000099EB5
:20F14000066001F04EBB10A8FAF7CCFD014640B19DF84070022F04D0D1484FF00D0207F0FD
:20F16000A5FC0DF1700C9DF84000FAF763FAFCF707BEFBF779FAFCF703BE0DF1700CFAF715
:20F1800071FAFCF7FDBD1D9EFA2E08D941F2A824C2F200044FF01202227101F09FBB0DF1AD
:20F1A000700CFAF75FFA41F2DC21C2F200018855FCF7E6BD0DF1700CFAF754FA41F2DC2544
:20F1C000C2F2000585F8FB00FCF7DABD0DF1700C219B93F84700FAF72DFAFCF7D1BD1D981E
:20F1E000FA2808D941F2A826C2F200064FF01201317101F073BB0DF1700C41F2DC27C2F2DA
:20F200000007385CFAF716FAFCF7BABD0DF1700C41F2DC22C2F2000292F8FB00FAF70AFA0D
:20F22000FCF7AEBD1D9EF62E08D941F2A824C2F200044FF01200207101F050BB219DA86C49
:20F24000FAF748F841F2DC23C2F200039851FCF797BD1D99FA2908D941F2A826C2F20006EF
:20F260004FF01302327101F039BB0DF1700C41F22C17C2F20007785CFAF7DCF9FCF780BD3D
:20F280000DF1700CFAF716FA41F22C15C2F200051E9BE85C1D9908420DF1700C0CBF002064
:20F2A000FF20FAF7C7F9FCF76BBD1D9EF92E08D941F2A820C2F200004FF01301017101F03B
:20F2C0000DBB41F22C12C2F20002905D9319597841EA00261C96002E3CF452ADFEF74CBC78
:20F2E0001D9BFA2B08D941F2A824C2F200044FF01300207101F0F2BA41F22C16C2F20006EA
:20F30000F25C002A43D1FCF73BBD1D99FA2908D941F2A824C2F200044FF01302227101F02D
:20F32000DDBA41F22C13C2F200035E5C7EB3FCF727BD0DF1700CFAF795F91C9038BBFCF7C0
:20F340001FBD0DF1700CFAF7B5F941F22C10C2F200001E99465C1D9B1E4218D0FCF710BD7C
:20F360000DF1700CFAF7A6F941F22C12C2F200021E98115C1D9E314209D1FCF701BD0DF182
:20F38000700CFAF76FF91C9000287CF4F9AC219E326A42B941F2A824C2F200044FF0030060
:20F3A000207101F09BBA02F1FF35356202F1010256F8227041F2DC31C2F200010F60FCF78B
:20F3C000DFBC219D95F847704FEAD71343EA470285F84720FCF7D4BC219890F847604FEA6F
:20F3E000560141EAC61580F84750FCF7C9BCFAF74BFDFCF7C5BC41F22417C2F20007FB78E0
:20F400004FF0010000FA03F03A7922EA00023A71FCF7B6BC41F2A824C2F200044FF00106F1
:20F42000267101F05BBA41F22411C2F20001CD7845B941F22410C2F200004FF00602C2703B
:20F44000FCF79EBC05F1FF3741F22413C2F20003DF70FCF795BC41F22416C2F200063178AF
:20F4600001F1FF35EFB237703379FF2B0BD1632F7CF686AC41F22416C2F200064FF063016C
:20F480003170FCF77DBC172F7CF67AAC41F22410C2F200004FF017020270FCF771BC00BFFD
:20F4A0003211002041F22415C2F200056F7807F1FF33D8B268702A79FF2A0BD100287CF411
:20F4C0005FAC41F22415C2F200054FF00C076F70FCF756BC3B287CF653AC41F22416C2F2D1
:20F4E00000064FF03B017170FCF74ABC41F2A824C2F200044FF00103237101F0EFB941F257
:20F50000A820C2F200004FF00102027101F0E6B941F2A826C2F200064FF00101317101F09B
:20F52000DDB941F2A824C2F200044FF00103237101F0D4B941F22415C2F20005EF78052F69
:20F5400008D941F22416C2F200064FF00002F270FCF716BC07F1010741F22410C2F2000020
:20F56000C770FCF70DBC41F22411C2F200010B7803F10103DDB20D700F79FF2F0BD1632DD2
:20F580007CF6FEAB41F22411C2F200014FF000020A70FCF7F5BB172D7CF6F2AB41F224101B
:20F5A000C2F200004FF000060670FCF7E9BB41F22415C2F200056B7803F10103DFB26F70D5
:20F5C0002879FF280BD10C2F7CF6DAAB41F22415C2F200054FF001026A70FCF7D1BB3B2F2B
:20F5E0007CF6CEAB41F22416C2F200064FF000017170FCF7C5BB41F2A824C2F200044FF06F
:20F600000103237101F06AB941F22417C2F20007F8784FF0010606FA00F6397986EA010541
:20F620003D71FCF7ADBB0DF1700CFAF71BF841F22412C2F200021071FCF7A2BB0DF1700CD9
:20F64000FAF710F8062841F22413C2F2000392BFD8700027DF70FCF793BB0DF1700CFAF7A7
:20F6600001F841F22416C2F200063070FCF788BB0DF1700CF9F7F6FF41F22411C2F2000118
:20F680004870FCF77DBB0DF1700CF9F7EBFF41F22415C2F20005A870FCF772BB0DF1700C5C
:20F6A00041F22410C2F200000079F9F7C3FFFCF767BB0DF1700C41F22412C2F20002D0780E
:20F6C000F9F7B8FFFCF75CBB0DF1700C41F22413C2F200031878F9F7ADFFFCF751BB0DF1B5
:20F6E000700C41F22417C2F200077878F9F7A2FFFCF746BB0DF1700C41F22416C2F200064F
:20F70000B078F9F797FFFCF73BBB41F2A824C2F200044FF00101217101F0E0B81D9A0F2A4F
:20F7200008D941F2A824C2F200044FF02700207101F0D4B8C24D05EB820041F22413C2F21E
:20F74000000315F822701F7046785E704FF000019970D97082781A71FCF712BB41F2A82317
:20F76000C2F200034FF001061E7101F0B7B841F22415C2F20005EF784FF0010101FA07F1DD
:20F780002A7941EA02002871FCF7FABA41F2A824C2F200044FF00103237101F09FB841F250
:20F7A000A826C2F200064FF00101317101F096B84FF00005139512951195199541F224174A
:20F7C000C2F200073A7802F164021692787800F1FF331593BE78149611A806F08DFF179935
:20F7E00019B101F1FF37FDB201E04FF0060541F22412C2F20002D570FCF7C2BA1D9E0F2E72
:20F8000008D941F2A824C2F200044FF02706267101F064B88A4800EB860141F22413C2F2DE
:20F8200000031D7800F826505F784F701A798A70FCF7A6BA41F2A820C2F200004FF001015C
:20F84000017101F04BB80DF1700C219B93F85000F9F7F0FEFCF794BA41F27022C2F2000297
:20F86000147814F0010F08D141F2A824C2F200044FF03002227101F031B841F28C26C2F2E1
:20F880000006306840B941F2A821C2F200014FF031030B7101F022B841F27021C2F20001ED
:20F8A0000B7803F0FE0242F004040C7041F29026C2F200064FF00000306000F07BBF41F24D
:20F8C0007026C2F20006307810F0010F08D141F2A826C2F200064FF03000307100F0FEBFCF
:20F8E00041F28C21C2F200010B6843B941F2A824C2F200044FF03402227100F0EFBF41F274
:20F900007024C2F20004227802F0FE0646F00200207041F29021C2F200014FF000030B60FD
:20F9200000F048BF219D95F846700DF1700CF9F799FE21993B1A91F8502002F00106981B1A
:20F940001C9081F84700FF2894BF0020012081F85000FCF715BA1D9BFA2B08D941F2A82438
:20F96000C2F200044FF01301217100F0B7BF41F22C15C2F200051E9FEF54FCF701BA4FF06A
:20F9800000021C921AE04FF001061C9616E04FF002001C9012E04FF003031C930EE04FF0CF
:20F9A00004051C950AE04FF005071C9706E04FF006011C9102E04FF007021C921D991B9192
:20F9C0001C98FAF775FAFCF7DBB90DF1700CF9F771FE1E9E41F22C13C2F20003985D1D9D1F
:20F9E00005439D55FCF7CCB91D9EF92E08D941F2A824C2F200044FF01202227100F06EBFD8
:20FA000041F2DC27C2F200071E99B955FCF7B8B941F2DC20C2F200001D9B80F8FB30FCF79B
:20FA2000AFB941F27846C2F20006316851B941F2A820C2F200004FF00106067100F04EBFA7
:20FA4000442500104E681D981E994FF001020DF16A03B0478DF86B009DF86A20D2F1010193
:20FA600038BF0021219B83F8501000283CF488A941F2A824C2F20004207100F02FBF41F2F5
:20FA80007842C2F20002116841B941F2A820C2F200004FF00106067100F020BF0B681D9820
:20FAA0001E9998478DF86B0000283CF469A941F2A824C2F20004207100F010BF41F2784262
:20FAC000C2F20002116841B941F2A820C2F200004FF00106067100F001BF4E681D981E99BF
:20FAE0004FF000020DF16A03B0478DF86B009DF86A30D3F1010238BF0022219981F85020C1
:20FB000000283CF43DA941F2A824C2F20004207100F0E4BE0A981E99F9F7C4FF0A9040B92E
:20FB200041F2A826C2F200064FF01702327100F0D5BE0A9B1A68966A46B941F2A820C2F2B7
:20FB400000004FF01503037100F0C8BE0A9988689DF8741041F2DC22C2F20002B0478DF855
:20FB60006B0000283CF40CA941F2A824C2F20004207100F0B3BE0A981E99F9F793FF0A90EF
:20FB800040B941F2A820C2F200004FF01703037100F0A4BE0A990868436943B941F2A821E7
:20FBA000C2F200014FF015020A7100F097BE0A9EB0689DF8741041F2DC22C2F200029847DB
:20FBC0008DF86B0000283CF4DBA841F2A824C2F20004207100F082BE0A981E99F9F762FF38
:20FBE0000A9040B941F2A821C2F200014FF017060E7100F073BE0A9E31688E6946B941F25B
:20FC0000A820C2F200004FF01503037100F066BE0A9A90689DF8741041F2DC22C2F20002ED
:20FC20000DF16A03B0478DF86B0000283CF4A8A841F2A824C2F20004207100F04FBE0A98E3
:20FC40001E99F9F72FFF0A901D997F2909D1051C18BF012541F2DC27C2F200073D70FCF74E
:20FC60008FB80A9A42B941F2A823C2F200034FF017061E7100F032BE0A9803685E6846B94C
:20FC800041F2A821C2F200014FF01500087100F025BE0A9A9068C9B241F2DC22C2F2000215
:20FCA000B0478DF86B0000283CF46AA841F2A824C2F20004207100F011BE0A981E99F9F7A3
:20FCC000F1FE0A9040B941F2A826C2F200064FF01700307100F002BE0A9A11688F6847B92C
:20FCE00041F2A821C2F200014FF015020A7100F0F5BD41F2DC26C2F200060A9880689DF8D2
:20FD0000741032780DF16A03B8478DF86B009DF86A30337000283CF433A841F2A824C2F2A3
:20FD20000004207100F0DABD0A981E99F9F7BAFE0A9040B941F2A826C2F200064FF0170101
:20FD4000317100F0CBBD0A9F3B68DF6847B941F2A820C2F200004FF01503037100F0BEBD11
:20FD600041F2DC26C2F200060A9988689DF8741032460DF16A03B8478DF86B009DF86A20F7
:20FD8000327000283BF4FCAF41F2A824C2F20004207100F0A3BD0A981E99F9F783FE0A90C3
:20FDA00040B941F2A820C2F200004FF01706067100F094BD0A9F3A68176947B941F2A821C0
:20FDC000C2F200014FF015020A7100F087BD0A98D0F808809DF8749041F2DC26C2F20006EF
:20FDE0003068F9F7A1FA0246404649460DF16A03B8478DF86B009DF86A30337000283BF400
:20FE0000BFAF41F2A824C2F20004207100F066BD0A984FF00001F9F745FE0A9040B941F23E
:20FE2000A821C2F200014FF017060E7100F056BD0A9B1968CE6A46B941F2A820C2F200005A
:20FE40004FF01503037100F049BD0A9A90689DF87410B0478DF86B0000283BF491AF41F27B
:20FE6000A824C2F20004207100F038BD0A981E99F9F718FE0A9040B941F2A820C2F20000E7
:20FE80004FF01703037100F029BD0A9A1068C36943B941F2A826C2F200064FF015023271C7
:20FEA00000F01CBD0A9988689DF8741041F2DC22C2F2000298478DF86B0000283BF460AFB1
:20FEC00041F2A824C2F20004207100F007BD0A981E99F9F7E7FD0A9040B941F2A826C2F2B1
:20FEE00000064FF01703337100F0F8BC0A990E68336A43B941F2A820C2F200004FF01501A5
:20FF0000017100F0EBBC0A9A90689DF8741041F2DC22C2F2000298478DF86B0000283BF416
:20FF20002FAF41F2A824C2F20004207100F0D6BC0A981E99F9F7B6FD0A9040B941F2A8218E
:20FF4000C2F200014FF017030B7100F0C7BC0A9A1068466A46B941F2A826C2F200064FF0DF
:20FF60001502327100F0BABC0A9988689DF8741010AAB0478DF86B001098F9F7ABF941F2A5
:20FF8000DC23C2F2000318609DF86B0000283BF4F7AE41F2A824C2F20004207100F09EBCA5
:20FFA0000A984FF00001F9F77DFD0A9040B941F2A826C2F200064FF01703337100F08EBC70
:20FFC0000A980668336B43B941F2A821C2F200014FF01500087100F081BC0A9A90689DF89B
:20FFE000741041F2DC22C2F2000298478DF86B0000283BF4C5AE41F2A824C2F200042071B5
:020000040803EF
:2000000000F06CBC1D99072908D941F2A824C2F200044FF00800207100F060BC40F2A0652F
:20002000C1F2000505EBC107D7F81029002A7BF4A7AEF7F71DFE002808BF012040F2A06609
:20004000C1F200061D9B06EBC301C1F81009FBF797BE1D9E072E08D941F2A824C2F20004D9
:200060004FF00800207100F039BC40F2A065C1F2000505EBC607D7F81029002A3BF480AE88
:20008000F7F7F6FD1D9B40F2A061C1F2000101EBC306D6F81059401B1C90D6F81479B84298
:2000A0008CBF0027C0EB07071B9740F2A062C1F2000202EBC3031B99C3F814194FF00006E6
:2000C000C3F81069FBF75CBE1D9EFA2E07D941F2A823C2F200034FF013021A71FEE30DF1AA
:2000E000700CF9F7BFFA41F22C15C2F20005A855FBF746BE0DF1700CF9F7DCFA0DF1700C01
:20010000F9F7B0FA1C9050B11E9B41F22C12C2F20002D75C1D9E3E43D654FBF731BE1E9F81
:2001200041F22C16C2F20006F05D1D9920EA0105F555FBF725BE1D9B1E9AD018C1B241F260
:20014000DC26C2F2000686F8FB10FA2907D941F2A824C2F200044FF012002071BEE341F2EA
:20016000DC35C2F200052F6841F2DC20C2F20000C01840F20003C0F60103F91806F096FCDB
:200180002A681E9956182E60FBF7FABD1D9BF82B07D941F2A824C2F200044FF01306267110
:2001A0009CE3F7F765FD00F104004CF6CD45CCF6CC45A5FB00174FEA9701219A566AB1FBA5
:2001C000F6F31C931D9D41F22C17C2F200074FEA134078557A194FEA132151709370FBF78D
:2001E000CFBD1D9BF82B07D941F2A824C2F200044FF01302227171E3F7F73AFD00F10400AC
:200200004CF6CD45CCF6CC45A5FB00274FEA9700219A516AB0FBF1F61D9B41F22C17C2F236
:200220000007F8184578FA5C4FEA024141EA0527837847EA03001B90361A26F07F451C950C
:200240000DF1700C1E9885422CBF00200120F9F7F1F9FBF795BD219991F846700DF1700CEA
:20026000F9F700FA381A1C90219B83F84700FF2894BF0020012083F85000FBF781BD1D9EA7
:20028000F92E07D941F2A823C2F200034FF013061E7123E341F2DC32C2F20002126841F211
:2002A0002C11C2F200014FEA122088558B195A70FFF76DB8219D95F847201C9295F84670D8
:2002C00085F8477085F84620FBF75ABD1D98072807D941F2A821C2F200014FF008040C71C1
:2002E000FCE2F9F713FE0DF1A80C4CF8380D003018BF0120F9F79EF9FBF742BD219B93F8FD
:20030000470093F846600DF1700CB04214BF00200120F9F78FF9FBF733BD219D95F84700F9
:2003200095F846200DF1700C801A18BF0120F9F781F9FBF725BD219F97F8470097F8461005
:200340000DF1700C88422CBF00200120F9F772F9FBF716BD219B93F8470093F846600DF150
:20036000700CB04294BF00200120F9F763F9FBF707BD219D95F8470095F846200DF1700C7A
:2003800090428CBF00200120F9F754F9FBF7F8BC219F97F8470097F846100DF1700C88425D
:2003A00034BF00200120F9F745F9FBF7E9BC1D98F62807D941F2A824C2F200044FF0120287
:2003C00022718BE241F2DC23C2F200031858F8F7ABFF219EF064FBF7D3BC1D99F62907D9E2
:2003E00041F2A820C2F200004FF01203037175E241F2DC25C2F200056858F8F795FF219F3F
:20040000B864FBF7BDBC41F2DC26C2F2000696F8FB201D9BD118FB2907D941F2A823C2F266
:2004200000034FF01201197158E21E9EC2F1FB00864207DD41F2A824C2F200044FF0130282
:2004400022714BE241F22C15C2F20005A81941F2DC27C2F20007F91806F028FBFBF790BC95
:200460002198466B326856683EB941F2A823C2F200034FF01E021A7130E21E9A41F2DC2328
:20048000C2F2000393F8FB309918FB2907D941F2A820C2F200004FF0120606711EE200F1CC
:2004A00034001D9941F2DC27C2F20007BA18B0478DF86B0000283BF463AC41F2A824C2F28F
:2004C000000420710AE241F2A821C2F200014FF001040C7102E20DF1700CF9F7EBF841F2C5
:2004E0002C15C2F200051E9FE85D1D9E30423BF447AC41F2DC33C2F20003099A1A6070E14A
:200500000DF1700CF9F7D6F841F22C11C2F200011E9D4F5D1D9807427BF432AC41F2DC3489
:20052000C2F20004099E26605BE19DF874000DF16B01FAF723FB8DF86A009DF86B302BB11D
:2005400041F2A820C2F200000371C7E100283BF417AC41F2DC32C2F200020999116040E18B
:200560009DF874000DF16B01FAF708FBD0F1010638BF00268DF86A609DF86B0028B141F2D4
:20058000A822C2F200021071A8E1219DEF6A17B98DF86A7002E09DF86A2062B90DF1700CF5
:2005A0001E98F9F70DFD30B941F2DC34C2F200040999216015E10DF1700C9DF86A00F9F725
:2005C00039F84FF00006219BDE62FBF7D9BB9DF874000DF16B01FAF7D1FA8DF86A009DF870
:2005E0006B302BB141F2A824C2F20004237175E100287BF4C5AB41F2DC35C2F20005099F37
:200600002F60EEE09DF874000DF16B01FAF7E8FA8DF86A009DF86B1029B141F2A826C2F2A9
:20062000000631715AE100287BF4AAAB41F2DC30C2F20000099A0260D3E09DF874000DF139
:200640006B01FAF7CDFA031C18BF01238DF86A3092E79DF874000DF16B01FAF78FFA011CBA
:2006600018BF01218DF86A1086E71D9EF62E07D941F2A823C2F200034FF012041C712DE1B1
:200680002198C06CF8F726FE41F2DC25C2F20005A851FBF775BB0DF1700CF8F7E3FF219F4F
:2006A00097F84710D1F1010238BF0022002814BF164682F0010687F84760FBF761BB0DF174
:2006C000700CF8F7CFFF219D95F84730584085F84700FBF755BB0DF1700CF8F7C3FF219FD6
:2006E00087F85100FBF74CBB04F058FD0DF1A80C4CF8380DFF2828BFFF20C0B2F8F79AFF86
:20070000FBF73EBB04F040FD0DF1A80C4CF8380DFF2828BFFF20C0B2F8F78CFFFBF730BB8C
:2007200004F046FD0DF1A80C4CF8380DFF2828BFFF20C0B2F8F77EFFFBF722BB04F01AFD62
:200740000DF1700C00280CBFFF200020F8F772FFFBF716BB41F2D830C2F2000001681D9ABB
:20076000881804F069F88DF86B0000283BF408AB41F2A824C2F200042071AFE01D9804F00A
:2007800019F8FBF7FDBA0DF1700CF8F76BFF04F00BF8FBF7F5BA41F2D836C2F2000635689C
:2007A0001D9BE81804F022F8FBF7EABA04F006F8FBF7E6BA41F28C20C2F20000016881B923
:2007C00041F27022C2F20002147804F00206F3B23BB141F2A824C2F200044FF035032371C3
:2007E0007CE041F27027C2F200073D7815F0010F7BF4C4AA219828B141F2DC31C2F20001EA
:200800000A68426041F29024C2F2000426683F2E00F2918006F101061B961C9616B94FF0B8
:2008200001071B97634E4FF0540541F27024C2F2000441F28C27C2F200071C9B05FB03607B
:2008400021909BB9217801F00402D1B209B93A6842B9217841F001026FF382022270426832
:2008600042B115E04FF001001C90E6E742687AB9402B02D003F1010301E04FF000031C93F3
:200880001B988342D9D14FF00000F9F7D9FED4E741F29026C2F20006336041F2DC35C2F247
:2008A00000052A604FF0000A5446FBF769BA219F396A41F000423A63FBF762BA4FF00006EB
:2008C000219D2E63FBF75CBAFBF75ABA0C9D41F2A820C2F200004FF00104047141F2A822AD
:2008E000C2F20002099E16605571F1F72DFEF1F72BFE219D286A78B14FF000041C94219B13
:20090000196A49B1F1F720FE1C9E06F101061C96219A156AB542F5D84FF00000F9F790FE2F
:20092000FBF765B94FF0000706F1FF344FF000005E46FDF711BD4FF000031C936FE74FF00C
:2009400002031C931B4EFDF751BF2BB0BDEC0A8BBDE8F08F01F10103D6F80051002D3DF4C6
:2009600049AF01F1020306F1A806412B7DF43EAFFDF79ABFBEF1000F3DF488AC10F803900E
:2009800001F8039003F1010393427DF47FACFDF78BBCF9180EEB030C13F8016F02F1FF356C
:2009A000B0423DF452AA2A46FDF75EBA05F1FF32FDF75ABAF00F00102DE9F04F2DED028B62
:2009C0008FB04FF0000841F27427C2F2000741F26823C2F20003039341F2882BC2F2000B58
:2009E00040F2A066C1F200069FEDB98B39684FF0FF3041B9F1F7A8FD386800280CBFFA20F3
:200A00004FF0FF30FFE7F6F7B9FC28B1B8F1320F09D808F1010806E0B8F1330F0CBF4FF05F
:200A200034084FF000083A68D2B9F1F78DFDB8F1320F0ED1039C2068F6F74CFD4FF000052A
:200A4000039B1D60F5F722FF4FF00200F9F736FD06E0B8F1340F03D14FF00100F9F72EFD09
:200A60009BF800104FF4117000FB0162D2F81842002CBBD04FF4117505FB01F303F5887425
:200A800006EB0409315DE0290CD199F801000E2808D14FF6FF704946D9F80021F8F7B4FB70
:200AA00010B36BE2325D02F01F0509EB05035A78294605F0010019F80550521B01F1FF3357
:200AC000002940F078820BE019F80300151A03F1FF3119F80120AA1A01F1FF330029F3D16A
:200AE00012F0FF0F40F04A82335D4FEA5310072800F23C82DFE810F008003A023A02350063
:200B0000A6003A028A002601335D09F1010513F01F0000F0338209F1020905F1020500F1F8
:200B2000FF3255FA82F402944FF000054FF0010A15E019F8011CE8B221405246FAF734F9C7
:200B4000002840F01B8205F101054FEA4404FF2CEFD909F101090299894500F00F825446A8
:200B6000E7E799F80140386870B1F6F7B3FC4FF000003860F5F78AFEFAF7DEFE4FF0010020
:200B8000F9F79CFCF1F7E0FC03990B686BB94BF24430C0F603004FF007014BF2B912C0F667
:200BA0000202F6F7ADFB039D286005A84FF00001F9F7B2FE7CB9F7F75BF8C1B201F1FF33DA
:200BC000DDB2FD2D41F27820C2F2000092BF01700122027009E041F27820C2F200000278A4
:200BE00002FB04F404EB1424047041F27824C2F2000421780EAB03F8241D4FF003004FF0CF
:200C000000014FF01602F9F77DFCEFE60DF11300F9F768F801469DF813508DF81450012D87
:200C200006D828B10DF115004FF00D0205F03EFF4FF006004FF000014FF00E0205ABF9F7F6
:200C400061FCD3E69BF800104FF4117303FB01F499F80100032872D8DFE800F002263E50AD
:200C60004FF00100FAF7F2FE4FF000050EAB03F8255D4FF0040029464FF00102F9F742FCB7
:200C80004FF0C800F8F7A8FA32599BF800004FF0010400940195D2F80CC04FF416512A4680
:200CA0004FF00803E04766E14FF0000141F2A823C2F2000319714FF001040EAB03F8254D93
:200CC0004FF004002246F9F71DFC54E1AFF300800000000000E06F40F9F7C6FC0EAB4FF0D0
:200CE000020103F8251D4FF004004FF000014FF00102F9F707FC4FF001043CE10EAB4FF0A3
:200D0000120203F8252D4FF004004FF000014FF00102F9F7F7FB4FF0C800F8F75DFA3559F0
:200D20009BF800004FF0010400944FF000020192ED684FF416414FF00803A8471BE14FF011
:200D4000000418E199F80150A5F102050C2D00F21081DFE815F00D0067007E000E010E017F
:200D60000E010E010E010E010E010E010E019D00315DC1F30403DAB2012A00F0FF8009F104
:200D8000050509F1080403EBC30003EB400101EBC10303F15403DAB202EB42002418C5EBC1
:200DA000040CACF1030E0EF0010A99F8029015F8010C04F017FB53EC182B04F025FE04F09C
:200DC000EBFB01464846FAF75FF805F10305A54240F0D780D2E015F8039C15F8010C04F038
:200DE00001FB53EC182B04F00FFE04F0D5FB01464846FAF749F805F1030515F803AC15F8E2
:200E0000010C04F0EFFA53EC182B04F0FDFD04F0C3FB01465046FAF737F805F10305A542E4
:200E2000D9D1ABE099F80230305DC0F30405A5F10305EAB209F103019C18FF2CC4BF5A423B
:200E4000D2B241F22C10C2F20000C01805F02EFE94E099F8023099F803500EAC04F8243DC0
:200E60000DF1150041F22C11C2F20001C918202D34BF2A46202205F019FE05F101024FF023
:200E800007004FF00301D2B22346F9F73BFBADE599F80240C4B999F80310A9B903F0FAFC24
:200EA000039A1068F6F716FB4FF0000303980360F5F7ECFC4BF25430C0F6030007F0E8FBB7
:200EC000F9F7B2FC002848D099F8025099F803404BF26430C0F6030044EA052107F0D8FBD5
:200EE00099F803A0494611F8022F40F20003C0F6010303EB022541F22C14C2F2000404EBD7
:200F00000A0001F102014FF0800205F0CFFD4FF68071CFF6FF71CAEB0100C2B2A018A91842
:200F20004FF0800205F0C2FD204629464FF48072F2F7C0FAA0B9204629464FF4807205F037
:200F40005FF980B94FF001004FF000010A460B46F9F7D8FA4FF001040DE04FF000040AE0BF
:200F60004FF0000407E04FF0000404E04FF0000401E04FF00004002C7FF438ADF8F794FEB4
:200F800034E5BAF1000F3FF426AF15F803AC15F8010C04F027FA53EC182B04F035FD04F0EF
:200FA000FBFA01465046F9F76FFF05F10305A5427FF411AFE2E700283FF486AD19F803106E
:200FC000521A03F1FF33B3F1FF3F7FF47DAD87E52DE9F84341F20843C2F2000318784FEA45
:200FE000400111F0FF0405D041F20842C2F20002147006E041F20845C2F200054FF00106BB
:201000002E7041F22C47C2F20007387841F20843C2F20003197808420CBF4FF000094FF0BF
:2010200001094FF000052C464FF0010741F20C46C2F20006A84604F01F0207FA02F0AB5970
:20104000184204D0204649464246F9F7ADFE04F10104E4B214F01F0FEDD105F10405202D7E
:20106000E9D1BDE8F88300BF41F22C43C2F20003187041F20840C2F200004FF00102027013
:20108000704700BF00B583B041F20C40C2F200004FF000014FF00802F0F754F84FF00003C1
:2010A00000934FF00100019041F23040C2F200004FF47A714FF0060240F6D173C0F60303CA
:2010C000F6F7A0FD03B000BD08B541F23040C2F20000F6F7F1FC4FF0CC00FFF7C5FF08BD9E
:2010E00089B14FEA501241F20C43C2F2000300F01F004FF0010101FA00F053F822100843DF
:2011000043F8220011E04FEA501241F20C43C2F2000300F01F004FF0010101FA00F053F827
:20112000221021EA000143F822104FF00000704708B54FF440404BF28441C0F6030141F29F
:201140005442C2F20002F9F747FC08BD10B584B0144649BB0DF10D0300930DF10E000190B6
:201160004FF0000001460DF10A020DF10B03F5F739FA4FF000018DF80C109DF80B201AB148
:201180004FF001038DF80C309DF80A0028B19DF80C1041F002028DF80C204FF000008DF878
:2011A0000F00039B236001E04FF0140004B010BD70B514468AB199B94FF000000146024670
:2011C000F5F788FA06462578F5F768FB85420AD2735D23704FF0000070BD4FF0160070BD75
:2011E0004FF0140070BD4FF0160070BD70B5154691B992F8FB3093B14FF000042646285DF6
:201200003146F5F761F904F1010495F8FB00A042F5D84FF0000070BD4FF0140070BD4FF0B5
:20122000000070BD10B586B0F1B941F26043C2F20003197841F26140C2F20000037802AC0D
:2012400000944FF01000019010461A464FF00103FAF73AF94BF28040C0F60300214607F0E9
:2012600017FA4FF0000001E04FF0140006B010BD2DE9F0411546042975D8DFE801F0030B85
:20128000741B640068782978F5F714FA4FF00000BDE8F0812A7841F26043C2F200031A70D2
:2012A000687841F26141C2F2000108704FF00000BDE8F0812C786D7805F1040546F267636D
:2012C000C6F2666383FB05204FEA600101EB810212F0FF054BD04FF00007A5F1050808F0DF
:2012E0000108042C94BF2646052630463946F5F7EBF8A41BE4B2A5F1050515F0FF053ED1FA
:201300001DE0042C94BF2646052630463946F5F7DBF8A01BA5F1050505F0FF0500F0FF04BB
:20132000042C94BF2646052630463946F5F7CCF8A11BCCB2A5F1050515F0FF05E1D14FF01A
:201340000000BDE8F0812C78F5F7A8FA844212D2204605F101014FF00102F5F7D7F94FF000
:201360000000BDE8F0814FF01400BDE8F0814FF00000BDE8F0814FF01600BDE8F0814FFAE5
:2013800088F6002EBDD0042C94BF2646052630463946F5F799F8A31BDCB2A5F1050515F097
:2013A000FF05AED1CBE700BF08B505293ED8DFE801F0030B151F29331046F5F743F900283C
:2013C0000CBF1620002008BD4BF24030C0F60300114607F05DF94FF0000008BD4BF2383074
:2013E000C0F60300114607F053F94FF0000008BD4BF23430C0F60300114607F049F94FF06D
:20140000000008BD4BF22C30C0F60300114607F03FF94FF0000008BD4BF22430C0F60300E1
:20142000114607F035F94FF0000008BD4FF0140008BD00BF08B5012805D0022814BF00227B
:201440000122114603E04FF000024FF001014FF00100F5F701FA08BD08B501F1FF310329B6
:2014600021D8DFE801F0020B12194BF27820C0F6030007F00DF94FF0000008BD4FF00000B5
:20148000FFF7D8FF4FF0000008BD4FF00100FFF7D1FF4FF0000008BD4FF00200FFF7CAFF71
:2014A0004FF0000008BD4FF0140008BD08B5F5F7EDF94FF001004FF000010A46F5F7CCF900
:2014C000F5F7F0F94FF00C004FF00001F4F7FCFFF5F7DCF908BD00BF037B13B9437B13B9AD
:2014E0000EE0994208D301F1FF318A18437B9A428CBF0020012001E04FF00000C0B2704715
:201500004FF00100704700BF70B4447A24B14FF0320606FB04F610E0C5784AF6EC34C0F6A9
:20152000030454F82550B5F5964F9DBF49F26466B6FBF5F606EB86060826847A24B14FF09A
:20154000320505FB04F501E041F28835C07A18B1FF2808BF012001E04FF0010001B10E6037
:2015600002B1156003B1186070BC704740F2A063C1F200034FF4117202FB00304FF0000116
:20158000C0F810124FF6FF73C0F82C32C0F81812704700BFF8B505460E4640F2A064C1F217
:2015A00000044FF4117303FB0044D4F8240200EB5007F6F75DFBD4F82812421A974202D98F
:2015C000B81AF5F7DBFE23689A6928464FF00101904740F2A060C1F200004FF4117101FBBA
:2015E00005014FF6FF7001F104013246F7F70CFEA31918714FEA10225A7106F10206C4F894
:2016000004614FF00000C4F8080121680B6A28469847F5F7EBFC2846FFF7A8FFF8BD00BFC4
:2016200038B504460D460368F92B08D841F22C10C2F20000185A03F10203236064E0A3F5C4
:201640007A72FA2A0AD841F22C11C2F200018A5C4FEA022003F10103236055E0A3F5FA6090
:20166000262811D84FF0000001460246F5F732F82368A3F5FA6281184978805C40EA01204F
:2016800003F1020323603FE0A3F6B8317C290DD803F10041A1F6B83041F22C12C2F20002C8
:2016A00032F8100003F1010323602DE0A3F57A627C2A0DD803F10041A1F57A6041F22C1253
:2016C000C2F2000232F8100003F1010323601BE0A3F59C50A0F108007C280ED84EF6784100
:2016E000C7F6FF715A1841F22C10C2F2000030F8120003F10103236006E055B14FF0010344
:201700002B704FF0000038BD2DB14FF000032B7038BD4FF0000038BD30B583B004460D4661
:2017200002A840F8084D68460DF10701FFF778FF9DF8073083B904F1FF34651902A941F8BF
:20174000085D68460DF10701FFF76AFF9DF80720101C18BF012001E04FF0010003B030BD70
:201760002DE9F0410D4617461E4640F2A061C1F200014FF4117404FB0010D0F83002037BD8
:20178000FF2B03D1427BFF2A00F09E802C68F92C17D821464FF00202FFF79EFE002800F05B
:2017A0009780002E40F0988041F22C10C2F2000027522B6803F102032B604FF00100BDE804
:2017C000F081A4F57A78B8F1FA0F1AD841464FF00102FFF781FE002800F08280002E40F0B3
:2017E00083804FEA172741F22C12C2F2000202F80870296801F1010129604FF00100BDE8E3
:20180000F081A4F6B8317C291BD804F10041A1F6B8344FEA44014FF00202FFF75DFE002849
:2018200066D0002E68D141F22C10C2F2000020F814702B6803F101032B604FF00100BDE851
:20184000F081A4F57A637C2B1BD804F10044A4F57A644FEA44014FF00202FFF73DFE00283D
:201860004ED0002E50D141F22C13C2F2000323F814702A6802F101022A604FF00100BDE83C
:20188000F081A4F59C52A2F108027C2A40D84EF67848C7F6FF78A0444FEA48014FF0020214
:2018A000FFF71AFE002837D0002E39D141F22C10C2F2000020F81870296801F101012960E2
:2018C0004FF00100BDE8F0814FF00000BDE8F0814FF00000BDE8F0814FF00100BDE8F081B2
:2018E0004FF00000BDE8F0814FF00100BDE8F0814FF00000BDE8F0814FF00100BDE8F08192
:201900004FF00000BDE8F0814FF00100BDE8F0814FF00000BDE8F0814FF00000BDE8F08172
:201920004FF00100BDE8F08130B583B040F2A064C1F200044FF4117505FB0040D0F8300249
:20194000B1F57A7F1BD3A1F57A7163B1837B13B9C37B13B907E0994223D38A1802F1FF3213
:20196000C07B824220D8C8B20DF10701F9F7A4F99DF80710D1F1010038BF002019E04FEAAB
:20198000D10402F107024FEAD20523B121462A46FFF7A2FD58B12819FA288CBF002001202E
:2019A00007E04FF0000004E04FF0000001E04FF0000003B030BD00BF08B5B0F57A7F21D211
:2019C00079B14FEAD00341F22C12C2F2000200F007004FF0010101FA00F0D15C0843D054EB
:2019E00008BD4FEAD00341F22C12C2F2000200F007004FF0010101FA00F0D15C21EA000094
:201A0000D05408BD00F11800C0B24FF00102F9F7CBF908BD10B540F2A064C1F200044FF4B2
:201A2000117303FB0044D4F81C02F5F753FD4FF00000C4F81C0210BD38B54FF4117101FB26
:201A400000F140F2A062C1F200028C18D4F80831D4F80451AB420BD08958E3188A6A1979B8
:201A6000904728B1D4F8080100F10100C4F8080138BD00BF08B540F2A063C1F200034FF48B
:201A8000117202FB0031D1F8082101F10401D1F800319A420BD140F2A061C1F200014FF4D0
:201AA000117202FB0010D0F81C02F5F7D1FA08BD70B582B005468DF8071040F2A064C1F20D
:201AC00000044FF4117303FB0044D4F81802002850D11AB12846FFF749FD4BE0F6F7C8F87D
:201AE000D4F82812431AC4F82802D4F81002D4F82422934204D800F10103B3F5807F04D18B
:201B00002846FFF733FD4FF00103D4F81012621802A911F8010D82F81001C4F81032B4F88F
:201B20002C024FF00102F7F76FFBC4F82C0208BB04F5887694F82032012B03D1304601F0F4
:201B4000F3FA38B994F82012022913D1304600F013F978B14FF00102C4F8182240F2A060D5
:201B6000C1F200004FF4117303FB0505D5F81C02F5F76EFA02B070BD10B541F26343C2F273
:201B800000031B78032B47D840F2A062C1F200024FF4117101FB032340F6E422C2F20002A0
:201BA00052E8001F01F1010142E80014012CF7D018B14FF00100C3F83C0241F26244C2F217
:201BC00000044FF001012170D3F840221AB1D3F81C02F5F73DFA40F6E423C2F2000353E8FC
:201BE000002FA2F1010243E80024012CF7D053E8002FB2F1004F0DD14FF0000243E8002413
:201C0000012CF4D04EF60450CEF20000016841F080510160BFF32F8F10BD00BF10B541F2BB
:201C20006343C2F200034FF004041C70FFF7F2FE10BD00BF2DE9F04F89B005460E4691F84C
:201C4000029009EB49094AF62058C0F6030809EB08074FF4117B0BFB00FB40F2A06AC1F271
:201C6000000A0BEB0A044FF00201F9F7CFFD41F26343C2F200031D70C4F83062304604F57E
:201C8000097104F50D7204F50E73FFF73DFC2846FFF76CFCF5F7ECFFC4F828024FF00100E0
:201CA00000904BF2B840C0F603004FF0040141F6A172C0F603022B46F5F716FBC4F81C0215
:201CC0005BF80A40F2784AF6EC31C0F6030151F8221019F808207B78BE7800964FF0000034
:201CE000019041F63926C0F60306029641F67526C0F60306039641F6B126C0F603060496D5
:201D000041F61D46C0F603060596069064682846A04709B0BDE8F08F08B541F26443C2F2F0
:201D2000000318604FF00100FFF726FF08BD00BF41F26243C2F200034FF000021A70704738
:201D400008B541F26443C2F20003186868B141F26341C2F200010A78032A09D84FF0000041
:201D6000FFF70AFF4FF0000008BD4FF0480008BD4FF0480008BD00BF10B4D0F80031032B1E
:201D800020D94278102A20D890F901404FF0010101FA04F448F2600261F31F4214420CD1DC
:201DA00014F00E0F11D0052B12D9807800F10500834214BF002001200CE0082B14BF00202D
:201DC000012007E04FF0000004E04FF0010001E04FF0000010BC7047072814D840B24FF0A9
:201DE000010303FA00F111F00A0F0FD111F0050F03D111F0F00F03D105E04FF0010070475E
:201E00004FF0040070474FF0000070474FF00200704700BF2DE9F04F83B005460E46174697
:201E20001C464FF0000001460246F4F753FC83463846FFF7D1FF8046002800F0A9800428F8
:201E400005D04FF00100002E00F0A78003E016F0010FF6D09FE0A7F1040A41F22C13C2F21E
:201E600000030193BAF1030F04D8019AA858F7F75BFA8146072F00F28280DFE807F004247D
:201E800016364C5E676FB5F5FA6F08D90BEB0502A2F5FA6108784FEA002323806FE001992B
:201EA000685C4FEA0023238069E0B5F5FA6F06D90BEB0502A2F5FA610B7823805FE0019B34
:201EC000E85C20805BE0B5F5FA6F0AD9A5F5FA618B449BF801009BF8003043EA00222280E1
:201EE0004DE001982A5A228049E0B5F5FA6F0AD9A5F5FA639B449BF800009BF8012042EA8E
:201F0000002121803BE0019BE85A4FEA102242EA0021218033E04FEA19434FEA132040EA6F
:201F20000321234623F8021B1FFA89F24FEA122040EA022161801C4621E0C9F30F412246D8
:201F400022F8021BA4F80290144618E0234623F8029BC9F30F4060801C4610E01FFA89F0DA
:201F60004FEA102141EA0022234623F8022B4FEA19404FEA102141EA002262801C464544E3
:201F800004F10204013E7FF46DAF4FF0010004E04FF0000001E04FF0000003B0BDE8F08F1E
:201FA0002DE9F04F8BB05FFA80FB40F2A063C1F200034FF4117404FB0B344FF000054FF445
:201FC000117000FB0BF1019101F5887640F2A062C1F200020392B71804970BE02668B36986
:201FE00058464FF0000198474FF00100C4F84002F4F7FCFF41F26243C2F2000318780028B9
:020000040803EF
:20200000ECD041F26441C2F200010E68002EE5D04FF00002C4F84022DDF80CA0DDF81090C9
:2020200060E3D4F83C0240B14FF00005C4F83C5241F26441C2F200010D682E78062E00F008
:20204000A4800CD8032E1CD003D8002E00F0AB811AE0042E42D0052E40F0A58167E0802E7A
:2020600000F07F8106D80F2E00F0C080102E40F09A812DE1812E00F08D81822E40F09381ED
:202080007EE14FF008062BE02A79B5F8057002F1FF33B3F5FA6F19D24FEA172040EA0721E1
:2020A00013FA81F6B6F5FB6F13D2019F07EB0A0101F10403687808712E785E706F885F8069
:2020C0004FEA02229A804FF0060104E04FF0FF3101E04FF0FF314FF007065FE14FF00706C8
:2020E0002F79B5F8051007F1FF327C2A19D84FEA112040EA012312FA83F1FA2914D8DDF89A
:20210000048008EB0A0202F1040368781071297859706A885A804FEA07279F804FF00601DF
:202120003CE14FF0FF3139E14FF0FF3136E1A9884FEA112343EA012087B24FEAD702FA2A18
:202140001ED8019E06EB0A0303F10401687818712E784E706B884B8007F007074FF0010023
:2021600000FA07F041F22C16C2F20006B25C0240002A14BFFF2300238B804FF0060101E07B
:202180004FF0FF314FF0060608E1A879FFF724FEAB88024610B34FEA132141EA032080B238
:2021A00000F1FF37BE18FA2E1BD8DDF804C00CEB0A0202F10403697811712F785F706E88A2
:2021C0005E804FF00101AA7903F10403FFF722FE002814BF06214FF0FF3104E04FF0FF31C8
:2021E00001E04FF0FF314FF00706D7E02A791646B5F8053002F1FF30B0F5F66F60D24FEA14
:20220000132141EA0327B9B24FEAD1031818FA2859D8019F07EB0A0808F1040C687888F82D
:2022200004002F788CF801706888ACF802004FEA0227ACF8047002F107004FEAD0078CF860
:20224000067008F10B00002A35D001F007014FF0010202FA01F7079741F22C17C2F20007D7
:20226000964606F1FF31114005910292002A00F0C182BBE2A846029E01E0A846029E012ABE
:2022800004BF00250570FD5C0D4202D00578154305704FEA4101802984BF013371464FEA92
:2022A0004202802A84BF0130724606F1FF35012A40F0E082DBE29CF8061001F1070104E0D7
:2022C0004FF0FF3101E04FF0FF314FF0070665E0E879FFF781FD2979B5F8056001F1FF3301
:2022E0007A2B2DD878B34FEA162242EA0627BAB202F1FF3601FB0063FA2B05D9A2F5FA6751
:20230000262F23D8022824D8019800EB0A0303F104066F781F71287858716F88DF804FEA49
:20232000012018814FEA41079F721046EA7903F10B03FFF76FFD78B1B17901F107010DE0FA
:202340004FF0FF310AE04FF0FF3107E04FF0FF3104E04FF0FF3101E04FF0FF314FF008066F
:202360001CE0B5F801104FEA112242EA012041F2D833C2F200031F6817FA80F6771BBAE1BA
:202380006B784FF0320000FB03F0F4F7F7FF4FF00207B0E16FF001014FF00106AE19B1F131
:2023A000FF3F0ED100E02E464FF0000341F26442C2F20002136041F26247C2F200073B7026
:2023C0008FE1002940F383815846FFF7E3F82068826958464FF00001904794F83872002F31
:2023E00000F07F8107F1FF3E0EF00108D4F83402F4F7C4FF002840F0DA8106E0D4F8340266
:20240000F4F7BCFF002840F0568199F800006B78984240F0668199F8012029788A4240F033
:20242000608141F23020C2F200004FF00001F4F7AFFB2F7807F1FF30032800F23581DFE847
:2024400000F00202595995F804E099F802700EF10702B7EBD20F40F02781B5F805504FEAC4
:20246000152040EA05239FB207F007024FF0010101FA02F14FEAD703BEF1000F00F01481FF
:202480004FF0010041F22C12C2F2000207460EF1FF3C0CEA000C4FF0000599F8038018EAF2
:2024A000000F00F02A812FE109EB050898F803C01CEA000F12F8038014BF41EA080828EA4C
:2024C000010802F803804FEA4000802884BF013538464FEA4101802984BF013339460EF145
:2024E000FF3E09EB050C9CF8038018EA000F00F0408145E199F802202B79B2EB430F40F025
:20250000D380E979072900F2CF8095F907704FF0010000FA07F313F00A0F16D113F0050F42
:2025200003D113F0F00F09D1BEE04FF0020ECDF808E04FF00108CDF814800CE04FF0040C75
:20254000CDF808C0CDF814C005E04FF0020CCDF808C0CDF814C0B5F805004FEA102343EAB2
:2025600000211FFA81F8002A00F09E804FF0000741F22C12C2F200020792CDF820B0099438
:20258000DDF818B01446E87907287AD8DFE800F004140D1D2844536209EB4700B0F8032042
:2025A0004FEA122308F804306BE009EB4703B3F8031008F8041064E009EB4700C2780379E9
:2025C00042EA032128F804105BE009EB4703B3F803104FEA112242EA012028F8040050E033
:2025E00009EB4703B3F8031007F101074FEA112242EA012060F31F4B09EB4703B3F803106D
:202600004FEA112242EA012060F30F0B5846F6F761FE48F8040034E009EB4703B3F8031056
:2026200061F31F4B07F1010709EB4702B2F8030060F30F0BEAE709EB4703B3F8031061F364
:202640000F0B07F1010709EB4702B2F8030060F31F4BDBE709EB4703B3F8031007F10107FB
:202660004FEA112242EA012060F30F0B09EB4703B3F803104FEA112242EA012060F31F4BC2
:20268000C4E70599884407F1010799F802200298131AD9B289F8021000297FF474AF099C29
:2026A000CDF818B0DDF820B041F23020C2F20000F4F77CFB15E007F1FF3202F0FF07D4F86D
:2026C0003402F4F75BFE002840F089809DE611F1020F06D141F26245C2F200054FF00003DD
:2026E0002B70354641F26247C2F200073B78002B7FF497AC7EE4EE19F3E712F8038028EAB7
:20270000010802F8038005E012F8038041EA080802F803804FEA40004FEA4101802984BF29
:2027200001333946BEF1010EBED0BCF1000F3FF4BBAE09EB050C9CF8038018EA000F12F80B
:2027400003C00CBF2CEA010C41EA0C0C02F803C04FEA4000802884BF013538464FEA410135
:20276000802984BF01333946BEF1010E7FF49CAE9AE712F803C02CEA010802F8038005E070
:2027800012F803C041EA0C0802F803804FEA4000802884BF013538464FEA4101802984BF31
:2027A00001333946BEF1010E7FF47EAE7CE707F1FF3111F0FF0794D04FFA88F3002B3FF4F1
:2027C0001DAED4F83402F4F7D9FD00283FF41DAE07F1FF3010F0FF077FF410AE81E707F187
:2027E000FF3111F0FF077FF409AE7AE74FF0000288F80B20FA5C07990A4205D098F80B2059
:2028000002990A4388F80B2007994FEA4101802984BF01337146DDF808804FEA4802013E14
:2028200002963FF448AD059E002E3FF423AD012A04BF0026067017F8038018EA010F04D002
:20284000067842EA060880F800804FEA4101802984BF013371464FEA4202802A84BF0130DB
:202860007246029E013E02967FF407AD23E54FF000060670FE5C0E4202D006781643067076
:202880004FEA4101802984BF013371464FEA4202802A84BF013072466E1E7FF4F0AC45466D
:2028A00009E500BF38B540F2A065C1F200054FF4117404FB005505F10404297162F07F0208
:2028C0006A71AB714FF00301FEF764FE38BD00BF2DE9F04F89B05FFA80FA40F2A063C1F26A
:2028E00000034FF4117404FB0A344FF4117000FB0AF1029101F5887540F2A062C1F20002A7
:20290000039205EB020B2668B76950464FF00001B847F4F76BFBD4F81002D4F81432984287
:20292000F1D094F81011D4F83452A94240F00A8341F23020C2F200004FF00001F4F728F9AC
:2029400094F8112102F1FF360F2E00F2EE82DFE816F010009E000F010F017801C801EC0227
:20296000EC02EC02EC02EC02EC02EC02EC02FB016B02BBF80260BBF804504FEA152343EAB2
:20298000052087B207F1FF32B2F5FA6F09D350469BF800109BF801204FF00303FFF782FF1B
:2029A000CAE24FEA162141EA0626B5B2504629463A464FF00003FEF7B7FF48B950469BF8A1
:2029C00000109BF801204FF00203FFF76BFFB3E2029B0398191801F1040201929BF8006013
:2029E0000E719BF80130019843704FF00008002F44D006E04FF001064FF0000905F101054E
:202A00000BE04FF000084FF00106C14641F22C11C2F20001059104940C4640F2E732954270
:202A20000CD84FEAD500225C05F0070342FA03F111F0010F0ED049EA06090BE005F11803CA
:202A4000D8B207A9F8F738F99DF81C1011B908B149EA060907F1FF374FEA4606802E03D85A
:202A6000002F00F08B82C9E7019A02EB080383F8039008F10108002FBCD1049C019981F868
:202A80000280504608F10301FEF784FD54E2BBF80250BBF804204FEA122646EA0227BEB25F
:202AA00006F1FF31B1F5FA6F09D350469BF800109BF801204FF00303FFF7F4FE3CE24FEA93
:202AC000152343EA052085B2E8B207A9F8F756F89DF81C204AB150469BF800109BF80120F5
:202AE0004FF00203FFF7DEFE26E2029F03997B1803F1040001909BF800201A719BF801701D
:202B0000477056B3AFB24FF000084FF00105C14605E04FF001054FF0000907F10107F8B2E5
:202B200007A9F8F72BF89DF81C1011B908B149EA050906F1FF364FEA4505802D03D8002EE9
:202B400000F02582E9E7019A02EB080181F8039008F10108002EDCD101E04FF00008019FCC
:202B600087F80280504608F10301FEF713FDE3E1BBF802304FEA132646EA032080B2079085
:202B8000BBF804704FEA172242EA0725AEB206F1FF317C2909D950469BF800109BF8012049
:202BA0004FF00303FFF77EFEC6E13146FEF7B4FD48B150469BF800109BF801204FF0020370
:202BC000FFF770FEB8E1029B03981D1805F104079BF800202A719BF8011079703EB34FF07F
:202BE000000806F1FF3303F0010907A84146FEF717FDA7F803004FF00105AE4240F0CF8111
:202C000015E007A84146FEF70BFD07EB4501A1F8030005F1010507A84146FEF701FD07EBA1
:202C20004503A3F8030005F10105AE42E9D14FEA4600C1B2B970504601F10301FEF7AAFCC6
:202C40007AE1BBF80220BBF804504FEA152646EA0527BDB265B1B5F57F4F09D050469BF86E
:202C600000109BF801204FF00303FFF71BFE63E14FEA122141EA02239EB2504631464FF0A0
:202C800001021346FEF750FE48B950469BF800109BF801204FF00203FFF704FE4CE10298A4
:202CA000039900EB01093046B5F57F4F14BF00210121FEF781FE9BF8002089F804209BF820
:202CC000017089F80570BBF80250A9F80650BBF80410A9F8081050464FF00601FEF75AFCEA
:202CE0002AE1BBF802604FEA162747EA06218BB208A941F8043D5046BBF804204FF00003CF
:202D0000FEF72EFD48B950469BF800109BF801204FF00203FFF7C6FD0EE10298039A8518E5
:202D200005F104069BF800702F719BF801107170BBF802307380BBF80400B08050464FF0D7
:202D40000601FEF727FCF7E0BBF80200BBF804704FEA172646EA072295B205F1FF31B1F5BF
:202D6000FA6F06D29BF8063005F10707B3EBD70F09D050469BF800109BF801204FF00303B6
:202D8000FFF790FDD8E04FEA102646EA00201FFA80F8504641462A464FF00103FEF7C4FD22
:202DA00018B1002D40F0D28027E050469BF800109BF801204FF00203FFF774FDBCE00BEB6A
:202DC0000700C17930462940FEF7F6FD4FEA4505802D84BF0137454606F1010630460BEB4B
:202DE0000702D1792940FEF7E7FD4FEA4505802D00F2F780F8E04E45E1D1029D03982A180C
:202E000002F104069BF8007017719BF801107170BBF802307380BBF80450B58050464FF0BC
:202E20000601FEF7B7FB87E0BBF802704FEA172242EA072083B20693BBF804504FEA15214F
:202E400041EA0526B5B25F1907F1FF32079205F1FF307C2809D950469BF800109BF80120E3
:202E60004FF00303FFF71EFD66E0504606A94FF000024FF00103FEF773FC50B1504607A942
:202E80004FF000024FF00103FEF76AFC08B155B934E050469BF800109BF801204FF0020347
:202EA000FFF700FD48E04FF0000705F1FF3808F00109504606A9BBF807203B46FEF750FCA1
:202EC0004FF00106B54240F0928017E00BEB4602504606A9B2F807203B46FEF741FC06F17E
:202EE00001060BEB4603504606A9B3F807203B46FEF736FC06F10106B542E7D1029D0398E6
:202F00002F1807F104069BF800203A719BF801107170BBF802307380BBF80450B5805046DB
:202F20004FF00601FEF736FB06E0504694F810114FF00103FFF7B6FC41F23020C2F20000DA
:202F4000F3F734FF5046FEF711FBDCE49BF80720404602F00101FEF72FFD08F1010608EBB5
:202F600005094FF002054FF000074FF00108C6EB090111F0010F3FF43EAF22E0049C019D43
:202F800005EB080080F8039008F1010876E5019B03EB080080F8039008F10108DFE5B9F1C4
:202FA000000F3FF42EAE07A84146FEF739FB07EB4502A2F8030005F10105AE427FF421AE90
:202FC00035E60BEB0703D97930462940FEF7F4FC4FEA4505802D84BF0137454606F101068C
:202FE00009E707F10107454606F1010603E7B9F1000F3FF46BAF0BEB4603504606A9B3F839
:2030000007203B46FEF7ACFB06F10106B5427FF45DAF73E740F2A063C1F200034FF41172ED
:2030200002FB003393F82032012B0AD140F2A063C1F2000302FB0030C0F834124FF0000027
:2030400070474FF0370070472DE9F04F89B004460D4691F8029009EB49094AF62058C0F692
:20306000030809EB08074FF4117B0BFB00FB40F2A06AC1F2000A0BEB0A064FF00101F8F743
:20308000C5FBC6F83052284606F509714FF000021346FEF739FA20466978FFF7BBFF20462E
:2030A000FEF764FAF4F7E4FDC6F828024FF0010300934BF2C840C0F603004FF0040142F6B9
:2030C000D102C0F603022346F4F70EF9C6F81C025BF80A60EA784AF6EC30C0F6030050F8AF
:2030E000221019F808207B78BD7800954FF00000019041F63925C0F60305029541F675251D
:20310000C0F60305039541F6B125C0F60305049541F61525C0F60305059506907568204653
:20312000A84709B0BDE8F08FD0F80031032B2BD94278102A2BD890F901204FF0010101FABB
:2031400002F212F06E0F06D112F4803F12D112F4004F05D11BE0082B14BF00200120704759
:20316000092B17D9807900F10900834214BF002001207047092B10D9807900F109008342D3
:2031800014BF0020012070474FF0000070474FF0010070474FF0000070474FF0000070478B
:2031A00042F28453C1F200031A78027058780870704700BF42F28453C1F200031B78834273
:2031C0001AD842F28452C1F2000252789A18904215DAC01AC3B242F28452C1F2000202EB06
:2031E000D300027A03F0070342FA03F000F001020A704FF0010070474FF0000070474FF0BB
:203200000000704770B442F28453C1F200031B7883424DD842F28452C1F2000252789A185A
:20322000904248DAC01AC0B200F007054FF0010404FA05F540F6E422C2F2000252E8003FAB
:2032400003F1010342E80036012EF7D042F28453C1F2000303EBD00393F8280028420CBFB6
:2032600000200120087093F8281021EA050583F8285052E8003FA3F1010342E80035012D2C
:20328000F7D052E8003FB3F1004F0DD14FF0000342E80035012DF4D04EF60450CEF2000032
:2032A000016841F080510160BFF32F8F204604E04FF0000001E04FF0000070BC704700BF87
:2032C00042F28453C1F200031A79027058790870704700BF42F28453C1F200039A78027024
:2032E000D8780870704700BF10B442F28453C1F200039B78834237D842F28452C1F2000265
:20330000D2789A18904232DAC01AC3B24FEAD30403F007004FF0010202FA00F359B142F20B
:203320008451C1F20001081990F8482043EA020180F848100AE042F28451C1F2000108192B
:2033400090F8482022EA030280F8482042F28450C1F20000021992F8681021EA030382F829
:2033600068304FF0010004E04FF0000001E04FF0000010BC704700BF42F28453C1F200032F
:203380009B7883421BD842F28452C1F20002D2789A18904216DAC01AC3B242F28452C1F2D9
:2033A000000202EBD30090F8482003F0070342FA03F000F001020A704FF0010070474FF08C
:2033C000000070474FF00000704700BF10B442F28453C1F200039B78834237D842F284520B
:2033E000C1F20002D2789A18904232DAC01AC3B24FEAD30403F007004FF0010202FA00F3B4
:2034000059B142F28451C1F20001081990F8682043EA020180F868100AE042F28451C1F2EE
:203420000001081990F8682022EA030280F8682042F28450C1F20000021992F8481021EA86
:20344000030382F848304FF0010004E04FF0000001E04FF0000010BC704700BF42F28453A4
:20346000C1F200039A790270D8790870704700BF827802F107024FEAE2014FEA410202F151
:203480000102037902EB8301407A0818704700BF70B401F0070400EBD10000F1FF31C4F13A
:2034A000080611F8010F40FA04F00CB9C0B204E04D7805FA06F52843C0B2082B08D8C3F139
:2034C00008034FF0FF0141FA03F31840107005E002F8010BA3F10803DBB2E2E770BC7047D6
:2034E0002DE9F00F9DF82070044618B94BF2DC44C0F6030402F0070C66464FF0FF0000FA74
:203500000CF5E8B201EBD20101F1FF31CCF108094BF2DC48C0F603084A786FB9082B09D841
:203520004FF0010000FA03F000F1FF3505FA06F505F0FF0022EA0002C5B294F800A00AFA96
:2035400006FA05EA0A0A4AEA020201F101018A460A70BCF1000F0DD04B450BDD4A7807B95F
:20356000024094F800B04BFA09FB2BEA05052A438AF80120082B06D9444518BF0134A3F11A
:203580000803DBB2C8E7BDE8F00F704708B504484FF000014FF0400203F0ACFA08BD00BFA2
:2035A0002C27001008B504484FF000014FF0200203F0A0FA08BD00BFAC25001038B54FF0E0
:2035C000000441F26C43C2F200031C6042F28455C1F2000505F1080021464FF4007203F000
:2035E00089FA284621464FF0080203F083FA38BD10B50C4642F28453C1F200039979814218
:2036000017D842F28452C1F20002D379CA18904212DA401AC1B242F28453C1F2000303EB94
:203620008102D2F8A801F5F77FFE20604FF0010010BD4FF0000010BD4FF0000010BD00BFC7
:2036400010B50C4642F28453C1F200031979814217D842F28452C1F200025379CA1890420F
:2036600012DA401AC1B242F28453C1F2000303EB8102D2F8A800F5F757FE20604FF00100EC
:2036800010BD4FF0000010BD4FF0000010BD00BF38B5054642F28453C1F200039C798442B2
:2036A00017D842F28450C1F20000C279A3189D4212DA0846F5F70EFE2D1BEDB242F2845466
:2036C000C1F2000404EB8504C4F8A8014FF0010038BD4FF0000038BD4FF0000038BD00BFFA
:2036E0002DE9F0418AB00446FFF768FF02A84FF000014FF0200203F0FDF94FF0000001A985
:20370000F7F70AF942F28453C1F200039DF804201A709DF8050098709DF8061019719DF848
:2037200007509D714FF000064FF0010841F26C47C2F200071D464AE06078FF2845D14FEA1B
:20374000531203F01F0108FA01F3386808B93C6008E0D8B20DF1280C0CEB820151F8201C5B
:2037600008422FD106F101060AA800EB8202DBB252F8201C43EA010042F8200C2046FFF7DD
:2037800077FE402871D8E37803F107024FEAE2014FEA410000F10100627900EB8200E17981
:2037A0004218402A64D8A078697842186A70E8781B18EB7021796A79881868716179EB79BA
:2037C000CA18EA7104F10A0401E004F105042378FF2BB1D1102E4ED842F28454C1F200045C
:2037E0006279402A4AD842F28450C1F20000C179102946D842F28453C1F200035C783CB194
:2038000040F24420C2F200004FF00101F7F7FAF842F28452C1F20002D07838B140F23C20BF
:20382000C2F200004FF00101F7F718F942F28451C1F200014B793BB140F22C20C2F20000F5
:203840004FF00101F7F736F942F28454C1F20004E279DAB140F23420C2F200004FF00101E6
:20386000F7F754F94FF0000412E04FF045040AE04FF0430407E04FF0460404E04FF00F043A
:2038800001E04FF00E04FFF799FE01E04FF0000420460AB0BDE8F08108B540F24420C2F208
:2038A00000004FF00001F7F7ADF840F23C20C2F200004FF00001F7F7D1F840F22C20C2F2CA
:2038C00000004FF00001F7F7F5F840F23420C2F200004FF00001F7F719F908BD2DE9F8433D
:2038E000044641F26C43C2F20003186884421AD14FF0000541F26846C2F20006357041F2FD
:203900006A43C2F200031D7041F27140C2F20000057041F26946C2F20006357041F2704382
:20392000C2F200031D70E57805F107054FEAE505E8B2667900EB860303F10103C018C6B28C
:20394000964240D842F28458C1F2000841F26842C2F20002177808EB070393F8E8010F46C4
:2039600007F8010B41F27141C2F2000191F8009008F1480049463A46E378FFF789FDEDB2C3
:203980007F1908F1680049463A46E378FFF780FD7A196379CBB141F27045C2F20005287825
:2039A00008F1080101EB80004FF000031946C518D5F8A051D55001F1010103F1040365796B
:2039C0008D42F4D801E04FF000063046BDE8F8832DE9F04782B0044617461E46002973D199
:2039E000FFF746FDC5B2B54270D1A3783E78002E59D041F26842C2F20002117842F2845093
:203A0000C1F20000421892F8E811B1424BD003F107054FEAE50507F1010741F26A40C2F254
:203A2000000090F8009042F2845AC1F2000A4FF00002009238460AF108014A46FFF750FD77
:203A40005FFA85F84744A3784FF00101009138460AF128014A46FFF743FD47442379CBB10D
:203A600041F26940C2F2000090F800C00AF1080101EB8C0C4FF000031A46F9580CEB0300F9
:203A8000C0F8A01002F1010203F1040321799142F3D801E04FF0000205EB42054FEA4502BC
:203AA00002F10102D5B241F26843C2F20003187842F28451C1F200010B1883F8E8614FF081
:203AC000000283F8F82149E04FF0000541F26840C2F20000037842F28451C1F20001CA183A
:203AE00092F8F801FF2839D000F10100C2B242F28451C1F20001CB1883F8F821082A2DD149
:203B000041F26A46C2F2000637788846A3784FF000060096304601F108013A46FFF7E0FCD2
:203B2000A3780096304608F128013A46FFF7D8FC207998B141F26942C2F20002117801F101
:203B4000270108F1080303EB81023346304642F8040F03F1010321799942F8D841F2684371
:203B6000C2F200031A7802F101021A7041F26A40C2F200000178A378CA18027041F271401F
:203B8000C2F200000178E378CA18027041F26940C2F2000001782379CA18027041F270406D
:203BA000C2F2000001786379CA180270284602B0BDE8F08730B40C18FA2C2BD869B341F2EC
:203BC0007443C2F20003196841F22C12C2F20002051B6FEA050303F001050B181B796FEA45
:203BE0000303835400F101039C421AD10FE0C81800796FEA0000985403F10103C81800794C
:203C00006FEA0000985403F101039C42EFD14FF0000004E04FF01A0001E04FF0000030BC41
:203C20007047002DE3D0C81800796FEA0000985403F101039C42DAD1E9E700BF10B503680F
:203C4000B3F1FF3F1FD04CF20002C0F6000290421FD211466FEA0003D218C2F3002200F56F
:203C600080700368B3F1FF3F1DD10CE000F5807318461A68B2F1FF3F05D003F5807003685C
:203C8000B3F1FF3F1CD14CF20001C0F60001884208D348F20004C0F6000420460A49EFF723
:203CA0009DFB204610BD8842F3D2002ADED000F580700268B2F1FF3FE5D08842D6D3E8E7AB
:203CC0008842D3D3E5E700BFFFBF00082DE9F041C0B080460F4614461E460D18FA2D5BD814
:203CE000684641F27443C2F2000319684FF4807202F0DCFEF7B141F22C17C2F200074FF0DB
:203D0000000EC5EB08026FEA020000F00102002C4DD146E024B9CA5D6FEA0200C3B200E069
:203D2000734600AA5018037101F101010A46002C5CD156E041F27441C2F20001086800F173
:203D4000040001A94FF0FA0202F05AFAF0B141F27444C2F200042068FFF770FF20604FF044
:203D6000000300934FF6FF7001A94FF0FA02F5F74BFAADF8FE00684621684FF48072EFF7EE
:203D800099FBD0F1010038BF002001E04FF0010030704FF0000001E04FF01A0040B0BDE8E7
:203DA000F08118F807106FEA0100C3B200E0734600A901EB0800037108F101018D42B9D09F
:203DC000002AA7D024B9CB5D6FEA0300C2B200E0724600AB5818027101F101018D4299D11A
:203DE000A8E7C85D6FEA0003DBB200E0734600A88218137101F101018D428BD19AE700BF68
:203E000041F27843C2F200031860704738B541F27843C2F200031868002860D14CF2000124
:203E2000C0F6000148F20002C0F600028A4256D04BF21450C0F60300FFF7E2FF48F2000476
:203E4000C0F60004D4F80031B3F1FF3F25D033483349814226D201F58073324DEA1A4FEA7D
:203E6000122404F1010004F001051C46D3F80011B1F1FF3F34D119E01C46D3F80011B1F120
:203E8000FF3F13D002F1010203F580731C46D3F80011B1F1FF3F3AD108E048F20004C0F61B
:203EA000000403E048F20004C0F600042068B0F1FF3F0FD04FF6FF7004F104014FF0FA02F4
:203EC000F5F7A2F9B4F8FE20824203D02046FFF7B5FE044641F27441C2F200010C6038BDA3
:203EE0004FF0000202F1010203F580738242DDD0002DC1D01C46D3F80011B1F1FF3FD5D0AE
:203F000002F1010203F580738242B5D1CEE702F1010203F580738242AED1C7E700C0000827
:203F200000800008FFC000084FF0000313704FF014007047012914BF14200020704700BF9C
:203F400008B54CF285004BF21C51C0F6030141F27C42C2F20002F6F73FFD08BD10B584B0EF
:203F60001446022902D003291CD113E06846EEF7D3F8024640F2CE40C0F2B7006946F5F7F4
:203F800065F907EE100AF8EE477AC4ED007A4FF0000009E01046EEF7F1FF00280CBF152067
:203FA000002001E04FF0140004B010BD10B582B01446B9B94FF0000001A9F6F7ADFC4FF0AB
:203FC000040384F8FB309DF8040020709DF8051061709DF80620A2709DF80730E3704FF064
:203FE000000001E04FF0140002B010BD10B58CB01446062949D8DFE801F004111F2A4848BD
:020000040803EF
:20400000370040F20023C0F6000393F84600107093F8471051704FF0000038E006A84FF023
:204020000001F6F779FC9DF8291021709DF82A2062704FF000002AE005A8F6F7BFFC059BCF
:204040004FEA1320207063704FF000001FE040F20020C0F60000B0F848104FEA112222704D
:2040600061704FF0000012E001A8EEF755F8024605904FF6FF7001A9F5F7C6F84FEA102312
:20408000237060704FF0000001E04FF014000CB010BD00BF10B5144692F8FB20FB2A28BF32
:2040A000FB2284F8FB206AB34FF00100187011B1814221D10DE04FF6FF70214694F8FB2041
:2040C000F5F7A2F84FEA10216170A0704FF0000010BD40F2CE40C0F2B700214694F8FB204C
:2040E000F5F7B4F84FEA104363704FEA1022A270E0704FF0000010BD4FF0000119704FF0E8
:20410000140010BD4FF0160010BD00BF10B51446032929D8DFE801F002080C20EDF7F6FFCA
:2041200020704FF0000010BD4FF00000107010BD41F29023C2F20003196840F6F072C1F2EE
:2041400000024FF0540000FB0123196A4FEA410222704FF0000010BD4FF00000F6F72EFCB8
:2041600020704FF0000010BD4FF0140010BD00BF08B5012914D021B1042914BF14200020D3
:2041800008BD082A20D84FF0FF304BF25053C0F6030353F82210F7F7BFFB4FF0000008BDFD
